:100000005446495300010000E0E30200278FFCDC66
:10001000177101031903251544563259177101014F
:100020001903251444563259177101011903251576
:100030004456325903000000000000000000000098
:100040005446435300200000C89F020000000000F7
:100050000080011001210000252100005915020037
:10006000292100002B2100002D2100003D2100004E
:100070003D2100003D2100003D2100002F21000016
:10008000312100003D21000033210000D16D00002E
:100090009B710000372100003D21000081610010AC
:1000A00037210000CB4E0000CF4E0000CB70000087
:1000B000372100000F6A000001610000D34E0000EC
:1000C000C967000037210000372100001D5C0000D7
:1000D0000000000000000000000000000000000020
:1000E0000000000000000000000000000000000010
:1000F0000000000000000000000000000000000000
:1001000000000000000000000000000000000000EF
:1001100000000000000000000000000000000000DF
:1001200000000000000000000000000000000000CF
:1001300000000000000000000000000000000000BF
:1001400000000000000000000000000000000000AF
:1001500000F003F800F020F8FEE70D480168890878
:100160008900002001C101C101C101C17047000027
:100170009C6A0010FEE7FEE7FEE7FEE7FEE7FEE70B
:10018000FEE7FEE7FEE703480047FEE7FEE7000064
:10019000202100003D21000000F002F800F068F886
:1001A0000AA090E8000C82448344AAF10107DA45D2
:1001B00001D100F05DF8AFF2090EBAE80F0013F0BC
:1001C000010F18BFFB1A43F0010318476831020002
:1001D000C83102000A444FF0000C10F8013B13F044
:1001E000070408BF10F8014B1D1108BF10F8015B90
:1001F000641E05D010F8016B641E01F8016BF9D183
:1002000013F0080F1EBF10F8014BAD1C0C1B09D1D9
:100210006D1E58BF01F801CBFAD505E014F8016B4B
:1002200001F8016B6D1EF9D59142D6D370470000DD
:10023000103A24BF78C878C1FAD8520724BF30C812
:1002400030C144BF04680C607047000000230024E4
:1002500000250026103A28BF78C1FBD8520728BFD6
:1002600030C148BF0B6070471FB51FBD10B510BD32
:10027000DFF80CD0FFF7F8FF07F084F81FF086F9DD
:100280000080011003B4FFF7F1FF03BC1FF086F9F3
:1002900008B500200346024600900121022000F02C
:1002A000D6FA08BD38B5FF4D0024FF48EC802C81FC
:1002B0006C81406980476861FF202871FB480023FA
:1002C0001A46046044608460C4600461012068715F
:1002D0002C7001460220009400F0B9FA012038BDCC
:1002E00038B5F04D02282C7922460DD0052810D0C3
:1002F000A24208BF38BD00200346024621460090B6
:1003000000F0A5FA2C7138BD022914BF0124022483
:10031000EEE7022914BF04240824E9E708B5009396
:1003200013460A460146012000F091FA08BD08B5BF
:100330000346009103220221012000F088FA08BD43
:1003400038B500240DF050FE002818BF012412F02B
:10035000C5FA002818BF0224D2480178A14208BF7C
:1003600038BD047000200346022100902246084652
:1003700000F06DFA38BD38B5CA4D04466878A04221
:1003800008BF38BD07F018F86C70002C0CBF0521B1
:1003900006210020034602460090022000F057FA92
:1003A00038BD08B500210B46024600910721022006
:1003B00000F04DFA08BD08B500210B460246009139
:1003C0000821022000F043FA08BD08B50021009181
:1003D000002814BF0122002200230321022000F084
:1003E00036FA08BD08B500200346024600900421F5
:1003F000022000F02CFA08BDAA490120887070473D
:10040000A84880787047A7490020887070472DE978
:10041000F04104460127002503F00700A14E88465D
:10042000012804BF0020708148D0022846D170897D
:100430009D4904280BD2002818BF306902D14868B2
:100440008047306110F8011B217030612FE00628D1
:1004500009D288688047718980B2C1F10501C9005D
:10046000C840207023E0082808D2086980477189B5
:10047000C1F10701C900C840207018E00C2808D25B
:10048000486980477189C1F10B01C900C8402070DB
:100490000DE00E2808D2886980477189C1F10D01ED
:1004A000C900C840207002E0FF202070002770893A
:1004B000401C80B270810E2828BF012588F80050AA
:1004C0003846BDE8F08130B403F007000024DFF8BF
:1004D000D4C1012804BFACF80640ACF80A401BD0D8
:1004E00013F0070F18D16F4BBCF80A00DB88022805
:1004F00005D2120242EA1322ACF8062009E00344B6
:100500009D1EB5F5806F04DADCF814502B4403F817
:10051000022C401CACF80A000C7030BC0020704764
:10052000F0B40746002003F007045E4D0646012C98
:1005300004BF6E81EE6025D0DFF868C1022CBCF8E4
:1005400008C003D013F0070F0DD01BE06A890CEB35
:100550000203B3F5806F15D26869C05C3870501C17
:10056000688101200EE0120242EA1C222A81EB6817
:10057000012B05D1B2F5806F24BF40F2FF322A81F2
:100580005A1CEA600E70F0BC704738B503F00700E3
:1005900000240D46012809D1424800231A4644810F
:1005A000C48019460220009400F051F92C700020FC
:1005B00038BD70B50C0082B04FF0000100F0DC8057
:1005C00025783B4B012D18BF022D04D0032D50D0B0
:1005D000002D66D09BE06278A2F1010C00EB0212C4
:1005E00002F810CC627800EB021202F80F5C1A6875
:1005F000B4F802C0D68C528C0CFB06FC9CFBF2F2C9
:1006000094F801C000EB0C1C2CF80E2C1A68B4F8FE
:1006100004C0938C128C0CFB03F393FBF2F263780F
:1006200000EB031323F80C2C6378A27900EB03137F
:1006300023F80A2C6378227A00EB031323F8082CA2
:100640006378627A00EB031323F8062C6378A27BAD
:1006500000EB031323F8042CE279052A08BF0121DB
:100660006278002D00EB021000F8021C4FD102B09E
:1006700070BD6278A2F1010C00EB021202F810CCFE
:1006800094F801C0032200EB0C1C0CF80F2C1A6824
:10069000B4F802C0D68C528C0CFB06FC9CFBF2F228
:1006A00008E069E000840010A45102006489001091
:1006B000F488001094F801C000EB0C1C2CF80E2CF0
:1006C0001A68B4F804C0938C128C0CFB03F393FBF0
:1006D000F2F2637800EB031323F80C2C627800EB42
:1006E000021222F80A1C627800EB021222F8081C9F
:1006F000627800EB021222F8061C627800EB02120C
:1007000022F8041C627800EB021000F8021C012D94
:1007100018BF032D05D00DF06AF9002804BF02B000
:1007200070BD06F049FE05281CBF02B070BD012D4A
:1007300004BFC0208DF8000005D0022D0CBFC220E0
:10074000C1208DF8000060788DF8010060880123D9
:10075000000A8DF80200A0788DF80300A088062218
:10076000000A8DF8040020798DF8050069460720FD
:1007700010F06BFF02B070BD01704170418081804C
:10078000C180018141818181817302B070BD354991
:100790000020C87070473348C07870473149012045
:1007A000C8707047304B03EB80004254704700B56F
:1007B00085B001788DF8001041788DF801108178AE
:1007C0008DF80210C1788DF8031001798DF80410AE
:1007D00041798DF8051080798DF8060000208DF89C
:1007E00007000290039006F007FF01280CD11EF0CD
:1007F000EBFE012801BF9DF8000046289DF801008E
:10080000012804BF05B000BD68461EF0E2FE05B039
:1008100000BD70471349002818BF01204871704778
:10082000104840797047012818BF70470F480129C8
:1008300004BF416841F4007105D0002906BF41683A
:1008400021F400717047416070470948704708B54E
:10085000DDF808C0CDF800C0DFF818C0DCF800C033
:10086000E04708BD008400106489001000100040BB
:10087000784C0200A45102007047F648D0F85003AB
:1008800000F00100704770B5F24D04000AD002F08C
:1008900067FA38B9D5F8500310F0010F1CBF0020DB
:1008A000A86005D10120A860002C08BF00202DD031
:1008B000D5F8600310F0010F0BD1D5F8600340F0BC
:1008C0000100C5F86003D5F8600320F00100C5F809
:1008D0006003E148016811F0010F07D1016841F0A0
:1008E00001010160016821F00101016004F02CFBAD
:1008F00000281CBFD5F8500310F0010F05D004F0FC
:100900001DFB002818BF04F02BFB0120286270BDDE
:10091000D048006A002818BF01207047C00000F1CD
:10092000804000F5A04041637047C00000F1804066
:1009300000F5A040006B00F4807070471021C000EB
:1009400000F1804000F5A0404163704730B4820957
:10095000C24B00F00F0000EB400053F822404FF470
:10096000847505EB8015D1F800C044F805C053F834
:1009700022204FF4867303EB80104968115030BC7D
:1009800070478209B54850F82200D0F8402161F341
:100990000D22C0F840217047B049800951F820006D
:1009A000D0F84001C0F305207047AA49D1F8402192
:1009B00060F31742C1F840217047A648D0F84001C3
:1009C000C0F3074070474FF4A072C0F3011302EB6D
:1009D0008312DFF888C200F00F03800903EB4303A2
:1009E0005CF82000002900EB8310815814BF41F00F
:1009F000010121F0010181507047984A810952F8A4
:100A0000212000F00F0101EB410102EB8111C0F345
:100A100001104FF4A07202EB8010085800F00100A2
:100A200070478E4A810952F82110D1F8E01100F088
:100A30000F00012201F0070102FA00F0084018BF80
:100A4000012070474FF4A072C0F3011302EB831230
:100A5000DFF808C200F00F03800903EB43035CF8E2
:100A60002000002900EB8310815814BF41F00201DF
:100A700021F0020181507047784A810952F8212003
:100A800000F00F0101EB410102EB8111C0F30110F5
:100A90004FF4A07202EB80100858C0F3400070477A
:100AA00081096F4A01EB410102EBC10100F00F0225
:100AB00001EBC201C0F3011051F8200070476849F2
:100AC00082091CD00122B2EB901F18BF7047654805
:100AD0000068C0F30800886163480268C2F30842F6
:100AE0000A620068C0F30800486260480268C2F306
:100AF00008428A620068C0F30800C862704755481F
:100B0000D0F82421C2F308020A60D0F8E421C2F32D
:100B100008428A60D0F8E421C2F30802CA60D0F823
:100B2000A422C2F308420A61D0F8A402C0F308006C
:100B3000486170472DE9F0030122830900F00F019D
:100B4000C0F3011CC0F3011622EA0C0C00290BBFF4
:100B500002254D1E00224FEA0C124FF0080404EB50
:100B6000CC043F4F03EB430C07EBCC0C0CEBC10167
:100B7000DFF8E88051F826604FF4587C58F82310CD
:100B80000CEBC50551F805C000F00F001CF0010F7B
:100B900000EB40004FF4927C0CEB801C40F2FF17FE
:100BA00029D02C48D0F844034FF032090005000D3D
:100BB00006FB09F60EBF0120B6FBF0F0401CFF2833
:100BC00088BFFF204E594FF0FF0909FA04F9C0B25F
:100BD00026EA0906A0403043485158F8230050F84F
:100BE0000C3007FA02F123EA0102114340F80C101D
:100BF000BDE8F003704751F80C0007FA02F3984380
:100C0000C6F3080303FA02F2104341F80C00BDE8F2
:100C1000F003704710B50020FFF78CFF0120FFF7AD
:100C200089FF1120FFF786FF0220FFF783FF1220C4
:100C3000FFF780FF4020FFF77DFF4120FFF77AFF9D
:100C40005120FFF777FF4220FFF774FFBDE8104007
:100C500052206FE700500040605B0040944C02005F
:100C6000188A001024590040E4590040A45A00405A
:100C70002DE9F04707464FEA9016FF480D0050F85F
:100C800026404FF000002062C4F84001C4F8000282
:100C9000C4F84002C4F8C002C4F8000308BFBDE8AD
:100CA000F08728682060686860606168012000291A
:100CB00008BF6060F1490860A868A060E868E0606B
:100CC0002869A0616869E061E8696062286AE06299
:100CD00021206063E063686A2064A86A6064E86A4F
:100CE000A064286BE064686B2066A86BA066E86B64
:100CF0006067286CA067686CE067A86CC4F8800027
:100D0000E86CC4F88400286DC4F88800686DC4F8E5
:100D10008C00A86DC4F89000E86DC4F8A400286E9B
:100D2000C4F8A800686EC4F8AC00A86EC4F8B0009F
:100D3000E86EC4F8B400286FC4F8B800686FC4F84F
:100D4000BC004FF0FF30C4F8E400A86FC4F8F00016
:100D5000E86FC4F8F400D5F88000C4F8FC004FF444
:100D6000107205F1840104F580701EF037FCD5F88F
:100D7000C40220F48030C4F84003D5F8C802C4F897
:100D80004C03D5F8CC02C4F85003D5F8D002C4F80F
:100D90005403D5F8D402C4F85803D5F8D802C4F8DF
:100DA0005C03002005EBC002D2F8DC3204EBC0018A
:100DB000C1F86033D2F8E022C1F86423401C032854
:100DC000F0DBD5F8F402C4F87803D5F8F802C4F8DB
:100DD0007C03D5F8FC02C4F80004D5F80003C4F87D
:100DE0000404D5F80403C4F80804D5F80803C4F8CB
:100DF0000C04D5F80C03C4F810040022002104EB05
:100E0000C20805EBC20000EB8103D3F8109308EB96
:100E1000810CCCF83094D3F83893CCF85894D3F8AC
:100E20006033CCF88034491C0229ECDB05EB8200EE
:100E3000D0F8883304EB8201C1F8A834D0F89C3391
:100E4000C1F8BC34D0F8B003C1F8D004521C052A54
:100E5000D4DB002E14BF8A488A48006830F0FF01B6
:100E600005D1D4F8901060F30301C4F89010D4F8C1
:100E7000500320F00100C4F85003D4F8600320F0C0
:100E80000100C4F86003D4F8680320F00100C4F83E
:100E90006803D4F8700320F00100C4F870033846EA
:100EA000BDE8F0470BE67848007870477648407810
:100EB00070477549887070477348807870477349E8
:100EC000D1F8542360F30902C1F8542370476F48E6
:100ED000D0F85403C0F3090070476B49486070476D
:100EE000694840687047684988607047664880680C
:100EF00070476549C86070472DE9F05F04460027D8
:100F0000384614F4803F18BF012014F4003F18BF86
:100F100040F0040014F4802F18BF40F0020014F4D5
:100F2000002F18BF40F0100014F4001F18BF40F04D
:100F3000400014F4800F18BF40F0080014F4000FB4
:100F400018BF40F02000DFF84081DFF8409198F8AA
:100F5000021010EA0105D9F8400320F48030C9F8E6
:100F6000400336D0D8F80C60D9F84803002740F089
:100F70000100C9F84803D9F8480320F00100C9F876
:100F80004803D9F8400340F48030C9F840034FF0DB
:100F9000630ADFF8FCB016E004F01DF95046D9F8FA
:100FA000481311F0010F0AD0D9F844030005000DD1
:100FB0001CBFBBFBF0F0C8F80800012703E0011ECE
:100FC000A0F10100EBDC301EA6F1010601DD002FCF
:100FD000E2D0D9F8500320F00100C9F85003D9F845
:100FE000600320F00100C9F86003D9F8680320F01D
:100FF0000100C9F86803D9F8700320F00100C9F8AE
:101000007003244A106820F0010010602248016833
:1010100021F00101016021490B6823F001030B60FD
:10102000F7B315F0010F05D0D9F8503343F00103A1
:10103000C9F8503315F0040F05D0D9F8703343F0D8
:101040000103C9F8703315F0020F05D0D9F86033E9
:1010500043F00103C9F8603315F0100F05D0D9F83B
:10106000683343F00103C9F8683315F0400F19D015
:101070000B6843F0010314E0944C02000458004054
:10108000F0FE0400E0FE0400188400100050004050
:1010900080F0FA02605B0040685B0040705B0040DB
:1010A0001AE00B6015F0080F03D0116841F0010140
:1010B000116015F0200F03D0016841F001010160BB
:1010C00088F80150012088F80000D9F8400340F466
:1010D0008030C9F8400321E0002088F80100ADB15C
:1010E000022088F80000D9F8400340F48030C9F8A5
:1010F0004003D9F8480340F00100C9F84803D9F883
:10110000480320F00100C9F8480307E0D9F840136C
:1011100021F48031C9F8401388F80000D9F8400163
:1011200014F0010F20F00D0018BF40F0010014F082
:10113000040F18BF40F0040014F0020F18BF40F075
:101140000800C9F84001D9F8000214F0100F14BFCC
:1011500040F0010020F00100C9F80002D9F8400277
:1011600014F0200F14BF40F0010020F00100C9F876
:101170004002D9F8C00214F0400F14BF40F0010043
:1011800020F00100C9F8C002D9F8000314F0800F64
:1011900014BF40F0010020F00100C9F80003FF482F
:1011A00014F4805F016814BF41F0010121F00101D6
:1011B0000160FB4814F4005F016814BF41F00101B5
:1011C00021F001010160F74814F4804F016814BF59
:1011D00041F0010121F001010160F34814F4004FD6
:1011E000016814BF41F0010121F001010160EF49E4
:1011F000086814F4807F20F00D0018BF40F0010053
:1012000014F4806F18BF40F0040014F4007F18BF7E
:1012100040F0080008600020FFF78CFC0120FFF779
:1012200089FC1120FFF786FC0220FFF783FC1220C7
:10123000FFF780FC4020FFF77DFC4120FFF77AFCA0
:101240005120FFF777FC4220FFF774FCBDE8F05F08
:1012500052206FE42DE9F04F840900F00F0343EAB8
:101260008411D34D4FEA911CC1F3011855F82C603D
:1012700003EB430C06EB8C174FF4A07606EB8818B3
:10128000024657F80870002017F0010F10D141F006
:1012900010018F09C1F3011155F8277006EB811178
:1012A00007EB8C17795811F0010F08BFBDE8F08FDC
:1012B00055F82410CF6907F0080801EB8C17D7F810
:1012C0000011DFF8F0A204EB440C0AEBCC0C1FFA7F
:1012D00081F902F00F05002103EB43060CEBC50575
:1012E000C2F3011A43EA011242EA8412DFF8C0C2D3
:1012F000C2F3811B5CF82BC0C2F3011B4FF4A07238
:101300000CEB861C02EB8B125CF8022012F0010F32
:101310001AD007EB811C55F82A20DCF844B1B8F14B
:10132000000FCBF3080B0EBF4FF0000CDCF844C1EC
:10133000CCF3023C02EBC20E0EEB021200EB4200B9
:101340000BFA0CF202FB0900491C0229CAD3BDE8C2
:10135000F08F2DE9F0418509AA01954893090024F1
:1013600050F82300D0F8401111F0010F34D0914E05
:1013700003EB430306EBC30302F00F0603EBC603C4
:10138000C2F3011211F0040F53F82220D0F80031FB
:1013900001F0080C9EB2D0F84431C3F3080318BF23
:1013A000C1F30744C769C1F3052117F0080F1ABF3D
:1013B000D0F84401C0F302300020BCF1000F18BF88
:1013C000491C03FA00F001FB004002EBC20170432C
:1013D00001EB021100EB4104012040EA8510FFF708
:1013E00039FF0646022040EA8510FFF733FFA119B6
:1013F0000844BDE8F08110B50020FFF7AAFF4FF4C4
:101400007A7148434CF25031B0FBF1F010BD6A489C
:101410004068C0F30C00704770B504460020FFF729
:1014200098FF05464020FFF794FF35B3624BB0B1FB
:1014300041F288310844A84211D9421B186800F0D3
:101440001F0104FB01F000EBC00C0CEB0010B2EB31
:10145000400F04D932204843B2FBF0F0441CB4F5ED
:10146000005F28BF41F6FF7402D2002C08BF0124A0
:10147000586864F30C00586070BDB4F5005F28BF75
:1014800041F6FF7402D2002C08BF01244B480168CA
:1014900064F30C01016070BD2DE9F041464F064632
:1014A000386810F01F0508BF01250020FFF751FF25
:1014B000DFF80C810446002E18BF002C3FD04149B4
:1014C00000204A68002A08BF01223309B3FBF2F169
:1014D000D7F850C31CF0010F1BD0B3EB420F1DD344
:1014E0003949B1FBF2F3B6FBF2F10A09B3FBF4F1AF
:1014F000102928BF0F218A4298BF114639B101290E
:1015000084BF01FB1430B0FBF1F007D908E00121E2
:1015100009E0B8FBF6F2A24288BF101B0029F6D002
:10152000102988BF0F21D7F85C2361F30302C7F8A5
:101530005C2332216943B0FBF1F0FFF76DFF78685F
:10154000C0F30C00684300EBC00101EB001004EB9A
:101550004000B8FBF0F0BDE8F08170B5164D0024F6
:10156000D5F8500310F0010F08D01648D5F85C13D9
:10157000406801F00F01484304012DE00020FFF70F
:10158000E8FE02462868696800F01F00C1F30C01FC
:10159000414301EBC10000EB011017E0005A00408D
:1015A000405A0040C05A0040005B00404059004093
:1015B000944C0200188A001000500040045800406B
:1015C0000008AF2F1884001080F0FA0212EB4000E0
:1015D0001CBFFE49B1FBF0F4204670BD002818BFC7
:1015E0000120FB49D1F85C2360F30302C1F85C23BE
:1015F0007047F748D0F85C0300F00F00704781098E
:10160000F44A00F00F0000EB400052F821104FF4B4
:10161000807202EB80100858EF4980B2B1FBF0F005
:10162000401C400870472DE9F041EA4B8209DFF881
:10163000A8C353F8223000F00F0731B1BCFBF1F121
:10164000491C4A08B2F5004F01D347F6FF72BCFBB4
:10165000F2F1491C4D08D3F880104FEA520C01F00A
:101660000704D3F88010DB4B4FEA9018C1F3031640
:1016700000F00F0153F8283001EB410103EB811119
:101680002FB3D1F80431F61C74439BB2A2EB44048F
:10169000D1F8006124F0010462F30F06C1F8006183
:1016A000D1F800216CF31F42C1F80021D1F80421C8
:1016B00063F30F02C1F80421D1F8182164F30F027B
:1016C000C1F8182101F090F82846BDE8F081F61C19
:1016D000ACF10E037443A3EB4404D9E78109BD4A7E
:1016E00000F00F0000EB400052F821104FF4807220
:1016F00002EB80100858000C7047830910F00F02AD
:10170000B44850F8230002EB420300EB8313D3F8F4
:1017100000C161F31F4CC3F800C118BF7047D0F877
:10172000802002F00703D0F88020C2F30312D21CFD
:101730005A430E39A1EB4202D0F8043122F00102E3
:1017400061F30F03C0F80431D0F8181162F30F01F0
:10175000C0F8181170479F4A810952F8212000F003
:101760000F0101EB410102EB8111C0F301104FF4B5
:10177000A27202EB80100858C0F308007047F0B462
:10178000944B840900F00F0C53F824300CEB4C05FB
:1017900003EB8516C0F30112D6F81C5106EB821636
:1017A0004D1BD6F8447161F30807C6F844714CEA42
:1017B000021141EA841101F00F02C1F3011101EBA2
:1017C0004201864A03F5C07352F821104A08C9073E
:1017D00053F822C0C90E40F2FF148C402CEA040CCE
:1017E000AD1EC5F3080404FA01F14CEA010143F807
:1017F0002210F0BC00F0F8BF830900F00F01C0F325
:101800000112744850F82300C36901EB410100EB59
:10181000811013F0100FD0F8281100EB8210C9B21C
:10182000D0F84401C0F3080008BF0021401A0004AA
:10183000000C08BF0120704703091B0203EB810164
:1018400001F1405101F500310007C00E0B6802FAAA
:1018500000F01843086070470209120202EB810190
:1018600001F1405101F5003100070968C00E21FA6D
:1018700000F000F00300704770B4DFF858C182092F
:1018800000F00F035CF8225003EB4303C0F3011098
:101890004FF4A87605EB831506EB80160C68AC5167
:1018A0005CF82220496802EB83124FF4AA7303EB21
:1018B0008010115070BC704730B4DFF818C1820935
:1018C00000F00F035CF8224003EB4303C0F3011068
:1018D0004FF4A87504EB831405EB801564590C6074
:1018E0005CF8222002EB83124FF4AA7303EB801002
:1018F0001058486030BC7047364910B4820983B034
:1019000051F8222000F00F0101EB410102EB81119F
:10191000C0F301104FF4A87202EB80128A580092B3
:101920004FF4AA7202EB8010085801900020014683
:101930006A4601234FEA511C01F01F0452F82CC0E3
:1019400003FA04F41CEA040F18BF401C491C2629A2
:10195000F0D303B010BC704730B4002210F00F0F6A
:1019600006D000F00F02C0F3011303EB4202521E37
:10197000184B80094FF4866553F8204005EBC205EB
:10198000D1F800C044F805C053F8200040F23443B9
:1019900003EBC2024968815030BC704710B400228A
:1019A00010F00F0F06D000F00F02C0F3011303EB8D
:1019B0004202521E074B80094FF4866453F820C040
:1019C00004EBC2045CF804C00AE000000008AF2F7A
:1019D00000500040944C0200A08601009C4C020084
:1019E000C1F800C053F8200040F2344303EBC202B8
:1019F0008058486010BC7047FE48C068704700229D
:101A0000FD49830951F82310CB6913F0080F0ED05C
:101A100000F00F0202EB420201EB8211C0F3011051
:101A20004FF4A27202EB80100858C0F30232104645
:101A30007047DFF8C4C310B482095CF82230DC6957
:101A400044F00804DC615CF8223000F00F0202EB85
:101A5000420203EB8212C0F301134FF4A27000EBB9
:101A60008310135861F30E33135010BC70470022DB
:101A7000E149830951F82310CB6913F0080F0ED008
:101A800000F00F0202EB420201EB8211C0F30110E1
:101A90004FF4A47202EB80100858C0F302421046C3
:101AA0007047D54A830952F8233000F00F0202EB49
:101AB000420203EB8212C0F301134FF4A47000EB57
:101AC0008310135861F3124313507047042988BFE1
:101AD00070472DE9F0030027DFF81C83840958F8CC
:101AE0002430DA69C0F3011C12F0080F4FF4A2721F
:101AF00002EB8C1C00F00F0202EB420205D003EB5C
:101B0000821555F80C50C5F30237DD69002615F033
:101B1000080F4FF4A475C0F3011005EB801504D035
:101B200003EB82104059C0F30246C91B7018042809
:101B300003DD081A011D042003E00028BCBF014496
:101B400000207E18D96941F00801D96158F82410A5
:101B500001EB821151F80C3066F30E3341F80C3072
:101B600058F8241001EB82114A5960F312424A518D
:101B7000BDE8F0037047A04A8009002952F8200010
:101B8000816914BF41F0080121F0080181617047AB
:101B90009949800951F820008069C0F3C00070475E
:101BA000954A8009002952F82000816914BF41F04C
:101BB000020121F00201816170478F49800951F8CB
:101BC00020008069C0F3400070478B4B820953F8B6
:101BD000223000F00F0202EB420203EB8212C0F34C
:101BE00001104FF4A67303EB801011507047824A26
:101BF000810952F8212000F00F0101EB410102EBB5
:101C00008111C0F301104FF4A67202EB8010085846
:101C10007047784A10B4D2F8400110F0010F0BD091
:101C2000D2F84C01D2F844110028C1F302311EBF92
:101C30000029C043C2F84C010123002003EB4301FB
:101C40008C0104EB801101F1804101F5A041D1F834
:101C5000402112F0010F0CD0D1F84C21D1F844C131
:101C6000002ACCF3023C1EBFBCF1000FD243C1F8E6
:101C70004C21401C0228E4D35B1C032BDDD310BC99
:101C8000704700225C49830951F82310CB6913F097
:101C9000080F0ED000F00F0202EB420201EB82119E
:101CA000C0F301104FF4A47202EB80100858C0F387
:101CB000005210467047012070472DE9F04F82B066
:101CC000022ADDE90B49DDF8348026BF921E4FEA77
:101CD000520C4FF0000C022B26BF9A1E5308002313
:101CE000464AA2FB04421709B8F1000F14BF0122B3
:101CF00000220192B9F1020F16BF5FEA09024FF00C
:101D0000010B4FF0000B82093B4C00F00F0606EB75
:101D1000460554F822404FF4B27E04EB851AC0F316
:101D200001140EEB841ECDF800A05AF80EA061F34A
:101D30005C6A6BF3186A05D167F3174A63F3CA1A32
:101D40006CF3C60A019969F3420A61F3000A00992B
:101D5000DFF8A49041F80EA059F822204FF4B47196
:101D6000C0F3011A01EB8A1102EB8512B8F1000FE2
:101D7000555814BF45F0800525F0800555500125C4
:101D8000B5EB901F1CBF02B0BDE8F08F04EB46001E
:101D90001B4951F82020183111F8208006EB46002D
:101DA000800100EB841000F1804000F5A040D0F8E5
:101DB00050491449FF26A1FB02914908A1EB810972
:101DC0004A44D2009640FFB297404FEA8802002072
:101DD00003F00F0393400CF00F0C4FF00F090CFAB7
:101DE00002FC09FA02F24FEA810805FA00F12142E9
:101DF0002DD009E000500040944C0200CDCCCCCC5A
:101E0000B44C0200ABAAAAAA08EBC00101F18041C0
:101E100001F5A041D1F8809C29EA060949EA0709A1
:101E2000C1F8809C810001F1804101F5A041D1F809
:101E3000A89C29EA020949EA0309C1F8A89CD1F83B
:101E4000BC9C29EA020949EA0C09C1F8BC9C401C67
:101E50000528CAD302B0BDE8F08F2DE9F04F84B059
:101E6000DDE90EA8DDF834C0B8F1000F14BF01247D
:101E700000240294BAF1020F16BF5FEA0A044FF081
:101E8000010B4FF0000B8409FA4D00F00F0707EB30
:101E9000470655F824504FF4B27E05EB8619C0F37F
:101EA00001150EEB851ECDE9009E59F80E9061F3E9
:101EB0005C696BF318697CD002996AF3420961F39B
:101EC0000009DDE9001BDFF8ACA341F80B904FF4EB
:101ED000B4715AF82440C0F3011901EB891104EBE5
:101EE0008614B8F1000F665814BF46F0800626F03D
:101EF000800666500126B6EB901F1CBF04B0BDE8FB
:101F0000F08F05EB4700DC49DC4C51F8201054F809
:101F1000204007EB4700800100EB851000F1804076
:101F200000F5A040D0F85009D54DFF26A5FB01755E
:101F30006D08A5EB850739444FEAC109009006FA00
:101F400009FE00200F21A400A1404FEA850B0125C6
:101F500005FA00F6009D2E4241D01568022D26BFDD
:101F6000AD1E6D080025121D1E68022E26BFB61E6E
:101F7000760800265CF8048BC24FA7FB08874FEA5F
:101F800007580BEBC00707F1804707F5A047D7F8C4
:101F900080AC4FEA18682AEA0E0A08FA09F84AEAF9
:101FA0000808C7F8808C870007F1804707F5A0472D
:101FB00000E01AE0D7F8A88C06F00F0628EA01081E
:101FC000A64048EA0606C7F8A86CD7F8BC6C05F02E
:101FD0000F058E43A5403543C7F8BC5C1B1D401C54
:101FE0000528B4D304B0BDE8F08F1168022926BFDC
:101FF000891E49080021D3F800B0BBF1020F26BFAB
:10200000ABF1020B4FEA5B0B4FF0000BCDF80CB0BD
:10201000DFF870B2DCF800E0ABFB0EEB4FEA1B1B05
:102020006BF31749DDF80CB06BF3CA1961F3C609FD
:1020300042E72DE9F00F8F4D84094FF4B27955F83E
:10204000244000F00F0505EB450604EB8614C0F3B1
:10205000011609EB8619DDE9098754F80940DDF816
:1020600020C0C4F3436BC4F3410904F0010A002902
:1020700018BFC1F800B0B8F1000F18BFC8F8009041
:10208000002F18BFC7F800A081094FF001085BD0EE
:10209000B8EB901F1CBFBDE8F00F704706EB450082
:1020A0007549764C51F8201054F820B005EB4500E6
:1020B000800100EB861000F1804000F5A040D0F8D0
:1020C00050A96F4C0020A4FB015464084FEA840916
:1020D000A4EB84042144CF004FEA8B0508FA00F1F9
:1020E00011EA0A0F2AD009EBC00101F1804101F584
:1020F000A041D1F8801CF940840004F1804404F52B
:10210000A044C9B2D4F8A86CD4F8BC4CEE4006F098
:102110000F06EC4004F00F041AB16400A41C42F84E
:10212000044B1BB17400A41C43F8044BBCF1000F1A
:1021300004D001EB810189004CF8041B401C0528E8
:10214000CCD3BDE8F00F7047C4F30740C4F3C3110C
:10215000C4F3C30412B16400A41C146013B1490099
:10216000891C1960BCF1000F04BFBDE8F00F704777
:1021700000EB80008000CCF80000BDE8F00F704755
:102180003C4A8009002952F82000C16914BF41F07F
:10219000200121F02001C16170473649800951F8C2
:1021A0002000C069C0F34010704730B490B00022E6
:1021B0004FF48045EC466C1001E0082A05D2531C10
:1021C00003EB8303B5FBF3F304E0D31F03EB8303BB
:1021D000B4FBF3F35B1A48BF5B424CF82230521C4D
:1021E000102AEAD30023009C01215CF82120A2429E
:1021F000BCBF14460B46491C1029F6D300F00F0251
:1022000002EB42014FEA8111C0F3011C01EB8C117A
:1022100001F18041840901F5A04135D00124B4EBDE
:10222000901F1EBF10B030BC70470CEB4200D1F8BD
:1022300050C9124A12F820200F25910000208D402D
:1022400003F00F028A4004FA00F111EA0C0F0AD0E1
:10225000810001F1804101F5A041D1F8D03CAB43B0
:102260001343C1F8D03C401C0528ECD310B030BC5F
:1022700070470000944C0200B44C0200CC4C0200A9
:10228000ABAAAAAACDCCCCCCD1F8680163F30300E9
:10229000C1F86801EAE781091CBF0020704700F01F
:1022A0000F0101EB41018901C0F3011001EB801026
:1022B00000F1804000F5A040D0F8680100F00F0068
:1022C000082834BF401CC01F00EB800034BF4FF40F
:1022D00080414FF40051B1FBF0F070472DE9F00759
:1022E0004FF0010991B0B9EB901F1EBF11B0BDE8CE
:1022F000F007704700F00F02C0F3011000EB42033B
:1023000002EB4202920102EB8010DFF83CC500F1C3
:10231000804000F5A0405CF82330D0F850A90F2091
:102320004FEA83084FF0000C4FF480466C4600FAE9
:1023300008F709FA0CF010EA0A0F36D051F8043BFE
:1023400000204FF4005501E0082805D2421C02EBA2
:102350008202B6FBF2F204E0C21F02EB8202B5FB7E
:10236000F2F2D21A48BF524244F82020401C1028F2
:10237000EAD30025009B012054F820209A42BCBFDC
:1023800013460546401C1028F6D34FEA8C0000F196
:10239000804000F5A040D0F8D02C05F00F03BA43E0
:1023A00003FA08F31A43C0F8D02C0CF1010CBCF16D
:1023B000050FBED311B0BDE8F007704770B401241B
:1023C000B4EB901F1CBF70BC704700F00F02C0F34D
:1023D000011000EB420302EB42029201DFF868C4F5
:1023E00002EB801000F1804000F5A0405CF8233043
:1023F000D0F850C900209B004FF480456E1004FABD
:1024000000F212EA0C0F16D0820002F1804202F5AF
:10241000A042D2F8D02CDA4002F00F02082A34BFD2
:10242000521CD21F02EB820234BFB5FBF2F2B6FBA4
:10243000F2F241F8042B401C0528E0D370BC704731
:1024400000F00F02C0F3011303EB4202FE4B8009C0
:10245000A3F1380C53F822205CF820000123002956
:10246000D0F8101403FA02F214BF11439143C0F8DC
:102470001014704700F00F01C0F3011303EB41018A
:10248000F14B0022800913F82110383B53F820004B
:10249000D0F81004012303FA01F1084218BF012209
:1024A0001046704770B410F0300F14BF01230023A2
:1024B0008609DFF898C300F00F024FEA90104FF43E
:1024C0009A7502EB42025CF820004FF0010405EB24
:1024D000821214D085584FEA430C5B420CEB430345
:1024E0009B1C04FA03F35B1E03FA0CF4194025EA63
:1024F000040401FA0CF12143815070BC704700299B
:10250000815804FA03F31ABF194381509943F3D059
:1025100070BC704730B410F0300118BF012184093D
:102520004FEA9013C94D00F00F0000EB40004FF44C
:102530009A7202EB801255F823004FF0010C0CD078
:1025400082584800C240494200EB4100801C0CFA0E
:1025500000F0401E30BC1040704780580CFA01F16A
:10256000084018BF012030BC7047B84B800953F8B1
:1025700020C0CCF8741053F820C01168CCF8781043
:1025800053F820005168C1677047B1490028D1F85D
:10259000AC0014BF40F0020020F00200C1F8AC0013
:1025A0007047AB490028D1F8AC0014BF40F00100DF
:1025B00020F00100C1F8AC007047A548D0F8E00059
:1025C000A449096808437047A149C1F8E400A24939
:1025D000086070479E48D0F89800A049096840EA12
:1025E0004100704770B44FEA0075860900F00F048F
:1025F0004FEAD565C0F30110A5F1020502F0010C08
:1026000005444FEA8C334FEA520012D001EB4101EE
:102610007CB305EB4502D20002EB8C3202EB810168
:1026200001EB800000F1405000F5C030406A70BC02
:10263000704701EB410202EB01117CB198226A4321
:1026400002EB8C3202EB810101EB800000F1405083
:1026500000F58030D0F88C0E70BC704703EB810120
:1026600001EB800000F1405000F58030006870BC44
:102670007047FFE703EB810101EB800000F1405060
:1026800000F5C030006870BC7047F0B44FEA0076C7
:10269000870900F00F044FEAD666C0F30110A6F1D7
:1026A000020602F0010C06444FEA8C354FEA520054
:1026B00012D001EB41017CB306EB4602D20002EBE3
:1026C0008C3202EB810101EB800000F1405000F5FB
:1026D000C0304362F0BC704701EB410202EB0111D4
:1026E0007CB19822724302EB8C3202EB810101EB48
:1026F000800000F1405000F58030C0F88C3EF0BC06
:10270000704705EB810101EB800000F1405000F5BE
:1027100080300360F0BC7047FFE705EB810101EBFF
:10272000800000F1405000F5C0300360F0BC7047FD
:10273000830900F00F02C0F301100CD0002A08BF7B
:10274000474805D0012A17D000280CBF4548464805
:1027500000EB81307047002A08BF4FF04050F7D09F
:10276000012A04D000280CBF40484148F0E7002867
:1027700014BF40484048EBE7002814BF3F4840489A
:10278000E6E710B44FEA007C840900F00F034FEA3B
:10279000DC6CC0F30110ACF1020C604410D0002BD3
:1027A00008BF38481CD000EB4000C00000EB81306F
:1027B00002EB420100EB8100334910BC0844704732
:1027C000002B08BF31480BD09823584300EB8130D1
:1027D00002EB420101EB021100EB81002C49ECE716
:1027E00010BC00EB813070472DE9F0074FEA901CD8
:1027F00000F00F04154804EB440150F82C0000F5DC
:10280000C07300EB8110D0F800014FF47A7280B2EF
:10281000B2FBF0F100FB1120002818BF01200D18B9
:102820001C4F002040F2FF1644EA001141EA8C11CF
:1028300001F00F02C1F3011101EB420157F8211021
:102840004A08C907C90E27E0CC4C0200944C02008C
:1028500000500040E0580040E458004098580040C4
:1028600000800030E4810030248300304C180030B8
:102870004C1D0030CC0E0030CC090030648100309B
:1028800024800030008001302480013000000130BD
:102890008C0E01309C4C020053F8228003EB820224
:1028A00028FA01F8D2F80CA0A8EB050906FA01F8FD
:1028B000C9F308092AEA080A09FA01F14AEA0109F2
:1028C000C2F80C90D2F8189029EA080848EA0101E9
:1028D0009161401C0228A7D3BDE8F00770470000B3
:1028E000FEF716B810B5FEF713F8012818BF10BD93
:1028F0000020FDF7C8FF21210020FEF70FF821215D
:10290000BDE810400120FEF709B810B5FDF7B4FF8F
:10291000FDF7FEFF01280AD10020FDF7B4FF2121B9
:102920000020FDF7FBFF21210120FDF7F7FF01212A
:10293000052001F044FE0121052001F040FEF74989
:102940000020887110BD10B54FF4066001F08DFEB7
:10295000BDE810404FF4066001F078BEEF4A014632
:102960001079002818BF0120002918BF012111711A
:10297000002151717047E94A916A90620846704798
:10298000E6490020C870887048707047E34900200D
:10299000C87088704870704710B50446014684229C
:1029A000DF481CF01BFE04F18401BDE810408422C6
:1029B000DC481CF013BE70B50007C00E0D46801E2B
:1029C00000EB400101EB0014D7484FF4987200EB84
:1029D000C40029461CF002FED44805F5987100EBAE
:1029E000C400BDE870404FF498721CF0F7BDDFF8EA
:1029F00040C348B14A424FF4806300EB810103EBCE
:102A0000820260461CF0EABD4FF4806160461CF013
:102A1000EABD2DE9F04105460020FDF7BDFFC54F99
:102A2000DFF814830446EDB14C2004FB00F2164697
:102A3000294638461CF0D2FD324605F5E461404691
:102A40001CF0CCFD04EB440000EB041407EB840005
:102A50004C211CF0C8FD08EB8400BDE8F0414C217E
:102A60001CF0C1BD4C21401C41430C4638461CF0B3
:102A7000BAFD21464046BDE8F0411CF0B4BD10B59A
:102A8000A64C2062FEF738FAFEF70DFAA169A2699A
:102A9000C1F307216FF30F02A261A369C2B243EA37
:102AA0000222A261022803D1A26942F00102A261BE
:102AB00081421ABFE269002A10BD012918BF002116
:102AC000012818BF0020814208BF10BDBDE810409A
:102AD00010474FF04020816941F002018161016996
:102AE00041F00301016100F0F8BF2DE9F0414FF022
:102AF0004022054690690C4640F002019161106940
:102B000040F00300106100F0E8FF0027002C7CD0AB
:102B10000020FDF7B8FE00202168FEF7A9F840204C
:102B20006168FEF7A5F82846FFF7A9FF0020FDF72A
:102B300064FF0126002832D0A068FFF76AFF7C48B6
:102B4000636953B1E1694FF4806C4A420CEB820235
:102B500003EB81011CF042FD1AE0784D4FF48061D7
:102B60001CF041FD0020295600290EDB0A09120243
:102B700002EB800202F1405202F500320907C90E51
:102B8000136806FA01F119431160401C2628EAD3A4
:102B90006B48A16969B14FF400721CF01FFDE06839
:102BA000A0B30120FDF729FFDFF87C815F4E28B13B
:102BB00008E04FF400711CF016FDF0E71120FDF75E
:102BC0001CFF68B1E56840464FF4987229461CF036
:102BD00005FD30464FF4987205F598711CF0FEFC27
:102BE0000220FDF70AFF18B91220FDF706FF68B1B1
:102BF000E56854484FF4987229461CF0EFFC52489F
:102C00004FF4987205F5987101E017E001E01CF0AF
:102C1000E5FC4120FDF7F1FE18B95120FDF7EDFE6E
:102C200060B1246954B1842221463D481CF0D6FC91
:102C3000842204F184013B481CF0D0FC3748C77063
:102C400087704770876201790021017147714FF4E5
:102C5000066001F00AFDBDE8F0414FF4066001F0A6
:102C6000F5BC10B50020FDF70EFE00F026FF2B4846
:102C7000406B002808BF10BD4FF04020016921F0D3
:102C800003010161816921F00201816110BD4FF4EE
:102C9000066001F0E0BC10B54FF4066001F0DBFC0B
:102CA000FDF736FE01280AD10020FDF7ECFD2121B9
:102CB0000020FDF733FE21210120FDF72FFE2348E0
:102CC000D0F8401321F48031C0F840130020FDF704
:102CD000DAFD00F0F2FE1148406B002808BF10BD7D
:102CE0004FF04020016921F003010161816921F069
:102CF0000201816110BD10B501F0B2FC10F060005E
:102D000018BF012010BD054AD169D061084670473F
:102D10000248006A704701488069704728840010A3
:102D20000080013000C001308C0E01308C4E01302B
:102D3000000002300000013000400130488A0010DD
:102D400000400230BC0F0130BC4F01300050004049
:102D500072B6FE498A6922EA0000886162B670474D
:102D6000FA480078002818BF0120704770B5FDF7B9
:102D7000CFFD002818BF70BD0024F44DEC70AC707E
:102D80006C7021212046FDF7C9FD21210120FDF7AE
:102D9000C5FD2C70BDE870400120FDF774BD70B515
:102DA0000446FDF7B5FD002818BF70BD0021E74DB2
:102DB000E970A970697021210020FDF7AFFD212184
:102DC0000120FDF7ABFD022C3CBF0120FDF7B6FD55
:102DD000012028706C62BDE87040FDF754BD10B54D
:102DE000FDF796FD002818BF10BD0020D74CE070FD
:102DF000A07060702121FDF791FD21210120FDF7D8
:102E00008DFD0120FDF79AFD012020706062BDE874
:102E10001040FDF738BD0020FDF735BD10B5CB4C97
:102E20000020A07060702121FDF778FD2121012094
:102E3000FDF774FD207800281CBF0120FDF77EFD02
:102E40000120BDE81040FDF71EBDC049C8627047B3
:102E5000BE48C06A7047BD4908637047BB48006BF5
:102E60007047BA4A00F00F00116B21F00F010843C0
:102E700010637047B54890F8300000F00F007047BD
:102E800070B5B24C0546E06A421CE262216B11F05B
:102E9000800F14BFC1F3021101F00F0139B1B2FB71
:102EA000F1F001FB1020002808BFFEF7B2FE2078E9
:102EB00050B1606A10B1606A401E6062606A0028AA
:102EC00004BF0020FDF7DFFC20212846FDF726FD8A
:102ED000A16A00291CBF28468847FDF7E4FF0228A5
:102EE00015D19B48D0F8481311F0010F0FD0D0F83E
:102EF000481341F00101C0F84813D0F8481321F0FD
:102F00000101C0F84813A06940F00200A061914897
:102F1000016841F02001016070BD0020B0E7012090
:102F2000AEE710B5FFF749FB0446FFF74DFB8A48B3
:102F3000044208BF10BD8548816941F004018161E8
:102F40000E2101EAD43104F001020A43816962F3DF
:102F50001F4181617F48016841F02001016010BD7F
:102F6000002818BF01207949486370477B487047A3
:102F70007B4870477548806B70477448C179427AC6
:102F8000914214BFC06B006C70477048006C704772
:102F90002DE9F04F0025DFF8C4918DB009F14C0404
:102FA000AC466F1E09F8057004F805C06D1C262D8F
:102FB000F8DB0025002805DD565D09F805606D1C6D
:102FC000A842F9DC00220126CDF804C06D46CDF8F8
:102FD00000C0002821DD19F902B0BBF1000F19DB98
:102FE000BBF1140FA8BFABF1140B04DABBF10A0F4D
:102FF000A8BF0BF1120BBBF1260F0BD24FEA5B18E7
:103000000BF01F0B55F828A006FA0BFB4AEA0B0A37
:1030100045F828A0521C8242DDDB002292460DF1C9
:1030200008084FEA521B02F01F0E55F82BB006FAA3
:103030000EFE1BEA0E0F1ABF08F802A00AF1010AE1
:1030400008F80270521C262AEBDB4FF0000A002819
:1030500016DD19F90A20002A0EDB142AA8BF143A3B
:1030600002DA0A2AA8BF1232262A3ABF18F802202A
:1030700004F80A2004F80A700AF1010A8245E8DB24
:10308000DFF8C89000220028C9F838C009DD14F91B
:1030900002A0924502D0C9F8384002E0521C824298
:1030A000F5DB304A0020A2F17204A2F1260A27546F
:1030B0000AF800C002F800C0401C2628F7DB0020F8
:1030C000002906DD13F800B004F800B0401C81426E
:1030D000F8DC0020CDF804C0CDF800C0002913DDD5
:1030E0002356002B0DDB262B0BD24FEA531B03F08C
:1030F0001F0355F82BE006FA03F34EEA030345F8E5
:103100002B30401C8842EBDB002003464FEA501B6B
:1031100000F01F0E55F82BB006FA0EFE1BEA0E0F3C
:103120001ABF08F800305B1C08F80070401C262805
:10313000ECDB0020002919DD2356002B04DB262BB5
:103140003CBF18F803301354401C0DE028840010D5
:10315000005000407C84001001000700488A0010E5
:103160006E8A0010E08A00108842E5DB0020C9F872
:1031700040C0002908DD1356834202D0C9F8402020
:1031800002E0401C8842F6DB11F0010F18BF252039
:1031900015D0420900F01F0355F8222006FA03F368
:1031A0001A420AD1420900F01F0055F8223006FAEF
:1031B00000F0184345F8220001E0401EE9D5002048
:1031C0000246430900F01F0B55F8233006FA0BFBAB
:1031D00013EA0B0F1ABF08F80020521C08F8007001
:1031E000401C2628EDDB002000290BDD2256002A9A
:1031F00005DB262A3CBF18F802200AF80020401CF4
:103200008842F3DB0020C9F83CC00029DCBF0DB0C8
:10321000BDE8F08F1AF90020824204D0C9F83CA022
:103220000DB0BDE8F08F401C8842F3DB0DB0BDE867
:10323000F08FFE487047FE48406C70472DE9F00162
:10324000FA4C002282B0551E04F1050CA5540CF86E
:103250000250521C052AF9DB00228B5CA354521C3D
:10326000052AFADB00230127194600280AD96256ED
:10327000002A04DB052A3CBF07FA02F21343491C6B
:103280008142F4D300210A466E4607FA01F818EA93
:10329000030F1ABF7254521C7554491C0529F4DBE4
:1032A000002100280AD96256002A04DB052A3CBF07
:1032B000B25C0CF80120491C8142F4D3DC4B0021A4
:1032C000002859649EBF02B0BDE8F00170471CF9A8
:1032D00001208A4205D0C3F844C002B0BDE8F00125
:1032E0007047491C8142F2D302B0BDE8F00170473B
:1032F00040F2DB114843CF4901EB80007047CE49D3
:10330000C0EB001001EBC0007047DFF824C3012BB5
:103310008CF807008CF8081003D9401C20F001003D
:1033200011468CF809008CF80A1000FB01F24FF6E8
:10333000FF7101EA4202ACF8122001EA4000ACF849
:1033400014007047BA48807A7047B948407A70478D
:10335000B74AD07211737047B548007B7047B448C4
:10336000C07A7047B54A107051707047B349085C15
:1033700070472DE9F047DFF8B892044699F8040049
:10338000002804BF99F801001CF032F90AF087FA0E
:1033900028B9002301227F2107200EF0C9F899F8EF
:1033A0000300002808BFBDE8F0874FF00008D9F8F7
:1033B000200047464646454610F0070F1CBFDFF881
:1033C000748210F0020F05D0B9F81210994A21F05A
:1033D00001018F1810F0F00F18BF974E10F4774FBF
:1033E00018BF974DD9F82C002060FDF75FFD10F055
:1033F000010F06D0FEF7FDF8022828BF99F8020059
:1034000000D20020E760C4E90108C4E90465012096
:10341000BDE8F08786480021C1704171704770B5E2
:1034200005460020FDF7B8FA4C2100FB01F21446D6
:10343000844928461CF0D2F8224605F5E460BDE830
:10344000704081491CF0CAB8F0B583B00020FDF788
:10345000A3FA044669460020FEF72EFA0022002C4B
:103460002AD96E464FF0010C4FF6F07502EB420080
:10347000002100EB02104B0901F01F0756F8233022
:103480000CFA07F73B4211D0CB075B0C03EB800330
:103490004F0803EB870303F1405303F580331B8888
:1034A0009BB2AB4202D903B00020F0BD491C2629D3
:1034B000E1D3521CA242D9D303B00120F0BD70B5B4
:1034C0000007C00E0D46801E00EB400101EB00140A
:1034D0005E484FF4987200EBC40128461CF07EF859
:1034E0005B484FF4987200EBC40105F59870BDE895
:1034F00070401CF073B82DE9F04F07460007C00E6E
:1035000083B0801E002527F03F0BE9464FF00108ED
:103510004FF6F0760290384665F31F1040EA0B0034
:1035200000F0FF0A5046FDF768FA00283DD05046EB
:10353000FEF765FA08FA00F4022C88BF02246946F7
:103540005046FEF7B9F90022002C2ED90298982196
:10355000284400FB01FA02EB4200002100EB021CB0
:10356000480901F01F0359F8200008FA03F3184234
:1035700015D001F001000AEB803000EB8C004B0805
:1035800000EB830000F1405000F58030B0F88C0E65
:1035900080B2B04203D903B00020BDE8F08F491CCF
:1035A0002629DDD3521CA242D5D36D1C022DB2D3E5
:1035B00003B00120BDE8F08F10B5044684222549F0
:1035C0001CF00CF804F18400BDE81040842222496C
:1035D0001CF004B82DE9F04F83B000200290402089
:1035E000FDF70BFAE9464FF001084FF6F077E0B12E
:1035F0004020FDF7D1F9044669464020FEF75CF90A
:103600000022002C3AD9002102EB420C480959F85B
:10361000203001F01F0008FA00F0034228D0C8074C
:10362000400C00EB8C004B0818E027E07084001081
:1036300028840010A01801100C20011035840010FF
:10364000FC20011000000130004001308C0E0130E0
:103650008C4E01300080013000C0013000EB83004F
:1036600000F1405000F5C030008880B2B84256D812
:10367000491C0529CAD3521CA242C4D3012670009A
:10368000A0F1020B002546EA0510C0B240F0400A46
:103690005046FDF7B2F9C8B35046FEF7B0F908FA44
:1036A00000F4022C88BF022469465046FEF704F954
:1036B0000021002C2AD90BEB050000EB40004FEA5B
:1036C000C00A01EB4102002002EB011C420900F09C
:1036D0001F0359F8222008FA03F31A4210D000F011
:1036E00001020AEB823202EB8C02430802EB8302F6
:1036F00002F1405202F5C032928C92B2BA420ED818
:10370000401C0528E2D3491CA142DAD36D1C022DCE
:10371000B9D3701CC6B2022EB1D901200290029812
:1037200003B0BDE8F08F2DE9F04100268E4D002852
:103730000C4645D000F00F01C0F3011001290EBF67
:1037400000210229BDE8F081022828BFBDE8F081F0
:103750000F18FDF7DDF85FEA00081CBF0020FDF739
:1037600092F800239820474303EB4300002200EB2C
:10377000031C02F0010007EB8030510800EB8C00C5
:1037800000EB810000F1405000F58030521CC0F881
:103790008C4E262AEDD35B1C022BE5D3B8F1000F2B
:1037A00008BFBDE8F081AE706E7021210020FDF7EA
:1037B000B5F821210120FDF7B1F82878A0B330E059
:1037C000FDF7A6F807001CBF0020FDF75CF80023FA
:1037D00003EB4300002200EB0310D107490C4FEA32
:1037E000520C01EB800101EB8C0C0CF1405C0CF5F0
:1037F000803C521CCCF80040262AEED35B1C312BB7
:10380000E6D3002F08BFBDE8F081AE706E702121B5
:103810000020FDF783F821210120FDF77FF82878AB
:1038200010B10120FDF78AF8BDE8F0410120FDF755
:103830002AB810B5FDF7E0FF4B49088210BD4A4B8E
:1038400010B4E02101EA102C1B8AC1B2C0F304229B
:10385000994288BF194664246143B1FBF3F102EB3E
:10386000C20303EB021201EB82014FF47A723F4B69
:103870000CFB02F2A3FB02329208521C520810F415
:10388000803F08BF494210F4003F14BF8818881ACF
:1038900000B210BC704710B5354C4FF4806135480C
:1038A0001BF0A1FE002001232156002910DB0A098C
:1038B000120202EB800202F1405202F500320907C7
:1038C000C90ED2F800C003FA01F14CEA01011160FF
:1038D000401C2628E8D310BD10B5254C4FF480615C
:1038E00024481BF080FE002001232156002910DB14
:1038F0000A09120202EB800202F1405202F5003284
:103900000907C90ED2F800C003FA01F14CEA01011F
:103910001160401C2628E8D341F2EC0116481BF048
:1039200062FEBDE8104041F2EC0114481BF05BBEA2
:103930000D4810B5006A12490840FFF7A0F84FF48F
:1039400080610C481BF04FFE40F68C610A481BF06A
:103950004AFE40F68C6109481BF045FEBDE8104068
:103960000020FDF759BD000028840010ABAAAAAAC8
:10397000488A001000000230000001300040013091
:103980000100FF0082B04FF4FA62009013E000BF24
:1039900000BF00BF00BF00BF00BF00BF00BF00BF2F
:1039A00000BF00BF00BF00BF00BF00BF00BF019845
:1039B000411E0191EBD20098411E009128BF019257
:1039C000F5D202B070472DE9F0410027634D012682
:1039D000002808BF2E701FD001282F7018BF6F70ED
:1039E0001AD04FF04028D8F8100040F00400C8F872
:1039F000100029785A4C002914BF49F6083059485C
:103A0000E06014BF58484FF0BB70A0605748006892
:103A100030F0FF0206D101E06E70E2E7E26860F389
:103A20000302E26089B1A06840F01800A0600120A4
:103A3000FFF7A8FFA06840F48050A0600120FFF7C6
:103A4000A1FFA06840F40070A0600120FFF79AFF7A
:103A5000687870B1E06840F02000E060A06820F471
:103A60000070A0600120FFF78DFFE06840F01000BB
:103A7000E060D4F8B00040F00100C4F8B0000120CC
:103A8000FFF780FFE6674FF4E0602061C4F88870BC
:103A90002878002818BFC4F89460E06820F030004F
:103AA000E060A06820F49050A060D8F8100020F0EA
:103AB0000400C8F81000BDE8F0812948C16821F071
:103AC0003001C160816821F4905181604FF0402045
:103AD000016921F00401016170474FF04020016944
:103AE00041F0040101611D491D480A783AB182681C
:103AF00042F018028260826842F4905282604978F3
:103B000019B1C16841F03001C160D0F8B01041F086
:103B10000101C0F8B0107047B0F5007F28BF40F237
:103B2000FF10C0F30800124941EA00200C49086464
:103B300070470B494FF0204008647047084A116CE9
:103B40004FF020401064506C11F0FF0FC0F30820BC
:103B50001CBF41F020411164704700007A840010BE
:103B60000060004005F4010020009B00D0FE04002E
:103B7000130000A04FF040200021016302224263A5
:103B8000826B02F03C0242F001028263026922F081
:103B900003020261026A22F001020262424A1368D1
:103BA00043F0010313603C2282612822C2613F4836
:103BB00001603F4801603F4850F88C2F42F480522A
:103BC00002603D4A481E10603C480160704710B5D5
:103BD00001F0F9FA39480468002C08BF30BFFAD068
:103BE0000021016001F0F3FA204610BD10B501F08C
:103BF000EAFA324B00204FF0402101221C6824B128
:103C0000186001F0E4FA204610BD72B6D1F838C051
:103C10000CF03C0CC1F838C00A6320BF0863D1F82F
:103C200038C00CF03C0C4CF0010CC1F838C062B646
:103C3000BFF36F8FBFF34F8FE0E710B504460F203F
:103C400000F0F8FC0F2000F0DDFC1D490A6842EA94
:103C50000400086010BD1A490A6822EA00000860E2
:103C60007047164A516850600846704770B514484E
:103C7000006814490968114D00EA010469680029C7
:103C80001CBF2046884714F0100F05D0094850F893
:103C90008C1F41F48051016007480460286840F49B
:103CA0000040286070BD00000048004024480040EB
:103CB0001048004000300040144800407C84001050
:103CC0001C48004018480040704770470022B2EB83
:103CD000D10F26D20368B3F1FF3F04BF4368B3F1AD
:103CE000FF3F17D18368B3F1FF3F04BFC368B3F14F
:103CF000FF3F0FD10369B3F1FF3F04BF4369B3F145
:103D0000FF3F07D18369B3F1FF3F04BFC369B3F13C
:103D1000FF3F01D0002070472030521CB2EBD10F82
:103D2000D8D30120704710B40023B3EBD20F30D2A8
:103D3000D0F800C00C68A44522D1D0F804C04C686B
:103D4000A4451DD1D0F808C08C68A44518D1D0F87E
:103D50000CC0CC68A44513D1D0F810C00C69A445A0
:103D60000ED1D0F814C04C69A44509D1D0F818C0C0
:103D70008C69A44504D1D0F81CC0CC69A44502D0FC
:103D800010BC00207047203020315B1CB3EBD20FF9
:103D9000CED310BC012070472DE9F041054601F05B
:103DA0001AFA002021264FF4825784464FF4E0226D
:103DB0001660C5F800C0116841F004011160116877
:103DC00011F0040FFBD1176080232C460021D4F89A
:103DD0000080B8F1FF3F04BFD4F80480B8F1FF3F82
:103DE0001DD1D4F80880B8F1FF3F04BFD4F80C808F
:103DF000B8F1FF3F13D1D4F81080B8F1FF3F04BFF2
:103E0000D4F81480B8F1FF3F09D1D4F81880B8F184
:103E1000FF3F04BFD4F81C80B8F1FF3F08D0C2F8C0
:103E200000C0401CC0B20828C2D30220BDE8F08107
:103E3000491C2034B1EBD30FC9D3C2F800C0012014
:103E4000BDE8F0812DE9F041054601F0C4F90020FC
:103E5000092684464FF4E0231E60C5F800C01968A7
:103E600041F004011960196811F0040FFBD12C46D0
:103E70004FF4806200212768B7F1FF3F04BF6768F5
:103E8000B7F1FF3F17D1A768B7F1FF3F04BFE7685D
:103E9000B7F1FF3F0FD12769B7F1FF3F04BF676953
:103EA000B7F1FF3F07D1A769B7F1FF3F04BFE7694B
:103EB000B7F1FF3F08D0C3F800C0401CC0B20328D0
:103EC000CAD30220BDE8F081491C2034B1EBD20FE7
:103ED000D1D3C3F800C00120BDE8F0812DE9F05F27
:103EE0008846814604274FF07F0A4FF0020B4FF4BB
:103EF000E02601F070F94946424653464FF0060C61
:103F0000C6F800B052F8040B41F8040BC6F800C024
:103F1000306810F0040FFBD15B1EF1D2002030603E
:103F20004C4645461F20D4E900C3D4E90221D5F808
:103F300000E0E64504BFD5F804C09C4505D1AB6858
:103F4000934204BFEA688A4208D07F1E03D34846E2
:103F5000FFF722FFCDE70220BDE8F09F10341035B7
:103F6000401EE0D20120BDE8F09F70B50D4604462A
:103F700001F031F94FF40072214628461BF02EFB68
:103F8000012070BD2DE9F0410546C005ADF5007D6D
:103F900014460E46C00D25D0A8466FF308086F469C
:103FA00001F019F94FF40072414638461BF016FB38
:103FB000C5F30800C0F50077A74288BF27466844CC
:103FC0003A4631461BF019FB4046FFF7E5FE022852
:103FD00044D069464046FFF781FF022843D03D4464
:103FE0003E44E41BB4F5007F19D34FF40072314610
:103FF00068461BF002FB2846FFF7CEFE02282DD0B4
:1040000069462846FFF76AFF02282CD0A4F5007401
:1040100005F5007506F50076B4F5007FE5D2C4B16C
:104020006F4601F0D8F84FF40072294638461BF06D
:10403000D5FA2246314668461BF0DFFA2846FFF7DC
:10404000ABFE02280AD069462846FFF747FF022840
:1040500009D00DF5007D0120BDE8F0810DF5007D52
:104060000A20BDE8F0810DF5007D0B20BDE8F08150
:1040700030B4354D2A68002101244FF0030C04FAB6
:1040800001F3034204D04B000CFA03F39A431A43A2
:10409000491C0C29F3DB2A6030BC7047F0B42A4D70
:1040A0002A68002101244FF0030C022604FA01F3D0
:1040B000034206D04B000CFA03F7BA4306FA03F3A7
:1040C0001A43491C0C29F1DB2A60F0BC70472DE92A
:1040D000F001002201251D4C0F2605FA02F30342D0
:1040E00017D0D31702EB537C4FEAEC0304EB8303A6
:1040F0001F682CF0070CA2EB0C0C4FEA8C0C06FA94
:104100000CF827EA080701FA0CFC47EA0C0CC3F884
:1041100000C0521C0C2AE0DB0B498A6A22EA00002C
:104120008862BDE8F001704707498A6A10438862D7
:1041300070470548416821F080014160416821F4E1
:1041400000714160704700000010004020100040E6
:10415000704772B64FF04020816941F040018161A3
:10416000C16941F04001C16162B6016A41F00101DB
:10417000016270474FF04020016A21F001010162A5
:1041800072B6C16921F04001C161816921F040012D
:10419000816162B6704710B572B64FF04024A069D5
:1041A00040F04000A061E06940F04000E06162B68C
:1041B000206A40F001002062D94843F63F71C16097
:1041C000002181638164C0F8D01003210A2000F02F
:1041D000F6F90A2000F016FA206A20F001002062A9
:1041E00072B6E06920F04000E061A06920F0400074
:1041F000A06162B610BDCA4A106051604843906029
:104200007047C74A10605160484310F0010F18BF53
:10421000401C90607047C249C1F8D0007047C04947
:10422000002818BF012088647047BD498863C868AA
:1042300040F00200C8607047DFF8E4C2CCF820000C
:10424000CCF82410CCF82820CCF82C300120CCF865
:104250003000DCF8340010F0010F05D020BFDCF88E
:10426000340010F0010FF9D110F0020018BF4FF028
:10427000FF307047AA48C16821F00201C160704751
:10428000A748C16841F00101C1607047A44B1862A2
:1042900059629A6201201864586C10F0010F04D022
:1042A00020BF586C10F0010FFAD110F0060018BFB3
:1042B0004FF0FF3070479A48C16821F00101C1609A
:1042C00070479748C16841F00401C1607047944A43
:1042D0008189116701685162416891628168D16288
:1042E00001211165516D11F0010F04D020BF516DF6
:1042F00011F0010FFAD1536F0361936F1B14838286
:10430000936FC3F30523C382936F03F03F030383CB
:10431000D36F1B144383D36FC3F305238383D36FFE
:1043200003F03F03C383D2F88030C3F3094303840F
:10433000D2F88020C2F30902428411F0020018BFB3
:104340004FF0FF3070477648C16821F00401C1602A
:1043500070477348C16841F00401C1607047027C36
:10436000017B02F03F0241EA02416D4A916501681A
:104370005162416891628168D16201211165516D7C
:1043800011F0010F04D020BF516D11F0010FFAD1CF
:10439000D36D8382D36D1B0CC382136E0383136EA4
:1043A0001B0C4383536E8383526EC2F30E42C2834F
:1043B00011F0020018BF4FF0FF3070475848C16835
:1043C00021F00401C16070475548C16841F00801FF
:1043D000C1607047DFF848C1CCF89820CCF82000C5
:1043E000CCF82430CCF828100120CCF89000DCF870
:1043F000940010F0010F05D020BFDCF8940010F0FD
:10440000010FF9D110F0060018BF4FF0FF307047D0
:104410004348C16821F00801C160704701684FEA54
:1044200031423F49C1F8BC204068C1F8C000C868AB
:1044300040F02000C860704701684FEA31423849B7
:10444000C1F8BC204268C1F8C020027A407A02F06C
:10445000010262F35F00C1F8C400C86840F02000A8
:10446000C86070472E4B18625A6299620120C3F8E7
:10447000B400D3F8B80010F0010F05D020BFD3F876
:10448000B80010F0010FF9D110F0060018BF4FF07E
:10449000FF307047224A106251620120C2F8B0001A
:1044A000D2F8B80010F0010F05D020BFD2F8B80044
:1044B00010F0010FF9D110F0060018BF4FF0FF30D7
:1044C00070471748C16821F02001C1607047144847
:1044D000C16841F01001C1607047A3F1050C104B99
:1044E000C3F8A8C018625A6299620120C3F8A000FC
:1044F000D3F8A40010F0010F05D020BFD3F8A4001A
:1045000010F0010FF9D110F0060018BF4FF0FF3086
:1045100070470348C16821F01001C1607047000076
:1045200000900040234810B5022140F8501F01219F
:1045300001611021416241F2060141610021816166
:104540000421816390214163416B41F0010141638A
:10455000C16B21F40021C163C16B41F40051C163FF
:10456000C16B21F00101C163C16B41F00101C16365
:104570004FF4817101610161032000F043F80021D3
:10458000032000F01CF8002010BD10B5032000F03F
:1045900045F808484FF4807101660021016610213A
:1045A000816702214165002010BD03490020087089
:1045B000704700000030004084840010704700F015
:1045C0000303DA004FF0FF0C0CFA02F24FF0050C77
:1045D0000CEBC30301FA03F300F00C0101F1E0213D
:1045E000002807DAD1F8140D90431A401043C1F89F
:1045F000140D7047D1F8000490431A401043C1F8DD
:104600000004704700F01F01012202FA01F1400985
:10461000800000F1E020C0F80011704700F01F0199
:10462000012202FA01F14009800000F1E020C0F807
:104630008011704700F01F01012202FA01F14009C8
:10464000800000F1E020C0F8801270474FF0E021B8
:10465000C1F8000170474FF0E021C1F880017047B8
:104660004FF0E020D0F8000170474FF0E021C1F892
:1046700080027047084800687047074A1168106058
:1046800008467047044A126800F1100352F82300EC
:1046900042F823107047000008ED00E002210C20D2
:1046A000FFF78DBF72B64FF04020816941F4805111
:1046B0008161C16941F48051C16162B6704772B6CF
:1046C0004FF04020816921F480518161C16921F45A
:1046D0008051C16162B67047AA4881B0016F11F480
:1046E000007FFBD1816E11F0010F1CBFD0F8841048
:1046F000009104D0D0F88410009A9142FAD0016F52
:1047000011F4007F04BF4CF27101016642F24131A5
:10471000816601B070479B4981B04FF40D528A66A3
:104720000A6FCA66012898BF012005D9401EB0F55E
:10473000803F28BF4FF6FF7082B24FF05C5040EAD6
:10474000022048664FF01140C1F88000086F10F455
:10475000007FFBD1886E10F0010F1CBFD1F88400E0
:10476000009004D0D1F88400009A9042FAD0086FEB
:1047700010F4007F04BF4CF27100086642F2413031
:10478000886601B070477F4881B0016F11F4007FE7
:10479000FBD1816E11F0010F1CBFD0F88410009185
:1047A00004D0D0F88410009A9142FAD04FF40D5101
:1047B000816601B070474FF04020806910F480504E
:1047C00008BF70476F48806E00F0010070476D4869
:1047D000406EC0F30F2070476A48D0F884007047DD
:1047E00010B50C20FFF726FF0C20FFF70BFF6549E3
:1047F0000220486710BD634910B5032088670C206C
:10480000FFF70CFFBDE810400C20FFF713BF5E4A16
:1048100011681060084670475A4810B5016FC166AC
:1048200059480068002818BF80475848016841F47B
:104830008051016010BD54484068704710B572B691
:104840004FF04020816941F480518161C16941F498
:104850008051C16162B603204A4988670C20FFF786
:10486000DDFE0C20FFF7E6FE00F03CF9484B04208B
:10487000C3F888004FF6FF70C3F88C0072B660333F
:10488000FFF749FF4FF40070186062B610BDF8B52D
:1048900072B63C48016F11F4007FFBD1816E11F0BC
:1048A000010F1CBFD0F88410009104D0D0F8841000
:1048B000009A9142FAD04FF40D51816634494FF479
:1048C00000320A6662B6D1F804124FF04025002982
:1048D00046D02D4C4FF6FF73591AA1602A6BD5F8BC
:1048E00034C002F00F020CF00F0C6244121D01FAEA
:1048F00002F2A2F54341DFF89CC0513961452FD245
:10490000D0F88400191AE160B1F5803F28D2224B1B
:104910004FF0000CA1FB03070CFB037301FB0C31F0
:1049200063461AF06FFE401C40082061B0F57A7FA4
:1049300038BF4FF47A70194B9968002908BF986006
:104940005A681A609968C3E901108A4215D98242EF
:1049500005D9814201D9616002E0606000E06260D7
:1049600000F0D0F872B6A86920F48050A861E86918
:1049700020F48050E86162B6F8BD8242EFD88142EF
:10498000EBD8E8E700C00040888400107C84001069
:1049900000A000404F62250000E1F505088B0010E3
:1049A0004FF04020816941F0040181610C480168A9
:1049B00041F404710160001F016821F004010160ED
:1049C000016841F0100101607047064908607047B6
:1049D000BFF34F8F054904480860BFF34F8FFEE7D0
:1049E00014ED00E008ED00E00400FA050CED00E035
:1049F0004FF04020816941F0040181610B4801685A
:104A000041F0010101600B490948C1F8C400704739
:104A10000948006842F27001084070470848074999
:104A20000160084981600021C1607047144C00405A
:104A300001005FA00060004000440040A0C00E00E4
:104A400000100040508A5900022824BF00207047FF
:104A5000DC4B53F8202043F820101046704770B507
:104A6000D94C206FD74D10F0010F05D00120E06622
:104A70002868002818BF8047206F10F0020F08BF79
:104A800070BD0220E0666868002808BF70BDBDE800
:104A90007040004710B572B64FF04020816941F078
:104AA00080018161C16941F08001C16162B6022269
:104AB000C5490A6501230B660323CB664A6572B6B6
:104AC000816921F080018161C16921F08001C161AA
:104AD00062B60920FFF796FD0221BDE810400920CB
:104AE000FFF76DBD72B64FF04020816941F0800143
:104AF0008161C16941F08001C16162B60220B249A1
:104B000008657047B0490220486572B64FF04020F2
:104B1000816921F080018161C16921F08001C16159
:104B200062B670474FF040208069C0F3C0107047F4
:104B3000A548016F11F4007F14BF4FF440714FF48A
:104B400080710166704710B59F4CE06F10F0020F46
:104B50004FF0010018BF0320606700F06DF94FF0BF
:104B600040210A6B496B02F00F02D04001F00F01A7
:104B7000C8400521B0FBF1F04FF405710009C4F8FD
:104B800080109249A1FB00104009C4F88400206FF6
:104B900010F4007F14BF4FF440704FF48070206613
:104BA00010BD8948016F11F4807F14BF4FF440712C
:104BB0004FF4007101667047834B30B4DA6F12F026
:104BC000010F14BF032202225A6700EB4005C5EB18
:104BD000C010C1EBC0004FF4FA744C43C0EB00109E
:104BE00000EB40007A4904EBC000A1FB00104FF03D
:104BF000402100220C6B4FF0020CC008496B04F0FE
:104C00000F0401F00F012144C8400521B0FBF1F071
:104C1000B0F5803F05D3511C4008CAB2B0F5803FC3
:104C2000F9D242EA0C2141F01001C3F88810C3F810
:104C30008C00186F10F4807F14BF4FF440704FF455
:104C40000070186630BC70475F48016F11F4003F78
:104C500014BF4FF440314FF48031016670475A4819
:104C6000016F11F4803F14BF4FF440314FF4003115
:104C7000016670475448006FC0F3002070475248E7
:104C8000006FC0F3402070474FF040218969C1F3A5
:104C9000C011002904BF002070474B4900280CBFF9
:104CA000D1F80002D1F8040270474FF040239A690E
:104CB000C2F3C012002A04BF00207047424A0028F5
:104CC0000CBFD2F88000D2F88800C0F30A200CBFD5
:104CD000D2F88020D2F8882002F00F02D3F830C03A
:104CE0005B6B0CF00F0C03F00F0363441A4491400C
:104CF000012202EB400048433449A1FB00100009A7
:104D00007047344901200870704770B432224FF068
:104D1000402351431A6BD3F834C002F00F020CF059
:104D20000F0C6244121DD14008BF012104D0B1F51F
:104D3000803F28BF4FF6FF719A69C2F3C012002A64
:104D40001CBF70BC704772B69A6942F080029A61CB
:104D5000DA6942F08002DA6162B602241A4A146506
:104D6000250415664FF0040CC2F888C0C2F88C10F8
:104D7000DFF864C0C2F86CC05467184902283CBF11
:104D8000104E46F820100021124801704FF40071B7
:104D90001166017819B920BF01780029FBD015668A
:104DA000C2F878C0C2F86CC0546572B6986920F039
:104DB00080009861D86920F08000D86162B670BC2C
:104DC00070470000A084001000A000401F85EB5138
:104DD000CDCCCCCC9C84001002000202B36C00004D
:104DE0004FF0E02100208861086127494860704742
:104DF00010B54FF0E02460610020A0610221401E48
:104E0000FFF7DDFB07202061BDE8104008F064BC1F
:104E100010B508F065FC4FF0E0210020086110BDDE
:104E200010B508F05DFC4FF0E02100200861164845
:104E30000188491C018010BD1348806870472DE926
:104E4000F041114C002705462780A0684FF47A7185
:104E5000B0FBF1F04FF0E026401E7061B761022117
:104E6000C81EFFF7ACFB0720306108F035FC218835
:104E7000A942FCD308F034FC3761BDE8F081034956
:104E80004843014988607047A884001040420F00E1
:104E90004FF04020816921F400518161C16921F402
:104EA0000051C1617047A8490A78824218BF06289C
:104EB00028BF7047A54AA64B52F830C0C3F808C0B7
:104EC00002EBC0025268DA60087070474FF0402071
:104ED000816941F400518161C16941F40051C161AE
:104EE000704710B501210720FFF769FB4FF0402004
:104EF000816941F400518161C16941F40051C1618E
:104F0000934A0021116093495160DFF83CC20021AF
:104F10009CF800303BB10CF110031C6894605B6896
:104F2000D3608CF800108C491161816921F4005123
:104F30008161C16921F40051C16110BD824840689E
:104F400070478348806970474FF04020806910F4B3
:104F5000005008BF70477E48006900F001007047AC
:104F60004FF04020806910F4005F04D0784B18693E
:104F700010F0010F01D10020704710B472494FF6B4
:104F8000FE7000248A684AB19A69D1F808C0624567
:104F900004D08C604C6010BC0120704700BF00BF83
:104FA00000BF00BF00BF00BF00BF00BF00BF00BF09
:104FB00000BF00BF00BF00BF00BF00BF00BF00BFF9
:104FC00000BF00BF00BF00BF00BF00BF401E0028E1
:104FD000D8DC8C604C6010BC002070475A49886057
:104FE00070475948806870475948016941F001018C
:104FF000016155490120486070475548016921F019
:1050000001010161504900204860704700210028DB
:1050100008BF4FF0006103D0022808BF4FF0806145
:105020004B48026922F040621143016170474849D0
:105030000120096901F04061B1F1806F04BF0220D5
:105040007047B1F1006F08BF0020704740484069C9
:1050500070473D48007870474FF04020806910F459
:10506000005F38D03A4A106910F0010F33D036484B
:10507000406801282FD090696FF07F43984238BF75
:1050800000EB400C27D25169B1EB9C0F01D30120FA
:10509000704700BF00BF00BF00BF00BF00BF00BF20
:1050A00000BF00BF00BF00BF00BF00BF00BF00BF08
:1050B00000BF00BF00BF00BF00BF00BF00BF00BFF8
:1050C00000BF00BF00BF00BF00BF00BF00BF00BFE8
:1050D00000BF9842D7D30020704710B50720FFF7D4
:1050E000A9FA0720FFF78EFA1948016941F010016B
:1050F000016110BD164810B5016921F01001016170
:105100000720FFF78BFABDE810400720FFF792BA9F
:105110000D4AD168D0600846704738B50C4CE0693C
:10512000E061094910F0020F1CBFA2698A60C968DA
:1051300000291CBF00018847E0690090074801680A
:1051400041F08001016038BDB4840010C4840010B7
:1051500000D00040D0121300660F00157C840010B0
:10516000704770B505464FF40D500406A066032045
:10517000E066264860664CF2710020662448C4F858
:10518000800042F24630A06602210020FFF717FAA5
:105190000020FFF737FA002D08BF70BDA06E42F265
:1051A00041310843A06670BD012110B588078167B1
:1051B0004FF40D5181660020FFF730FABDE8104032
:1051C0000020FFF737BA01208107486770470120A8
:1051D0008107886770474CF2710081070866704745
:1051E0000C4A11681060084670470A4808B5006804
:1051F00018B18047002818BF08BD4CF2710188071C
:105200000166016FC166006F009008BD075E5F37E1
:1052100000AF2F91F4840010FE4900208871704780
:10522000FC488079704770B5FA4C00254FF4E46172
:105230002570E570F8481AF0D6F94FF4E461F748A4
:105240001AF0D1F9A56025714C21F5481AF0CBF977
:105250004C21F4481AF0C7F965717421F2481AF02C
:10526000C2F97421F1481AF0BEF9E56070BDE94851
:105270000079002818BF01207047E64840790028CF
:1052800018BF01207047E348C078002818BF0120EC
:105290007047E548704770B5E54DE64E0446014657
:1052A0002A783078E04B1044420018461AF0A5F9ED
:1052B0002A783078DD4B10444200214618461AF017
:1052C0009CF9D44801214171817941F00401817137
:1052D00070BDD048C0687047CF4870472DE9F04195
:1052E000CC4F80463878002814BFD348D34805787F
:1052F00014BFD348D348047805FB04F6FEF729FF12
:1053000021462846FEF777FFC3494346C34A08466D
:10531000FEF792FFFEF72EFF72004146BF481AF0DB
:105320006CF90120F870B87940F00100B8710120E3
:10533000BDE8F0812DE9F047B64D044601462878D6
:10534000DFF8D4C2DFF8F082DFF8F092BC4EBD4F38
:10535000002815BF98F8002099F8002033783B7892
:1053600002FB03F04FEA400260461AF046F9287843
:10537000DFF8A8C22146002815BF98F8002099F848
:10538000002033783B7802FB03F04FEA400260468E
:105390001AF033F90120E870A87940F00100A871F3
:1053A000BDE8F0879B488068704770B5A64C0546FD
:1053B000014622789A4852001AF01FF922782946AD
:1053C000520098481AF019F9924801210171817927
:1053D00041F00201817170BD2DE9F04FADF25C7DAD
:1053E000DFF830820120CDF8400798F80300CDF8AF
:1053F0003C0798F80400CDF8380798F805B001F09C
:10540000DBFF0446FDF76CFACDF85807FDF7A8FC62
:10541000CDF85407FBF7FBFFCDF85007FBF746FD2F
:10542000CDF84407FBF73FFD0646FDF75BFAFCF7B6
:1054300094F80830050998F80100002804BF0420FA
:10544000C8F8140014D001F0CFFF0746022C19D081
:1054500008F00CFC02280CBF09200720C8F8140033
:10546000062F04BF0220C8F81400002088F80100AD
:10547000FBF71CFD10F0010F12D002F00AF93C28D6
:1054800008D00DE014F0B9FD10F4817F14BF3C206A
:105490001E20E3E7FFF758FD002818BFFFF7DCFDEB
:1054A0004FF00109022E14D102F0A6F888B9022C9F
:1054B00004D0052C08BF052007D00AE04FF47A700D
:1054C00068434FF47A7190FBF1F0C8F8140088F843
:1054D0000190D8F814000428BCBF0420C8F81400B8
:1054E00098F80100B8F81410000240EA014040F0BA
:1054F00001020023912107200CF01AF8DDF844077F
:1055000010F0010F25D1022C23D00020FBF784FFDF
:10551000FDF765FC0025AA4607F0E2F901281ED038
:105520000DF5E460FDF725FF002800F0E7810DF59B
:10553000E46007F0FDFED8F81400C01EA842ACBF1E
:1055400001260026DDF82C0748B3DDF8380750B1F6
:1055500044E0FDF70BFC0020CDF84007DAE74FF000
:10556000010A00F0B5B96846DDF82C171AF04FF8BB
:105570000746AEB1344C39462078420028481AF02C
:105580003CF820783946420026481AF036F888F868
:10559000049098F8060040F0020088F806001DE02C
:1055A000FEF7D7FD284C01212078FEF724FE1D4A86
:1055B0003B46A2F14C010846FEF73EFEFEF7DAFD3F
:1055C00020783946420017481AF017F888F80490F6
:1055D00098F8060040F0020088F80600DDF8280779
:1055E000002800F0EC80DDF83C07002840F0E78060
:1055F00098F80000DDF82847002877D1D8F808701F
:10560000F7B30D480078CDF84C070D480078CDF879
:1056100048071BE0F884001034210110148B00109F
:1056200074A00010C0A00010542801100CA100109C
:105630004685001047850010448500104185001004
:10564000458500104285001048850010FEF781FD59
:10565000DDF84817DDF84C07FEF7D3FD21463A4642
:105660000846FEF713FEFEF785FDF648007802288F
:1056700004BF384607F07FFBF2480078092800E0B5
:1056800003E004BF204607F076FBEF4800780128CE
:1056900011D9EC4F3878042804BF204607F06BFB83
:1056A0002146684619F0B8FF04463878052804BF3B
:1056B000204607F060FB01F09FFFB8B1E3480022ED
:1056C0000378E3480778002F10D90020002B0AD96F
:1056D00002FB0301401C34F911C083424FEAEC0C79
:1056E00024F811C0F4D8521CBA42EED37EB398F815
:1056F0000020D8482146002A0CBFD44AD64A127846
:1057000014BFD64BD24B1B7802FB03F24FEA420286
:1057100019F073FF98F80000D14B2146002814BF00
:10572000CD48CA48027814BFCC48C948007802FB6B
:1057300000F04FEA4002184619F05FFF88F8039026
:1057400098F8060040F0010088F8060030E0FFE716
:10575000CDF8484798F80000002814BFBE48BB4861
:10576000077814BFBD48BA48047807FB04F0CDF8A9
:105770004C07FEF7EEFC21463846FEF73CFDB549E6
:10578000B74A0846DDF84837FEF756FDFEF7F2FC4B
:10579000DDF84C07DDF848174200B14819F02DFF3D
:1057A00088F8039098F8060040F0010088F8060099
:1057B000A4480078032804BFA64807F0DCFADDF807
:1057C0003007002873D0BBF1000F70D1044698F861
:1057D000000038BBD8F80C7027B3A2480178A24863
:1057E00000780844401C4008019002200090FEF719
:1057F000B0FCDDE90010FEF704FD21463A460846FC
:10580000FEF744FDFEF7B6FC98480078022804BF76
:10581000384607F04CFC95480078092804BF20461C
:1058200007F045FCD6B192488E4E8F4F2146337813
:105830003A781A44520019F0E0FE32783B788D48ED
:105840001A442146520019F0D8FE88F8059098F8BD
:10585000060040F0040088F8060021E08148264652
:105860000178814800780C18FEF773FC601C400832
:105870000221FEF7C0FC7E4933467E4A0846FEF709
:10588000DBFCFEF777FC620031467A4819F0B5FE82
:1058900088F8059098F8060040F0040088F80600A3
:1058A00072480078032804BF714807F000FCFDF738
:1058B000B1FDDDF8440710F0010F18BFFBF799FEAA
:1058C0006D1CD8F81400A84211DCD8F8100070B193
:1058D000FDF708F8DDF85007FBF79EFDDDF85807E7
:1058E00088B1DDF8540760B1FDF779FA0BE0DDF817
:1058F0004007002818BFFDF772FA0DE601F0C2FD5F
:105900000AE6FDF733FABAF1000F04BF0420C8F825
:10591000140009D0DDF83C0788F80300DDF83807EB
:1059200088F8040088F805B0B8F814104FEA0A2087
:1059300040EA01420023912107200BF0F9FD0DF20E
:105940005C7D5046BDE8F08F10B50024FDF7E0F90E
:10595000494910F0070F0AD0CA78002A08BF01246D
:1059600010F0020F03D00A79002A08BF012410F0BA
:10597000F00F03D04879002808BF01240020002C34
:1059800008BF10BD00200870BDE8104024E508B530
:1059900040F20F3101F0AAFE012804D1FFF7D4FF35
:1059A000009002F018F83448C17800291CBF4179F2
:1059B000002904D0007900281CBF012008BD002068
:1059C00008BD08B540F20F3101F090FE012804D166
:1059D000FFF7BAFF009001F0FEFF2748C1780029C9
:1059E0001CBF4179002904D0007900281CBF012088
:1059F00008BD002008BD70471F4910B50022CA70BD
:105A00000A714A7100281CBF012048700CF082FE08
:105A1000BDE81040FAF7E6BC002818BF012016497F
:105A2000C87170471448C079704710B54FF4E461ED
:105A3000084819F0D8FDBDE810404FF4E46108486B
:105A400019F0D1BDC18500104385001041850010BB
:105A50004285001034210110448500104585001056
:105A6000148B00104685001047850010C785001074
:105A7000542801100CA10010F8840010F948704758
:105A8000F9480178F948007848434100F54819F091
:105A9000AABD70B50646F4480478F4480578FEF7C8
:105AA00058FB29462046FEF7ACFBF14A3146ED484B
:105AB000FEF7ECFBFEF75EFBEE480078152818BFFA
:105AC00070BDE848BDE8704007F055B970B50446B0
:105AD000E5480578E5480678FEF73BFB3146284661
:105AE000FEF78FFB2246E2491046FEF7CFFBFEF79A
:105AF00041FBE0480078162804BF204607F03BF938
:105B0000204670BD002818BF0120DB49C8707047CF
:105B100010B5D94C002804BFA06010BDDFF85CC3ED
:105B2000D7490B78D7490A7801465A435200604654
:105B300019F063FDD148A06010BD10B54C21D248CA
:105B400019F051FDBDE810404C21D04819F04BBD73
:105B5000CD487047002818BF0120C7490871704719
:105B600010B57421CA4819F03EFDBDE810407421FB
:105B7000C84819F038BD002818BF0120BE49487137
:105B8000704710B5BC4C002804BFE06010BD742203
:105B90000146C14819F031FDBF48E06010BD70B545
:105BA000B54D00210446E970297169710CF0B2FD10
:105BB000FAF718FC002C14BF012000202870BDE863
:105BC000704009E42DE9F04F89B04FF4E461AB482F
:105BD00019F009FD7421B04819F005FDFDF798F89A
:105BE0000446FCF77DFE0890FDF7BAF80790FBF736
:105BF0000EFC0690FCF776FEFBF758F910F0010F4B
:105C00000BD001F046FD3C2807D1FFF79DF920B1EC
:105C10000420FFF748F9FFF71FFA0020FBF7FCFB11
:105C2000FDF7DDF800252E4606F05AFE012853D078
:105C30006846FDF79EFB00285ED0684607F078FBBB
:105C400014F0070F1CD08E48DFF830B2DDF8089052
:105C500090F800808B48DA460778FEF77AFA012040
:105C6000FEF7DDFA39464046FEF7CBFA5246494682
:105C70005846FEF70BFB0020FEF7D1FAFEF77AFA42
:105C800014F0F00F20D08548DFF80CB2022701781D
:105C90008348DA46DDF8109000780844401C4FEA4B
:105CA0005008FEF756FA0120FEF7B9FA3946404689
:105CB000FEF7A7FA524649465846FEF7E7FA002093
:105CC000FEF7ADFAFEF756FAFDF7A4FB6D1C102D9A
:105CD00003D2FDF784F8A7E701260520FFF7E3F8D4
:105CE000FCF700FE0698FBF797FB089848B1079869
:105CF00028B1FDF774F804E001F0C4FB94E7FDF768
:105D000035F8DEBB5C4F14F0070F1BD05C48DFF8A2
:105D10006CC101785B48E046007801FB00F210207E
:105D20000021002A88BF03460AD938F9115005EB33
:105D30005005B5FBF3F52CF81150491C8A42F4D8F4
:105D40004E48B86014F0F00F18D05448524B017808
:105D500053481C4600780A184FF010014FF000001D
:105D60000AD034F9105005EB5105B5FBF1FC23F8CE
:105D700010C0401C8242F4D84748F86009B0304651
:105D8000BDE8F08F012070474FF47B3070474FF42F
:105D90007B3000687047034600209A682C2A88BF31
:105DA0002C220021B1EB920F28BF704753F821C07D
:105DB000491C6044B1EB920FF8D37047394A01682F
:105DC000914214D14168B1F5807F10D983680022D7
:105DD0002C2B88BF2C230021B1EB930F09D250F854
:105DE00021C0491C6244B1EB930FF8D30AB10020E3
:105DF0007047012070474FF47B312A4B0A689A4262
:105E000060D191F827300022012B08BF012205281C
:105E100004BF91F82300704713DC012804BF087FFA
:105E20007047022804BF91F820007047032804BF80
:105E300091F821007047042804BF91F822007047B0
:105E400053E0142808D015282ED0162833D0172850
:105E500004BF1846704748E0002A1CBF91F8240090
:105E6000704726E0349200104185001042850010F2
:105E700034210110C1850010F884001054990010DD
:105E8000448500104585001074A00010C0A00010CB
:105E9000542801100CA1001080A1001046850010AC
:105EA000478500104353494D002A1CBF91F8250037
:105EB00070472D207047002A1CBF91F826007047BC
:105EC00028207047052812D007DC01280DD00228B1
:105ED0001CBF032804280AD007E0142818BF15287F
:105EE000E7D01628ECD0172801D0FF2070470020FB
:105EF00070472DE9F047ADF5007D00244FF40071A7
:105F0000684619F070FBFF20A04660F307082D20BB
:105F1000254660F3070560F30F25282060F3174539
:105F20004FF47B37F74E64F31F654FF481794FF0E0
:105F30002C0AFF224FF40071684619F072FBCDE97C
:105F400002A4CDE9064805940A94CDE900690494B9
:105F5000CDE908453846FDF71FFF69463846FDF78D
:105F6000BDFF012818BF00200DF5007DBDE8F087BA
:105F70002DE9F047ADF50C7D894605461F46904654
:105F80004FF0000A4FF400716846949E19F02BFB05
:105F90004FF0000CCDF800C24FF47B34CDF804C2B2
:105FA000CDF808C2CDF80CC2CDF810C2CDF814C29D
:105FB000CDF818C2CDF81CC2CDF820C2CDF824C24D
:105FC000CDF828C2CF492068884206D0FFF791FF5C
:105FD0000DF50C7D5046BDE8F087D4E901120DF5B2
:105FE000007AE3688AE80F0004F110010DF5047AE5
:105FF0000FC98AE80F00D4E90801A26A8A92CDE9A4
:10600000880184988DF820928DF82182401C8DF8AB
:1060100022728DF81C528DF823628490002D14BFDB
:106020008698859800F1010014BF8690859080AB1A
:1060300082980021CDF80CC22C2894BF02462C2255
:106040000020B0EB920F06D253F820C0401C6144F0
:10605000B0EB920FF8D348428390FF224FF40071C7
:10606000684619F0DEFA80AC94E80F008DE80F0066
:1060700084AC94E80F0004AC84E80F00DDE98801EB
:106080008A9A4FF47B34CDE908010A922046FDF745
:1060900083FE69462046FDF721FF012818BF002036
:1060A0000DF50C7DBDE8F0872DE9F041ADF50C7DD7
:1060B0000F46804616464FF40071684619F093FA71
:1060C000002580954FF47B34819582958395849546
:1060D000859586958795889589958A9589492068BB
:1060E000884218D16068B0F5807F14D9A068214635
:1060F0004FF0000C2C2888BF2C200023B3EB900F0E
:1061000011D251F823205B1C9444B3EB900FF8D3C9
:10611000BCF1000F07D0FFF7ECFE002804BF0DF51F
:106120000C7DBDE8F0810FCC0DF5007C8CE80F00F4
:106130000FCC0DF5047C8CE80F00D4E90001A268B7
:106140008A92CDE988018DF824828DF825728DF828
:10615000266201208DF827028298002180AB83956A
:106160002C2894BF02462C220020B0EB920F06D2BE
:1061700053F820C0401C6144B0EB920FF8D3484262
:106180008390FF224FF40071684619F04AFA80AC00
:1061900094E80F008DE80F0084AC94E80F0004AC85
:1061A00084E80F00DDE988018A9A4FF47B34CDE959
:1061B00008010A922046FDF7EFFD69462046FDF7EB
:1061C0008DFE012818BF00200DF50C7DBDE8F08183
:1061D0002DE9F04F4C4D4FF0000885B06C4247461A
:1061E00046461720FFF707FE4FF47B3284464549A9
:1061F0001068884217D15068B0F5807F13D9936832
:1062000000212C2B88BF2C230020B0EB930F80F0B3
:10621000FF8052F82090401C4944B0EB930FF8D314
:10622000002900F0F580FFF764FE002804BF05B0E8
:10623000BDE8F08F1420FFF7DEFD02901520FFF778
:10624000DAFD00901620FFF7D6FD40B2019016202F
:10625000FFF7D1FD404240B20390FCF759FDDFF853
:10626000AC908246002089F8030089F8040089F880
:1062700005000CF04FFAFAF7B5F8002089F8000095
:10628000FFF7AAF81AF0F00F05D019F0CFF901289E
:1062900008BF48F001081AF0070F7DD01C481E4ABD
:1062A000002690F800E01B48037899F80200A3EB61
:1062B000000984468145C4BFAEEB0C01A1F1010B7E
:1062C0001CDD61468B4516DD01F1010A01FB030768
:1062D0000AFB030A32F8177032F81AA0A7EB0A0774
:1062E0003FB2002FB8BF7F423FB2B742C8BFBEB275
:1062F000491C8B45E8DC401C8145E2DC0098002805
:106300000CE000004353494DF1D8FFFFF884001022
:1063100042850010418500103421011018BF8642CB
:1063200088BF48F002080027E246AEEB0A00009062
:106330005045C8BFA9F1010B1BDD6046834513DD45
:106340000AFB030132F811E002EB41014988AEEB90
:10635000010109B20029B8BF494209B2B942C8BF18
:106360008FB2401C8345EBDC00980AF1010A5045CE
:10637000E3DC0298002818BF874288BF48F0040871
:10638000E2460098504516DD614689450EDD0AFB60
:10639000031032F9100000E017E0A842C8BF05461C
:1063A000A042B8BF0446491C8945F0DC00980AF1B8
:1063B000010A5045E8DC0198002806DD854202DC30
:1063C0000398844201DA48F00808FF2F88BFFF27AE
:1063D000FF2E88BFFF267F2DC8BF7F2504DC15F167
:1063E000800FB8BF6FF07F057F2CC8BF7F2404DC0F
:1063F00014F1800FB8BF6FF07F04E0B20090EBB2F1
:10640000F2B2F9B24046FFF7B3FD05B0BDE8F08F38
:10641000BCF1000F18BFBCF1010F3FF40BAF02E756
:10642000FE4988707047FD4890F902007047FB48AC
:1064300000787047F94840787047F8480021C171EA
:10644000417141728172C1727047F44920F07E40FF
:10645000C8617047F148C0697047F048408A70478A
:10646000EE48808A7047ED48B0F916007047EB4857
:10647000B0F918007047E948B0F91A007047E748CA
:10648000007B7047E548C078002818BF012070479E
:1064900010B54FF4E461E24819F0A5F8DF49002097
:1064A000C87010BD2DE9F74F90B000250C46DD49AE
:1064B0000195029503950495059506950795089510
:1064C000099508681746052A08BFB0F9786005D015
:1064D000062F0CBFB0F97A60B0F97460B0F976009D
:1064E000B04209DA13F089FD10F4817F03D0CD4862
:1064F0000068B0F8766036B2324601A9109819F0FB
:106500009AF8059800B22080BDF826106182BDF887
:106510001E106181BDF82010A181BDF82210E1811B
:10652000BDF824102182BDF81810A180BDF81A1002
:10653000E180BDF81C1021810028B8BF25808DF8AE
:106540002850B948B94900788DF82A008DF82950AB
:1065500009788DF82B107142ADF82E10ADF830008F
:1065600080B2ADF82C60ADF80000DDE90A232146C9
:10657000109800F0C1FC052F11D0E582A58225837B
:10658000A088002804BF4FF40040A0806089002844
:1065900004BF47F6FF70608113B0BDE8F08FFEF7CF
:1065A0009BFE002119F04CF8002800F0F180DDF886
:1065B00028C0DDE90B0ACCF3072310994FEA1C62CF
:1065C000ADF80050ADF8345099469A4269D91FFA97
:1065D0008AF50CF0FF0603FB056E1FFA8EF80E9588
:1065E00031F91880BDF80060BDF834500FFA80FB17
:1065F000D845C4BF761CB6B24FEA204BD845BCBFC5
:106600006D1CADB2ADF800600EF101081FFA88F8FC
:10661000ADF8345031F918800FFA80FBD845C4BF6B
:10662000761CB6B24FEA204BD845BCBF6D1CADB24C
:10663000ADF80060DDF83880CCF3074B03FB08BEF3
:10664000AEF102081FFA88F8ADF8345031F918801D
:106650000FFA80FBD845C4BF761CB6B24FEA204B78
:10666000D845BCBF6D1CADB2ADF80060AEF10108FD
:106670001FFA88F8ADF8345031F918800FFA80FB12
:10668000D845C4BF761CB6B24FEA204BD845BCBF34
:106690006D1CADB2ADF800605B1CADF834509A4291
:1066A00095D80CF0FF03CCF3074E9E456CD91FFA2A
:1066B0008AF609FB063C1FFA8CF8BDF800C031F9D8
:1066C00018800FFA80FBADB2D845C4BF0CF1010CA5
:1066D0001FFA8CFC4FEA204BD845BCBF6D1CADB2F5
:1066E000ADF800C009F1010808FB06381FFA88F868
:1066F000ADF8345031F918800FFA80FBD845C4BF8B
:106700000CF1010C1FFA8CFC4FEA204BD845BCBFA2
:106710006D1CADB2ADF800C0A2F1020808FB06384E
:106720001FFA88F8ADF8345031F918800FFA80FB61
:10673000D845C4BF0CF1010C1FFA8CFC4FEA204B6A
:10674000D845BCBF6D1CADB2ADF800C0A2F10108C8
:1067500008FB0636B6B2ADF8345031F916600FFAC0
:1067600080F84645C4BF0CF1010C1FFA8CFC4FEABF
:1067700020484645BCBF6D1CADB2ADF800C05B1CE7
:10678000ADF834509E4592D8E582BDF80010A18244
:10679000DDF830900A9E109D4FF0000C052F4DD073
:1067A0002048062F006803BFB0F87A100227384649
:1067B000B0F874101CBF01270020B4F90230B4F9FE
:1067C0000020934241D18A423FDDC6F307210144B4
:1067D000C0EB166A8A452ED9C6F30742F0B2D21B27
:1067E0003844A2F10108804517D91FFA89F201FB4C
:1067F000020292B235F9123005EB4202B2F90220E0
:10680000B3EB020B48BFA2EB030B0FFA8BF262450E
:10681000C8BF9446401C8045E7D809E010850010A9
:10682000F4A100100C870010418500104285001073
:10683000491C8A45D0D8A4F818C0A1E6FE48022712
:106840000068B0F878103846B7E7228398E6084326
:1068500018BF7047F948C16911F0807F08BF7047C1
:10686000F5490968096F11F4003F08BF704700211E
:106870001170182101827047F048406A70472DE975
:10688000FF5FEF480027DDF83CA005780E98119EC9
:106890008B46B9463C4650452CD006FB050E109859
:1068A0003BF91EC006FB05093BF91900BCEB0001D2
:1068B00048BFA0EB0C0106FB05A83BF91840B4EB60
:1068C000000C48BFA0EB040C01EB0C0004B232F941
:1068D0001EC032F91900BCEB000148BFA0EB0C014F
:1068E00032F918C0BCEB000248BFA0EB0C028818BC
:1068F0000FFA80F9012B37D04FF0010818F0A5FEF0
:10690000D049002C0A7807DD109906FB05113BF9E8
:1069100011101431282909D80099B1F914103C2913
:1069200004DC0099B1F916103C2926DD0E9902EB22
:106930000A0C11448C4520D9129B139D13442A4400
:106940008B421CBF8D1A15F1020F30F9115000EB6C
:106950004106B6F90260A5EB060508D01E353C2DB0
:1069600008D94FF0000808E0A1450CDD0AE00A351F
:10697000142DF6D8491C8C45E2D8A14503DDB8F1A9
:10698000000F00D0012704B03846BDE8F09F7047E3
:10699000AA48B0F90E007047A8490020C881704786
:1069A0000021018041804FF400428280C18001813A
:1069B000521E42818181C181018241828182C182D4
:1069C000018370479D4980208870704770B59B4D4A
:1069D00004466FF07F06686A844209D044EA0122C7
:1069E00000236B2107200AF0A3FD002C08BFAE7026
:1069F000686A204308BFAE706C6270BD2DE9F04735
:106A00008A460646002513F0E0FA044613F0D9FA48
:106A100004FB00F1894F0AB22044002497F90210C8
:106A20007B6AA1466FF07F084BB1B7F91A10323A72
:106A300091421EDD0124BAF1000F16D107E011F1D9
:106A4000800F18BF0A29A8BF0225EEDB3CE0002119
:106A500000280AD936F91120B2F5487F01DA00245E
:106A600007E0491C8142F5D31CB1786A01282BD17B
:106A700006E010F0E3FD01280CBF01240125F4E736
:106A800014B3386A4EF6C42188420BD200F09AFC47
:106A90000021022811D0042808BF4FF4FA71386A87
:106AA000084438624EF6602181420FD20325C7F8B0
:106AB0002090002487F8028008E00BF028FE0028D0
:106AC00014BF11210821EAE7C7F82090786A8442B0
:106AD0000AD044EA052200236B2107200AF028FD92
:106AE000002C08BF87F80280786A204308BF87F827
:106AF00002807C62BDE8F0872DE9FF4F8BB04F4DDF
:106B0000DDE918A704460020287068700BF013FE1A
:106B1000002840F0448100F04FFC052871D0287B0C
:106B2000019049494448DDF8309091F800B0006880
:106B3000444990F8866009780091B0F98480B5F9ED
:106B400018003228688A05DA002804BF7006060E8D
:106B500004D100E010B9287901282BD10BF02AFECE
:106B600040BB012F26D0BAF1010F02D1A88AC82854
:106B700020D8A88A002804BF688A00281AD00BF001
:106B8000C6FD012819D0B9F80000E881009900205D
:106B90001BEB01030AD039F91010B5F90E20914210
:106BA000C8BFE981401C80B28342F4D8B5F90E0019
:106BB00040450EDD0020A87223E01F48006890F8D1
:106BC00087600198012814BF4FF03C084FF041083E
:106BD000D9E7E86910F4803F13D017480068006FC8
:106BE00010F4803F0DD0A87A401CC0B2A872B04209
:106BF00007D9102028820120287200204FF0FF348E
:106C0000A87210F01BFDA0B100F0DCFB042810D12D
:106C1000287F10F0800F0CD00748006890F87000B3
:106C200010F0800F05D00720288201204FF0FF349C
:106C300028720BF06CFD09E00C8700101085001025
:106C4000418500104785001046850010012871D14C
:106C5000FE48BAF1000F00680A9090F888106BDCCB
:106C6000012F69D0E86910F4003F12D00A98006F34
:106C700010F4003F0DD0687A401CC0B268728842A0
:106C800007D9112028820120287200204FF0FF34FC
:106C900068720C980090EE484FF0000B012F0078BE
:106CA0000390EC48007801900A9890F887000690CD
:106CB00045D00198400807900398400809900020AB
:106CC000049082460590DDE9001001EB400002903F
:106CD00000231A461946BAF1000F0CBFDDE9007611
:106CE000DDE902760020002E88BFA6F1010E29D929
:106CF00037F91080B8F1640FD8BF002214DD704559
:106D00000DD207EB400CBCF902C0B8EB0C0948BF30
:106D1000ACEB08090FFA89FCDC45A8BFE346491C27
:106D2000002A04BF01225B1C401C8642E0D8012BD4
:106D300005D807E033E0FFE700206872A9E70020EC
:106D4000E8722CE0BAF1000F0CBF049105910AF132
:106D5000010ABAF1020FBBD3079904988842EED911
:106D6000099905988842EAD9BBF1320FE7DCE87A45
:106D7000401CC0B2E872E96911F4801F0FD00A9973
:106D8000096F11F4801F1CBF0699884207D914208F
:106D900028820120287200204FF0FF34E87213F09F
:106DA0002CF910F4807F28D000F006FB022824D1B3
:106DB0004FF0010818F04EFC074613F006F906469E
:106DC00013F0FFF8024600210020002E08D900FB36
:106DD000021337F913300F2B0FDB401CB042F6D3F0
:106DE000B8F1000F09D0491C0129EDD9B8F1000F05
:106DF00003D001204FF0FF3428720EF05AFD032813
:106E000023D1002000900190287C8DF80000BDF86F
:106E10000000022264F30F20ADF80000E979BDF80C
:106E2000020061F30300697961F30710297A61F3C5
:106E30000820A97961F34920ADF80200E889ADF88E
:106E40000400062168460EF037FDB4F1FF3F26D05E
:106E5000002C07BFA87901280FB0BDE8F08FFEF71E
:106E60000FFE0024AC71012028704FF4E4617A48D1
:106E700018F0B9FBEC7000F0A5FA04280D982CD09E
:106E8000002818BFFEF756FA0E98002804BF0FB06E
:106E9000BDE8F08F0FB0BDE8F04FFEF7FCB9287ADF
:106EA00001281CBF0FB0BDE8F08F0D98FEF7F1FD73
:106EB00000242C72012068704FF4E461664818F0D9
:106EC00092FBEC700D98002818BFFEF733FA0E986D
:106ED0000028DFD10FB0BDE8F08F002818BFFEF703
:106EE000FDF90E98002804BF0FB0BDE8F08F0FB079
:106EF000BDE8F04F18F0B3BB2DE9F8070023DDF82B
:106F000020C0C2F30724ADF80030160E2546D3B2D8
:106F10001FFA8CFCC2F30747A64259D904FB0C3870
:106F20001FFA88F230F9129000EB4202B2F902A087
:106F3000B9EB0A0248BFAAEB090212B2BDF90090F0
:106F40009145B8BFADF8002008F1010292B230F9C6
:106F5000129000EB4202B2F90280B9EB080248BF7E
:106F6000A8EB090212B2BDF900809045B8BFADF898
:106F7000002004FB0C78A8F1030292B230F91290C1
:106F800000EB4202B2F902A0B9EB0A0248BFAAEB39
:106F9000090212B2BDF900909145B8BFADF80020CA
:106FA000A8F1020292B230F9128000EB4202B2F96B
:106FB0000290B8EB090248BFA9EB080212B2BDF972
:106FC00000809045B8BFADF80020641CA642A5D84B
:106FD000A7F10108984563D96F1CB41E761E05FB06
:106FE0000C3292B230F9129000EB4202B2F902A0D8
:106FF000B9EB0A0248BFAAEB090212B2BDF9009030
:107000009145B8BFADF8002007FB0C3292B230F9C1
:10701000129000EB4202B2F902A0B9EB0A0248BF9B
:10702000AAEB090212B2BDF900909145B8BFADF8C4
:10703000002004FB0C3292B230F9129000EB4202B5
:10704000B2F902A0B9EB0A0208E000000C870010B8
:107050004685001047850010F4A1001048BFAAEB38
:10706000090212B2BDF900909145B8BFADF80020F9
:1070700006FB0C3292B230F9129000EB4202B2F9E8
:1070800002A0B9EB0A0248BFAAEB090212B2BDF98D
:1070900000909145B8BFADF800205B1C98459ED884
:1070A000BDF800004880BDE8F80770472DE9FF4FA4
:1070B000DFF8C0B2044689B0DBF800001D46164672
:1070C000B0F87AA012F0C9FB012804BF4FF6FF7098
:1070D00000EA4A0A12F091FF10F4817F07D0B5F957
:1070E000141001232046169A18F0BEFA04E001227B
:1070F00020461699FFF7D6F99F4F002425463C718C
:10710000DDF82880FEF7E8F80094019402940394D7
:1071100004940594069407940894DBF800006946EB
:10712000B0F87420404618F086FADBF80010BDF97C
:107130001A00B1F9741049428842B8BF0125BDF860
:107140002000B0F5E17F88BF01258B48057112F062
:1071500054FF10F4817F0DD11698B0F91200002869
:1071600008DC0BF0D4FA012804D083480079012808
:1071700040F0CA8012F041FF10F4817F00F0BC8023
:1071800047F6FF7003907D484FF00009179C007888
:1071900001907B484D46077812F02FFF10F4817F55
:1071A0000EBF5046DBF80000B0F876000FFA80F80A
:1071B00012F023FF10F4817F1DBFDBF80000B0F850
:1071C00076004042CAF1000000B2029012F015FFB2
:1071D00010F4807F19BF4FF0010B4FF0220C4FF0DD
:1071E000000BBC46002000900398804568DADDE97A
:1071F000002000287CD9ACF1010005900198401EC8
:107200000490ACF1020003905846E34538BF13B236
:1072100051D202FB070A1FFA8AF136F91110002930
:10722000B4BFC1F1000E8E46C6451ADD41450BDDE7
:10723000B4F904E0714502DDA180E080238109F109
:1072400001010FFA81F90CE0DDF808E08E4508DD58
:10725000B4F90AE08E4502DD6181A081E381691CF9
:107260000DB20599884223D206EB4A0136F91AE09D
:10727000B1F902A0BEEB0A0148BFAAEB0E0109B2A8
:10728000DDF800A052451CBFDDF810A0524505D026
:1072900058451CBFDDF80CA0504504D1B4F902A03C
:1072A0008A45B8BF6180B4F900A08A45B8BF218083
:1072B000401C6045ADD30198521C8242A4D317E014
:1072C000DDE90001002913D95B46E3450CD200FB40
:1072D000073189B236F9112002998A42BCBF691C74
:1072E0000DB25B1C6345F2D30199401C8842EBD37D
:1072F000A4F81090658204E0062230461799FFF743
:10730000D1F81999012008701798B0F910000028D9
:1073100008DC1798B0F91200002803DC1648007941
:10732000012814D112F069FE10F4817F07D00523E3
:1073300047F6FF71189A0A9818F096F904E00522AA
:1073400018990A98FFF7AEF81A9901200870169854
:10735000418A094841821699098A81821699498988
:10736000C1821699898801831899098A41830DB0D1
:10737000BDE8F08F0C8700101085001042850010CA
:107380004185001010B50AF0D1FF0BF0B3F80020D2
:1073900010BD0000FE49C8707047FD48C0787047B6
:1073A000FB4908717047FA4800797047401E02286F
:1073B00094BF012000207047F54800787047F448DA
:1073C00080787047F2480078022805D005281CBF55
:1073D0000020704706F0FFBA0BF07CB9EC4908704A
:1073E0007047EB4948707047E9484078704770B57E
:1073F000E74E044682B030780D46A0421ED00022EF
:10740000612100928DF800108DF801408DF8025036
:1074100001928DF8030002281FD0052814BF002018
:1074200006F0D9FA8DF8040012F065FE8DF805001B
:1074300007220023694610460AF007F93078844293
:1074400018BF7070B570072C24BF02B070BDDFE8A4
:1074500004F016070B13160F16000BF03BF9E1E7CB
:10746000284600F0C7FA0AE028460BF0DBF906E0F0
:10747000284606F0A5FA02E028460AF04BF93470D7
:1074800002B070BDC34900200968B1F8B01011F412
:10749000807F08BF7047FCF79ABBBE49002009688F
:1074A000B1F8B01011F4807F08BF7047FCF79EBBA5
:1074B000B84900200968B1F8B01011F4007F08BF86
:1074C000704718F0D6B8B249487900281CBF401E52
:1074D0004871704770B5B0480068AD4C10F0130F9C
:1074E0000FD010F0100F05D0AC4951F88C2F42F49A
:1074F00080520A60AA4908606079002804BF012010
:1075000060714FF040208069A24D10F0020F296891
:1075100006D1A448006810F0010F01D0607940B195
:10752000B1F8B010002011F4807F18BFFCF75EFBAB
:1075300007E0B1F8B010002011F4806F18BF18F008
:107540009DF89949084208BF70BD2968D1F8B0106C
:10755000090C617170BD10B572B6FDF725FEBDE86E
:107560001040FDF735BA10B5012802D0022805D029
:1075700007E04FF47F30FCF70FFC02E08C498B48AA
:10758000086072B6FDF710FEBDE81040FDF720BAA6
:107590007F4900288A7918BF01208871C0B28242D1
:1075A00008BF70470022002818BF012200230121D4
:1075B000022009F0BDBF76488079002818BF01205D
:1075C000704770B5724C0028E57918BF0120E07152
:1075D000C0B2F8F7E6FEE079854214BF002870BD1E
:1075E000247818F050F8022C1CBF052C70BD022125
:1075F0002046BDE87040FAE66548C079002818BF0B
:10760000012070476248007A70472DE9F041604DD3
:1076100000281CBF0020287204D1287A002818BF37
:10762000BDE8F081634E37683020FCF737FD062156
:107630003020FCF74CFDF06A40F03000F0625E4C08
:107640004FF07F0811E0FDF7C6FDF06A10F0100F53
:1076500003D0287A40F07E002872F06A10F0200FE4
:1076600003D0287A40F001002872201EA4F1010402
:1076700003DD287A38EA0000E5D13020FCF754FD1C
:107680003760BDE8F08142488069704740484069F2
:1076900070473F484069002818BFC07A70473C498E
:1076A000C86170473A48C0697047394908627047F5
:1076B0003748006A70473748026802F5C873118A74
:1076C000508A02F5A872FBF763BC10B506F07DFF87
:1076D000002818BFC07A10BD10B506F076FF00284C
:1076E0000CBF4FF0FF3090F9240010BD2DE9F04F92
:1076F000DFF89CA099B00E46CAF8180006F065FFA6
:10770000CAF8140000287CD090F800C08AF809C09C
:1077100041788AF80A10837804460CF101008AF84F
:107720000B3000F0FE008AF80C00E2788AF80D2099
:1077300020798AF80E0060798AF80F000AF11100AA
:107740004FF0000B80F800B080F801B020788AF884
:1077500010006046FBF7D9FD9AF80F109AF80E005A
:10776000FBF7F6FD6946204606F04DFFE089DAF8A2
:107770001C5000281CBF6843050BB4F81280DAF8CF
:107780002090B8F1000F08BF4FF48058E78A15E049
:10779000388500100C870010184800400030004069
:1077A00014480040144C004008001300AD2007B0FE
:1077B000304C00400010004080380100002F08BF0E
:1077C0004FF480574FF480501890002016F0040FAB
:1077D00018BF052016F0080F18BF40F0020016F081
:1077E000020F18BF40F0F00016F0010F18BF40F470
:1077F000774016F4807F18BF40F4803016F4007F85
:1078000000E03EE018BF40F47E00E16901EA0006B6
:1078100000981090059812900798CDF844B0CDE9E3
:10782000130B01981590A07A17900398169010A941
:107830003046FBF75AF916F0070F61D006F0A3FBAC
:1078400018B101460020F9F7EEFE06F0B3FB6843DD
:10785000050B06F0CFFB09FB00F0000B4030C1091F
:107860000A20012202FA00F30B4201D1401EF9D591
:10787000A0F10509207B002818BFA0F1010B11D150
:107880000CE05A480068B0F8B00010F4807F18BFD0
:10789000FCF7ACF9002019B0BDE8F08F0020FAF732
:1078A000AEF88346607B002814BF401EFAF7DFF86D
:1078B0000BEB0901052905DDA9EB010101F1050922
:1078C000052104E00029BCBFA9EB01090021814486
:1078D000B9F1050F05DDA9F10500C5404FF0050917
:1078E00007E0B9F1000F04DAC9F1000085404FF05C
:1078F00000090020FAF79DF849460020FAF7D1F870
:1079000016F0F00F43D0207C70B116F0100F03D0AA
:10791000411E0120FAF78DF816F0400F04D0207CAC
:10792000411E0220FAF785F8207D70B116F0200F75
:1079300003D0411E1120FAF77CF816F0800F04D016
:10794000207D411E1220FAF774F8607C70B116F0A9
:10795000100F03D0411E0120FAF7A3F816F0400FD4
:1079600004D0607C411E0220FAF79BF8607D70B164
:1079700016F0200F03D0411E1120FAF792F816F0EE
:10798000800F04D0607D411E1220FAF78AF8E07A59
:1079900000281CBF0001F9F77FFD029806F0CFFA1E
:1079A000049830B12B469AF80A209AF8091017F07B
:1079B0006FFE3A4641462846189B17F06EFE069821
:1079C000FEF7A6F80898FEF7DCF80AF0C7FF19B032
:1079D0000120BDE8F08F10B5FBF75DF906F0B7FAAE
:1079E000034900204861012010BD00000C870010F1
:1079F00038850010FE4908707047FD4800787047D0
:107A0000FC4810B4FC4A016891421CD14168B1F5B0
:107A1000987F18D8D0F808C00146BCF5007F12D86E
:107A200000220B461146B2EB9C0F24BF10BC7047DE
:107A300053F82140491C2244B1EB9C0FF8D3002A93
:107A400004BF10BC7047002010BC7047E948FCF729
:107A5000A3B9E7490120087070472DE9F0411746A6
:107A60000E4605461024FFF711FE15F0070F18BF4C
:107A7000062403D115F0F00F18BF08243246102C4D
:107A800028BFBDE8F081002A08BFBDE8F08120448E
:107A90003B4690F920102046BDE8F04106F0DBBDE2
:107AA0002DE9F04FADF6446D0646FFF7EFFD804639
:107AB00016F0070F75D06F4605253846FBF7AFFC6B
:107AC00008F1050498F925104FF464633A462846F6
:107AD00006F0C1FD94F82000002862D1FFF763FC96
:107AE000FFF764FC01285CD14FF0260B12245120D3
:107AF00005F02EF881460021084604F0B7FF054640
:107B00000121002004F0B2FF0746BC48007851284C
:107B100004BF002005F02FF94FF000435A1E00204B
:107B20000BFB04F435F810109942C8BF0B46914284
:107B3000B8BF0A46401C8442F4D8981800EBD070B5
:107B40004110002262F3070AAD4862F30F2A61F385
:107B50001F4A3860C7F804A007F10803002C12D9A7
:107B600035F81200401A00EBD07040107F28C8BFD3
:107B70007F2004DC10F1800FB8BF6FF07F009854B5
:107B8000521C9442ECD8FFF70EFC4FF4443101EB49
:107B9000802004F108023946FCF7F4F9484604F065
:107BA000D7FF16F0F00F04BF0DF6446DBDE8F08F5F
:107BB00007256C46FBF7ACF810F0300F0CBF022025
:107BC00001206946FBF77BFC98F927104FF41873E6
:107BD0002246284606F03FFD0DF6446DBDE8F08FC5
:107BE0002DE9F34F89B0002006900878039048688B
:107BF0000490886805900D7B487B0190887B8A8A79
:107C0000D1E9088BC0F5807602EA00070998B1F93E
:107C10001090B1F912A0896910F0010F07914FF08F
:107C2000000044D000900198002840F2D7800098CE
:107C3000012101FA00F20798104018BF012000242A
:107C40000290610904A804F01F0250F821100120DD
:107C50009040014200F0B7803BF9020B0299A0EB83
:107C60000A0000290CBFA9EB000509EB000538F953
:107C7000020BA0EB0A0014BF4844A9EB0000002D42
:107C8000B4BF694229460028B8BF4042884278D92B
:107C9000224600990398FAF7A5FC0246C0F3042097
:107CA000D1B212F4803F6FD0002D6FDB70E0FAF795
:107CB00002F8009001980321684301EB400020F096
:107CC00003024146584617F098FC0098F9F7F3FF75
:107CD00001984FF0000B002852D90121079801FAB2
:107CE0000BF2104018BF012000250290690904A87A
:107CF00005F01F0250F8211001209040014237D0BA
:107D000038F9020B0299A0EB0A0000290CBFA9EB7D
:107D1000000409EB00042A4659460398FAF762FC6E
:107D2000C0F30421C2B210F4803F02D0002C02DB69
:107D300003E0002C01DD941B00E09419BC4205DD3A
:107D40001F293ABF0024491C3C4606E0002C04DAF7
:107D50000029C6BF3C46491E002400F4783040EAA2
:107D6000012040EA04032A4659460398FAF78DFC9D
:107D70006D1C262DBAD301980BF1010B8345ACD3B2
:107D80002CE020E000E001E0002D01DD8D1900E095
:107D90008D1BBD4205DD1F283ABF0025401C3D4616
:107DA00006E0002D04DA0028C6BF3D46401E00252F
:107DB00002F4783141EA002040EA050322460099A6
:107DC0000398FAF762FC641C262CFFF43AAF009883
:107DD0000199401C00908842FFF429AF09980328BC
:107DE00026BF0120069006980BB0BDE8F08F00007A
:107DF0005C85001000EE030054435246C18500101C
:107E000046544F462DE9F04F8BB0002205920A7878
:107E100000924A6802928A6803924D7B8A7B0492A0
:107E2000B1F91080B1F9122007920C6A8A690892A0
:107E3000898A049AC0F1080A01EA020600283BD0A8
:107E4000BAF1000F7ADB4FF0000B002D77D901203B
:107E500000FA0AF00690AAF10100012101FA00F0EF
:107E600009900121089801FA0BF2104018BF012077
:107E700000270190790902A807F01F0250F821108D
:107E80000120904001427DD034F9021B0798081A66
:107E9000019900290CBFA8EB000908EB00093A463C
:107EA00059460098FAF79EFB034610F4803F72D0C3
:107EB000B9F1000F74DA71E04FF0000B002D3ED9DC
:107EC0000121089801FA0BF2104018BF0120002789
:107ED0000190790902A807F01F0250F82110012033
:107EE000904001424BD034F9021B0798081A0199BF
:107EF00000290CBFA8EB000908EB00093A465946D7
:107F00000098FAF76FFBFE49014011F4803F17D04B
:107F1000B9F1000F29DA11F4F8511CBFA1F58071F5
:107F200041F4803121D110F4604F1ED0A0F50050F3
:107F30004FF4D05110F4003F17D014E04AE042E073
:107F4000B9F1000F11DD11F4F85118BFA1F58071DE
:107F50000BD110F4604F08D0A0F500504FF4D05171
:107F600010F4003F01D04FF48D3100F43830084355
:107F700040F080033A4659460098FAF786FB7F1C8A
:107F8000262F02E016E006E00AE0A2D30BF1010B77
:107F9000AB4595D317E0B9F1000F01DD0698834397
:107FA000BAF1000FC4BF099803433A4659460098F6
:107FB000FAF76BFB7F1C262FFFF45CAF0BF1010B74
:107FC000AB45FFF44EAFBAF1000FC2BF05980BB03E
:107FD000BDE8F08F0027002D2ED904980DF1080A76
:107FE0004FF0010BC0F5807940F4807800246009DF
:107FF00004F01F015AF820000BFA01F1084215D0D5
:10800000224639460098FAF7EDFAC1B201EB590160
:1080100001EA0801B14288BF314620F0FF0040EA82
:108020000103224639460098FAF72FFB641C262CE0
:10803000DDD37F1CAF42D9D3012005900BB0BDE842
:10804000F08F2DE9F04F89B0002204920A78009257
:108050004A6802928A6803924A7B0192B1F91060E1
:10806000B1F912B00C6A8969C0F1050805910028C0
:1080700037D0B8F1000F70DB4FF00009002A6BD940
:1080800008F10800012101FA00FA401E01FA00F08F
:1080900006900121059801FA09F2104018BF01204D
:1080A00000250790690902A805F01F0250F8211069
:1080B0000120904001425FD034F9020B0799A0EBF8
:1080C0000B0000290CBF371A37182A46494600987A
:1080D000FAF788FA034610F4803F3FD0002F41DAC8
:1080E0003EE00027002A4FD90120059900FA07F247
:1080F0000A4214BF4FF0010A4FF0000A0025690937
:1081000002A805F01F0250F8211001209040014202
:108110001BD034F9020BBAF1000FA0EB0B000CBF1F
:10812000A6EB000906EB00092A4639460098FAF743
:1081300059FAB9F1000FC8BF40F4803040F48053C1
:108140002A4639460098FAF7A0FA6D1C262DD6D398
:1081500001987F1C8742C7D316E01AE0002F01DD8B
:1081600023EA0A03B8F1000FC4BF069803432A4666
:1081700049460098FAF789FA6D1C262D92D301988A
:1081800009F10109814584D3B8F1000F04BF012032
:108190000490049809B0BDE8F08F2DE9F04F89B044
:1081A000002204920A7800924A6802928A68039236
:1081B0004A7B0192B1F91060B1F912B00C6A896979
:1081C00005915049C968421AC2F10308814277D823
:1081D0003DD101984FF00007002871D90120059981
:1081E00000FA07F20A4214BF4FF0010A4FF0000AEA
:1081F0000025690902A805F01F0250F8211001208E
:10820000904001421BD034F9020BBAF1000FA0EBF1
:108210000B000CBFA6EB000906EB00092A46394605
:108220000098FAF7DFF9B9F1000FC8BF40F4003049
:1082300040F400432A4639460098FAF726FA6D1CA6
:10824000262DD6D301987F1C8742C7D34FE0B8F1C3
:10825000000F51DB01984FF00009002847D908F1C1
:108260000D00012101FA00FA401E01FA00F006900B
:108270000121059801FA09F2104018BF01200025DC
:108280000790690902A805F01F0250F8211001208B
:108290009040014223D034F9020B0799A0EB0B0068
:1082A00000290CBF371A37182A4649460098FAF7B2
:1082B00099F9034610F4003F03D0002F05DA02E0DD
:1082C00015E0002F01DD23EA0A03B8F1000FC4BF57
:1082D000069803432A4649460098FAF7D6F96D1CDA
:1082E000262DCED3019809F101098145C0D3B8F1FB
:1082F000000F04BF01200490049809B0BDE8F08F7E
:10830000001F01005C8500102DE9F14FADF54E7D99
:108310000020C090BF9072B6FAF7FAFC0746FCF74F
:1083200001FC48B1FCF7A6FCC090FCF78DFCFCF703
:10833000A6FCBF90FCF793FCFAF7CBFBFAF7D0FA58
:10834000C590FAF70DFDC490FAF7CCFAFAF792FD52
:10835000BC900020FAF785FD0120F9F748FCC89091
:108360001120F9F744FCC9900220F9F740FCCA90AB
:108370001220F9F73CFCCB90FCF71DFAC390FCF7F8
:1083800002FA4FF49350FCF770F962B60020F9F747
:10839000FFFBC29001210020F9F7EDFB0020F9F767
:1083A0000CFC0021C1900846F9F7FAFB0120F9F70F
:1083B00082FCCC900020FAF7DEFAC7900020FAF792
:1083C000CDFAC690F9F723F8CD900020F9F724F8FC
:1083D000002006469EAD45F82060401C0C28FAD3CC
:1083E00017F0070F4FF001040AD040F68C61FE48E9
:1083F0009E9417F0F8F840F68C61FC4817F0F3F8FB
:1084000017F0F00F47D00120F8F7F7FA38B19821AC
:10841000F74817F0E8F89821F64817F0E4F811202B
:10842000F8F7EBFA38B19821F34817F0DCF8982107
:10843000F24817F0D8F80220F8F7DFFA38B198219F
:10844000EF4817F0D0F89821EE4817F0CCF812203A
:10845000F8F7D3FA38B19821EB4817F0C4F898210F
:10846000EA4817F0C0F80120F8F7C7FA002818BF4B
:10847000A0941120F8F7C1FA002818BFA194022097
:10848000F8F7BBFA002818BFA2941220F8F7B5FA43
:10849000002818BFA3944FF0405ADFF874B3DFF8F8
:1084A00074939E984FF0FF0858B330468DF80060E3
:1084B00001A9F9F701FA9DF80000F9F71DFA8DF806
:1084C0000C009DF80000F8F767FA8DF80D009DF894
:1084D0000000F9F7D6FB00280CBF4FF0FF31002158
:1084E00006918DF80E80B9F80200ADF81000ADF8D5
:1084F00012609DF80000F9F77FF9ADF81400CDE99E
:1085000008AB9F986F4640B38DF8286007F12C01A7
:108510003046F9F7D1F99DF82800F9F7EDF98DF813
:1085200034008DF8354010968DF83680B9F8020089
:10853000ADF83800ADF83A609DF82800F9F75CF91D
:10854000ADF83C009DF80C009DF80D1048430AEB77
:1085500040010BEB4000CDE91210A0984FF4806A67
:1085600002264FF0AA3BE0B38DF8504007F15401CA
:108570002046F9F7A1F99DF85000F9F7BDF98DF8FB
:108580005C009DF85000F9F73AFA04FA00F08DF813
:108590005D009DF85000F9F72AFB1A908DF85E8077
:1085A000B9F80400ADF86000ADF862A09DF8500085
:1085B000F9F722F9ADF8640097481C9097481D9090
:1085C0009DF85D00022809D99DF85C10801E484383
:1085D0001C9901EB40001C908DF85D601A9800B169
:1085E00000E007E09DF850004FF0AA31F9F7EDFAEE
:1085F000CDF868B0A198E0B3112007F17C018DF8A7
:108600007800F9F759F99DF87800F9F775F98DF8C0
:1086100084009DF87800F9F7F2F904FA00F08DF87B
:1086200085009DF87800F9F7E2FA24908DF88680AD
:10863000B9F80400ADF88800ADF88AA09DF878007C
:10864000F9F7DAF8ADF88C00754826907548279050
:108650009DF88500022809D99DF88410801E4843A2
:10866000269901EB400026908DF88560249800B192
:1086700000E007E09DF878004FF0AA31F9F7A5FA7D
:10868000CDF890B0A298E0B307F1A40130468DF880
:10869000A060F9F711F99DF8A000F9F72DF98DF810
:1086A000AC009DF8A000F9F7AAF904FA00F08DF8E3
:1086B000AD009DF8A000F9F79AFA2E908DF8AE80E3
:1086C000B9F80400ADF8B000ADF8B2A09DF8A00074
:1086D000F9F792F8ADF8B400534830905348319010
:1086E0009DF8AD00022809D99DF8AC10801E4843C2
:1086F000309901EB400030908DF8AD602E9800B1BC
:1087000000E007E09DF8A0004FF0AA31F9F75DFA0C
:10871000CDF8B8B0A398E0B3122007F1CC018DF8E2
:10872000C800F9F7C9F89DF8C800F9F7E5F88DF821
:10873000D4009DF8C800F9F762F904FA00F08DF84A
:10874000D5009DF8C800F9F752FA38908DF8D68018
:10875000B9F80400ADF8D800ADF8DAA09DF8C8006B
:10876000F9F74AF8ADF8DC0031483A9031483B90CF
:108770009DF8D500022809D99DF8D410801E4843E1
:108780003A9901EB40003A908DF8D560389800B1E5
:1087900000E007E09DF8C8004FF0AA31F9F715FA9C
:1087A000CDF8E0B0F8F782FB10F0010F0BD0FEF728
:1087B00070FF3C2807D1FCF7C7FB20B10420FCF771
:1087C00072FBFCF749FCFAF70AFB4FF00008C346BE
:1087D000C2464646C14604F083F801287DD0BBF16D
:1087E000800F7AD8AAA827E00000013000400130AD
:1087F0008C0E01308C4E0130240F0130244F01309B
:10880000BC0F0130BC4F01305410013054500130C6
:10881000004000305C850010CC090030CC490030AD
:10882000CC0E0030CC4E00304C1800304C5800308C
:108830004C1D00304C5D0030FAF79BFD00286ED0D7
:10884000AAA804F075FDBC98002818BF00273BD0EB
:108850009EA850F82700A0B307EB8701684600EBFD
:10886000C104207810F00F0F2BD0F9F7C0F910F0E9
:10887000010F26D0216A257B01F0030000EB850261
:10888000D21C22F0030221F00301CDE9BD1278A928
:108890000C1878A8BD9916F0B0FE0020002D0BD959
:1088A000411934F8102034F8113024F81030401CED
:1088B00024F811208542F3D878A9BE9ABD9816F005
:1088C0009CFE7F1C0C2FC3D31AF1010A7DD04FF000
:1088D000000A5046B0AD012700E077E00BF1010B34
:1088E00045F82070401C0C28FAD3052E6ED2DFE824
:1088F00006F003172A3D500000249EA850F82400DB
:1089000048B104EB8401684600EBC1014846FFF71B
:1089100044FC45F82400641C0C2CEED33BE068E0DA
:1089200000249EA850F8240048B104EB8401684656
:1089300000EBC1014846FFF784FB45F82400641CA6
:108940000C2CEED327E000249EA850F8240048B158
:1089500004EB8401684600EBC1014846FFF752FA78
:1089600045F82400641C0C2CEED314E000249EA8CF
:1089700050F8240048B104EB8401684600EBC101C3
:108980004846FFF72DF945F82400641C0C2CEED363
:1089900001E04FF001080121002055F82020CAB164
:1089A000401C0C28F9D3A9B11F2E0DD2761CCE98ED
:1089B00007FA06F1014207D1761C042E04D8CE989E
:1089C00007FA06F10142F7D001E005E017E04FF0A9
:1089D000000901E009F10109FAF71CFDB8F1000FE7
:1089E0000DD1BC98002818BFF9F713F9FAF7F7F979
:1089F000F1E6FEF752FDB8F1000F3FF4ECAEFAF7E6
:108A000009FDF9F76FFF0520FCF74DFA0120C89921
:108A1000F9F7DBF81120C999F9F7D7F80220CA99BC
:108A2000F9F7D3F81220CB99F9F7CFF8BC98FAF7F9
:108A300018FA0020C199F9F7B3F80020C299F9F7A4
:108A40009AF8CC98F9F737F9C798F9F794FFC698D0
:108A5000F9F784FFCD98F8F7DFFCC59830B1C498DA
:108A600010B1FAF7BCF901E0FAF780F9FCF75AF80F
:108A700048B1C098002818BFFCF75AF8BF980028E2
:108A800018BFFCF78EF8C398002818BFFBF724FE28
:108A9000B8F1000F0CBF012000200DF54F7DBDE89F
:108AA000F08F70B5FB4D1646D5F844231205120D14
:108AB0001DD000281CBFC1F30800FBF72DF8D5F826
:108AC000480340F00100C5F84803D5F8480320F0FA
:108AD0000100C5F848030022341E23DDD5F84813F1
:108AE00040F21F2011F0010F08D1401E01D20020DA
:108AF00070BDD5F8481311F0010FF6D0D5F8440336
:108B0000C0F30B000244D5F8480340F00100C5F85B
:108B10004803D5F8480320F00100C5F84803641E57
:108B2000002CDBDC1001B0FBF6F080B270BD2DE94B
:108B3000F84F040016D0D848006CC0F30829FAF7A3
:108B4000FDFF49EA004200239621072008F0F0FCCF
:108B5000D048D0F8401341F48031C0F8401332209F
:108B600000900AE0FAF7E5FF0120BDE8F88F00BFAA
:108B700000BF00BF00BF00BF0846411E0091F6D2F3
:108B80004FF0000840F2FF17C246464608EB0700C8
:108B900000EBD0704510A9B264220120FFF781FFDD
:108BA000F0B1A04288BF6F1E38BF05F101081ED189
:108BB000AA461FFA8AF14FF064024FF00100FFF756
:108BC00070FF0446002352469721072008F0B0FCAE
:108BD000A4F58050AF38A0289CBF0120BDE8F88FD5
:108BE000B9F1000F10D04846FAF796FF0EE0011BCE
:108BF00048BF211A321B48BFA21B9142BCBFAA46E4
:108C00000646B845C2DDD4E7FAF793FF49F480324F
:108C100000239721072008F08BFC0020BDE8F88F87
:108C20002DE9F04F9D4CADF50F7D01272678FEF71D
:108C3000C3FB012840F0878104F061FD984800687B
:108C4000B0F91E10B0F91C0016F02CFD16F0020F42
:108C500000F0708180ADFEF7D3FE4FF00008A8B1A0
:108C6000B0E80E1080AC84E80E10B0E80E1084ACB2
:108C700084E80E10B0E80E1088AC84E80E1070E89E
:108C80000C12806B8C91CDE98D2022E0FF223C21DB
:108C9000284616F0C6FC834880904FF49870819067
:108CA0003C20CDE982085020CDE984084FF0FF3008
:108CB0008B908A90CDF818828990CDE98780ADF8A5
:108CC00038828DF83A82CDF83082CDF834828DF832
:108CD0003B827548FBF760F88598401C8590F9F752
:108CE000F8FE41F2FF00FFF722FF6C498860F9F7B8
:108CF000B8FF40F233390025CDF8008075E02846F2
:108D000005F063FC00286FD0008900EA090434F004
:108D1000CC0069D040F20F312846FEF7E7FC00286E
:108D200062D0F9F7F5FF009900295BD1F9F7A7FEAA
:108D300024F0EE0030F47E4015D01F20FFF7E4FA57
:108D40000090F9F7CFFD009800284BD16FB114F0D7
:108D5000010F1CBF0720FEF7A3FE14F0100F1CBF6D
:108D6000F020FEF79DFE0098E0BB14F0220F06D025
:108D7000FCF728FF0090F9F7B5FD009890BB8FB382
:108D800014F0020F16D0FCF70DFB8346474801781C
:108D90004748007848434FEA400AFEF777FC4FF017
:108DA000060C5FEA0B0205D090F926105346604688
:108DB00005F051FC14F0200F14D0FCF78AFA044699
:108DC0003C4801783C48007808444FEA400AFEF7E6
:108DD0005DFC01460820220004D091F9281053467A
:108DE00005F039FCFEF7F7FD6D1C05F0EAFBA84223
:108DF000009802D9002882D003E0002808BF012093
:108E000000D0002018B1FCF7BDFF01281FD08798C3
:108E10000023401C8790502084901A46212107206F
:108E200008F086FB00231A461946FE20CDF8008084
:108E3000FDF79EF880AC05F09CFB50B381698891EA
:108E4000C169899141698A91C0688B903CE016F0B4
:108E5000080F14BFA220A12010498490886858B13F
:108E60000D48006CC0F30820ADF838029DF83A02B6
:108E7000401C8DF83A0206E0ADF838829DF83B02BE
:108E8000401C8DF83B02C1F808808698401C8690F3
:108E9000D0E713E000500040006000405C85001007
:108EA0000C8700105443524600EE03004485001026
:108EB0004585001046850010478500104FF0FF30B3
:108EC0008B908A9089908890A04880904FF49870F9
:108ED00081903C20CDE982080021A3682246084603
:108EE00052F820C0401C6144B0EB930FF8D34D42C0
:108EF000FF224FF400716846E56016F092FBA2680D
:108F0000F4E804018DE827000FCC04AD85E80F00DC
:108F10000FCC08AD85E80F00D4E90001A2688C4CA5
:108F2000CDE90C010E922046FAF736FF694620463D
:108F3000FAF7D4FF0020FCF75FFD00233246402102
:108F4000072008F0F5FA0DF50F7DBDE8F04F03F0AE
:108F5000F3B9804A022804BF91807047042808BFF3
:108F6000518070470146002002297A4A04BFB2F9B5
:108F700004007047042908BFB2F90200704770B5B9
:108F80000126FEF73DFD20B10069A12818BFA228E7
:108F900001D0002070BD002405F013FB002834D957
:108FA000204605F012FB00281EBF058925F0CC00E5
:108FB00030F47C4024D040F20F312046FEF796FB7F
:108FC000F0B115F0010F0AD0FAF73EFA38B944F4BF
:108FD000807200232021072008F0AAFA002615F04D
:108FE000100F0BD00120FAF786FA38B944F48052FA
:108FF00000232021072008F09BFA0026FEF7EBFC57
:10900000641C05F0DEFAA042CAD8304670BD0020CC
:109010007047002070474F48407870474D49002006
:109020004870704770B5002105220846FFF739FDEA
:109030000023484A00282BD05178002908BF13612B
:10904000A0F5805CACF1F80CBCF10E0F20D9491CE6
:10905000C9B25170D2F810C00A296044106121D9F8
:109060003D495370096CC1F308249CB14BF6F521BE
:10907000884294BF651C651E2846FAF74DFD44EAF8
:10908000054200239521072008F052FA012070BD07
:10909000537007E041F2FF00FFF749FD00281CBFB5
:1090A000012070BD002070BD10B5FEF7A9FC38B3DB
:1090B000264A0168914223D14168B1F5987F1FD8B3
:1090C000D0F808C00146BCF5007F19D800220B4635
:1090D0001146B2EB9C0F07D253F82140491C2244A1
:1090E000B1EB9C0FF8D35AB9188F00281CBFA0F51C
:1090F0007F41B1F1FF0103D0FAF70EFD012010BD51
:10910000002010BD10B5FEF77BFCD8B10F4A0168F6
:10911000914217D14168B1F5987F13D8D0F808C0B3
:109120000146BCF5007F0DD800220B461146B2EB7C
:109130009C0F09D253F82140491C2244B1EB9C0FEB
:10914000F8D30AB1002010BD188F10BD5443524609
:1091500000EE03005C8500100060004070470020B6
:10916000704710B503F00700042808BFFEF7F3F9B5
:10917000002010BD10B403F007020024FE4BDFF8FE
:10918000FCC3012A02D0022A17D013E005208CF874
:109190000000FB48CCF80C4000681A68532111709D
:1091A0001A68452151701A68010A91701968C870CF
:1091B0001868047110BC002070479CF80020052A34
:1091C00014D1DCF80C20052A28BF104605D21B68F4
:1091D0009B5C0370501CCCF80C00052806D10120C4
:1091E000CCF80C40087003208CF8000010BC012063
:1091F000704770B503F007020125DF4CDF4B4FF0DD
:10920000000C012A02D0022A25D022E00520187085
:10921000DB48C3F80CC000682268AC2111702268DA
:10922000010A5170216888702068C570206880F834
:1092300004C005F03FF948B1D24D286805F043FA63
:1092400020B128682168007E487102E02168FF2073
:109250004871002070BD1A78052A10D1DA68062AF4
:1092600028BF104604D22468A45C0470501CD86047
:10927000062804D1C3F80CC00D700320187001201B
:1092800070BD03F00702022A1CBF00207047202295
:1092900002700120087070472DE9F041B74F0D466C
:1092A000064613F0070F04D003F00700022808D089
:1092B00004E012F0040F1CBF0020B8700020BDE8CD
:1092C000F08103F033F8002814BF0124002403F0D8
:1092D00030F8002814BF0222002242EA0403B878C2
:1092E000002814BF0422002242EA0300307001204B
:1092F0002870BDE8F08170B503F0070C00269F4C84
:109300009D4DBCF1010F0AD0204613F0070F0078E5
:109310000DD0BCF1040F08BF062818D029E0E66084
:1093200028680670286846700520207021E005280E
:109330001FD1E068022803D22B681A54401CE06059
:10934000022816D10120E6600870062010E0286887
:10935000007855280BD128684078AC2818BFBC2865
:1093600005D128680122411C062002F0C5FF032018
:109370002070002070BD70B503F0070200257E4C00
:109380007E4B012A02D0022A24D021E00520187049
:10939000DD6002F07FFF41F6E8710144B0F5783FEF
:1093A00010D8CA78086862F31F60774A904208BFF5
:1093B000002007D10A18236812791A54401C142877
:1093C000F8D305E0002021680D54401C1428FAD37E
:1093D000002070BD1A78052A13D1DA68142A28BF34
:1093E000104607D2D4F800C01CF802C080F800C0B4
:1093F000501CD860142804D10120DD6008700320BF
:109400001870012070BD70B503F0070200255A4C9A
:109410005A4B012A02D0022A3FD03CE005201870A6
:10942000DD6002F037FF41F6E8710144B0F5783FA6
:109430002BD8CA78086862F31F60534A904224D13F
:109440002268087C10702268487C50702268887CF2
:1094500090702068CA7CC27020680A7A0271226803
:10946000487A50712268887A90712268C87AD071DF
:109470002268087D10722268487D50722268887DBB
:109480009072C87D2168C87205E0002021680D54E3
:10949000401C0C28FAD3002070BD1A78052A13D17D
:1094A000DA680C2A28BF104607D2D4F800C01CF88E
:1094B00002C080F800C0501CD8600C2804D10120E4
:1094C000DD60087003201870012070BD70B503F0D6
:1094D00007020025284C294E012A02D0022A36D044
:1094E00033E005F046F840B3D0E906212368C068B0
:1094F0001A70D4F800C0130A8CF80130D4F800C0F8
:10950000130C120E8CF802302368DA702268117185
:1095100023680A0A5A7123680A0C090E9A71226894
:10952000D171216808722268010A51722268010C07
:109530009172010E2068C17204E021680D54401C34
:109540000C28FAD305203070F560002070BD327809
:10955000052A10D1F2680C2A28BF104604D22368CD
:109560009B5C0370501CF0600C2804D10120F56056
:1095700008700320307009E0E44C02007885001088
:10958000044C00400C87001034CD12AB012070BD9C
:1095900070B503F007020024F94DFA4B012A02D0FE
:1095A000022A3ED03BE0052018700026DC6002F065
:1095B00071FE00F50051B0F5783F98BF11F0030F30
:1095C00027D1F14A0868904204BF0022104620D1FA
:1095D00051F82030401C1A440728F9D302B1C6B113
:1095E00028680A7C02702A68487C50702A68887C47
:1095F00090702A68C87CD0702A68087D10712A682B
:10960000487D50712A68887D9071C87D2968C8712D
:1096100005E0002029680C54401C0828FAD30020DB
:1096200070BD1A78052A13D1DA68082A28BF1046B7
:1096300007D2D5F800C01CF802C080F800C0501C4A
:10964000D860082804D10120DC600870032018705D
:10965000012070BD2DE9F04103F0070C0027C94E31
:109660004FF00508BCF1010F0DD013F0070F0FD01C
:109670003246BCF1020F127810D0BCF1040F08BFC3
:10968000062A26D058E086F800807770F76053E00D
:109690007270BE48F062062030704DE0052A15D188
:1096A000F268042A28BF104609D2C2F10303D6F893
:1096B0002CC0DB002CFA03F30370501CF06004286C
:1096C00004D10120F7600870032030700120BDE84C
:1096D000F08170780125002410F0010F11D002F004
:1096E000D9FDB0F5783F23D86A030021B1EB900F84
:1096F00007D252F8043B491C1C44B1EB900FF8D33D
:10970000B5B1707810F0020F0ED004F032FF78B1CE
:1097100082680021B1EB920F06D250F8043B491C3D
:109720001C44B1EB920FF8D3002D18BFF46200D1A6
:10973000F762777086F800800020BDE8F081F0B510
:1097400003F0070C00268E4D8E4C83B0BCF1010F48
:109750000ED013F0070F1DD0224603271278BCF15C
:10976000020F26D0BCF1040F08BF062A36D03CE019
:1097700002AA01A9684603F0BEF9052020702968F5
:1097800001980870296800984870296802988870C4
:10979000E6602AE0E068032803D229680A54401CE6
:1097A000E060022821D306212170032808BFE6606B
:1097B0001BE0052A0FD1E268032A28BF104604D215
:1097C0002B689B5C0370501CE060032803D10120D0
:1097D000E6600870277003B00120F0BD2868827829
:1097E0000178407803F07AF9277003B00020F0BDCB
:1097F00008B503F0070001280AD104F05BFE38B178
:1098000001208DF80000024669460D2002F074FD2B
:10981000002008BD08B503F0070001280AD104F0B4
:1098200049FE38B100208DF80000012269460D2064
:1098300002F062FD002008BD08B503F00700012812
:1098400009D104F037FE30B103208DF80000012269
:10985000694602F051FD002008BD0020704708B5A0
:1098600003F0070001280AD104F024FE38B10B20D0
:109870008DF8000001226946032002F03DFD002022
:1098800008BD1FB513F0070F0ED104F013FE58B139
:109890009DF80800F0280AD004F00CFE20B1012247
:1098A00002A9092002F028FD04B0002010BDFEF737
:1098B000CDF8F9E70020704770B503F00700304C91
:1098C000304D012808D013F0070F12D0042804BF30
:1098D0002878062816D01FE00020E860216808706C
:1098E00021684870216888702168C8700520287038
:1098F00012E0E86804280FD221680A54401CE8608E
:10990000062008E004F0D6FD30B10422104621689C
:1099100002F0F2FC03202870002070BD10B503F0A7
:109920000700012804D103F0EAFE1649002008715F
:10993000002010BD10B503F0070C124CBCF1010F54
:1099400006D013F0070F09D0BCF1020F20D015E0AC
:109950000020E06007F0E3FDE0610FE0E068002830
:1099600004BF1002E06106D0012804D1E069104371
:10997000E06107F0D3FDE068401CE060002010BD0E
:10998000E44C02007885001054464953EFBEADDE2A
:10999000E26812B1012A04D007E0A18B090A017024
:1099A00003E0237F037001200870501CE060012059
:1099B000E5E710B503F0070CFE4CBCF1010F06D033
:1099C00013F0070F09D0BCF1020F18D015E00020EA
:1099D000E06007F0A7FDE0610FE0E068002804BF49
:1099E0001002E06106D0012804D1E0691043E06173
:1099F00007F09BFDE068401CE060002010BDE268BD
:109A000012B1012A04D007E0A18B090A017003E01A
:109A1000237F037001200870501CE060012010BDFE
:109A200070B503F0070CE34D0E460446BCF1010F80
:109A300006D013F0070F07D0BCF1020F18D015E0C5
:109A40000020E860286111E0E868002804BF1002E7
:109A5000E86108D0012806D1E869104381B2E861C5
:109A6000E88810F0DFFAE868401CE860002070BD6C
:109A7000286902280ED2E88810F0D8FA2B6982B241
:109A8000002B04BF100A207004D0012B02D12270D9
:109A9000012030702869401C2861012070BD10B47D
:109AA00003F0070CC34CBCF1010F08BF00200BD022
:109AB00013F0070F03D0BCF1020F09D005E0E068F6
:109AC000002808BFE280401CE06010BC0020704706
:109AD000E2681AB9A379037001200870501CE06095
:109AE00010BC012070472DE9F047064603F007003F
:109AF000B04F8946012808BF002037D0DFF8B88270
:109B0000AE4D13F0070F02D0022833D02FE0F868D3
:109B1000002808BF7A7027D0012804BF1002F8611E
:109B200022D0022820D1F8691043F8617E7884B2EF
:109B300004F0C0FCC0B1062E16D2DFE806F0030622
:109B4000090C1013A8F80E400EE0A8F80C400BE02A
:109B50002868848308E02868A0F8144104E0286895
:109B6000048601E028684486F868401CF8600020FC
:109B7000BDE8F087386902282AD297F801A00024AE
:109B800004F098FCC8B1BAF1060F16D2DFE80AF06B
:109B90000306090C1013B8F80E400EE0B8F80C409C
:109BA0000BE02868848B08E02868B0F8144104E0D2
:109BB0002868048E01E02868448E3869002804BFB4
:109BC000200A307004D0012802D1347089F80000D6
:109BD0003869401C38610120BDE8F0872DE9F0416B
:109BE0001C4615460E46074604F064FC88B17248D0
:109BF00014F0070F04D004F0070102290CD008E08C
:109C0000002D1ABF90F8EC00C0084FF0FF300CF0A8
:109C1000FBF80020BDE8F08190F8EC00C008387037
:109C200001203070BDE8F0812DE9F0411C46154659
:109C30000F46064613F0070F08D104F03BFC28B18D
:109C4000022D3CBF284609F07EFD03E004F007002A
:109C5000022802D00020BDE8F08109F06DFD3070CF
:109C600001203870BDE8F08170B503F007020026CE
:109C7000534C504D012A02D0022A15D012E008F0B0
:109C8000F1FD21680870FDF797FB2168487004F02A
:109C900077F921688870FDF795FB2168C870052069
:109CA0002870EE60002070BD2A78052A10D1EA687D
:109CB000042A28BF104604D223689B5C0370501C02
:109CC000E860042804D10120EE60087003202870A9
:109CD000012070BD70B503F00702394C0025354EE8
:109CE000012A02D0022A54D051E0FDF789FE002853
:109CF00036D04169FF292CBFFF21C9B222681170FB
:109D00008169FF2934BFC9B2FF2122685170C1693E
:109D1000FF2934BFC9B2FF21226891702268017CFB
:109D2000D170226890F820101171018C2268090A04
:109D30005171016A2268090C9171016A2268090E49
:109D4000D171016BFF2934BFC9B2FF2122681172A2
:109D5000406BFF2834BFC0B2FF202168487215E075
:109D60002068057020684570206885702168502043
:109D7000C8702168FF2008712168487121688871C6
:109D80002168C8712068057220684572F56000205E
:109D900070BDF2680A2A28BF104604D223689B5C73
:109DA0000370501CF0600A2802D10120F560087091
:109DB000012070BD78850010A83001100C870010BC
:109DC000E44C020003F00702FB4B4FF0000C012AA9
:109DD00008BFC3F80CC001D0022A01D00020704790
:109DE000DA68022A3DBF80F800C0501CD8601046D7
:109DF000022803D10120C3F80CC00870012070476D
:109E00002DE9F047064603F00700EB4F8A464FF076
:109E10000008012808BFC7F80C8001D0022802D032
:109E20000020BDE8F087F868A0BB0024254602F0BA
:109E300031FA014600F5005018384FF400524FF047
:109E40004009B1F5783F20D890F803C003686CF35F
:109E50001F63DFF868C3634517D1091FB4EB910F87
:109E600006D252F8043B641C5D40B4EB910FF8D36A
:109E7000C17D406961F31F60A84206D104F01AFB5E
:109E8000012804BF8020307001D086F80090F86867
:109E9000401CF860012803D1C7F80C808AF8000044
:109EA0000120BDE8F0872DE9F04103F0070200260C
:109EB000C34CC14D012A02D0022A56D052E0C148FB
:109EC00000680520287004F0F5FA002849D0BE4F3C
:109ED000386804F0F8FB002843D010F086F880467C
:109EE00010F087F839680A7E12F0040F11D0C98A81
:109EF0002268090A117039682268897D51703968B1
:109F00002268898A090A917039682268097DD170AE
:109F100010E0898A2268090A117039682268097D6F
:109F2000517039682268C98A090A917039682268B3
:109F3000897DD17022684FEA18211171216881F85A
:109F400005802268010A91712168C8713868226809
:109F5000817C11722268017C5172008B2168000A99
:109F60008872EE600020BDE8F0812A78052A10D1C1
:109F7000EA680B2A28BF104604D223689B5C037052
:109F8000501CE8600B2804D10120EE60087003200B
:109F900028700120BDE8F0812DE9F04703F00702A9
:109FA0000025874C844B012A02D0022A5CD058E05D
:109FB000052018700026DD6002F06CF900F50053F2
:109FC000B0F5783F98BF13F0030F44D17F4A19686A
:109FD000914204BF0022114608D153F821C0491C08
:109FE00062440729F9D3002A08BF01269F7C93F811
:109FF00013807EB3002241F6E8710144B0F5783F4A
:10A0000007D8CB78086863F31F606C4B984208BF91
:10A0100001228E7C91F81390002A08BF002013D0F3
:10A0200004F0A7FA216880690E70216881F8019018
:10A030002268010C000E91702168C87020680771B9
:10A04000206880F805800CE021680D54401C06282B
:10A05000FAD306E0FFE7002021680D54401C0628D3
:10A06000FAD30020BDE8F0871A78052A13D1DA6800
:10A07000072A28BF104607D2D4F800C01CF802C037
:10A0800080F800C0501CD860072804D10120DD6092
:10A090000870032018700120BDE8F08770B50546F0
:10A0A00003F007000C46022829D104F003FA30B36C
:10A0B000454800220068037EC3F380008000C3F39C
:10A0C000400100EB410003F001010844082812D2CE
:10A0D000DFE800F00406080A0C0E111004220AE062
:10A0E000052208E0062206E0072204E0022202E040
:10A0F000032200E001222A700120207070BD0020A0
:10A1000070BD10B503F0070C2B4CBCF1010F06D04D
:10A1100013F0070F0AD0BCF1020F1AD017E000208D
:10A12000E06020610FF0E1FFE06110E0E0680028EE
:10A1300004BF1002E06107D0012805D1E069104397
:10A14000E06180B20FF0CEFFE068401CE0600020CC
:10A1500010BD2269022A0BD212B1012A04D007E0F5
:10A16000A18B090A017003E0237F037001200870AE
:10A17000501C2061012010BD70B503F007010026BE
:10A180000D4D0446012908BF2E6301D0022901D0DC
:10A19000002070BD286B002804BF0D4815F087FA19
:10A1A000296B102928BF267002D20948405C207014
:10A1B000481C2863012070BD7885001034CD12AB97
:10A1C000E44C0200044C00400C87001054464953F4
:10A1D00014A900102DE9F04103F007010026FB4D02
:10A1E0000746012908BF2E6301D0022902D00020B2
:10A1F000BDE8F08195F8300000F00F042879204385
:10A2000004D1F34815F053FA01202871052C28BF1A
:10A210002E71EF48005D3870286B401C28630120C8
:10A22000BDE8F08170B5044603F007000D46022832
:10A230001CBF002070BD15F03FFA2070012028706F
:10A2400070BD2DE9F04103F007020026E14DDF4C1F
:10A25000012A02D0022A1AD016E00520207000221E
:10A2600011461046E66002F046FC4FF6FF7101EA27
:10A2700040006061FDF7A0F8032803BF287820287C
:10A28000D54802F04BFCA0620020BDE8F0812278A6
:10A29000052A1DD1D4F814C0E268624528BF1046D3
:10A2A00007D212F0010F1CBF6378037013D0501C4B
:10A2B000E06060450CD10120E6600870032020704A
:10A2C000FDF77AF8032806BF2878202802F033FC2F
:10A2D0000120BDE8F081A76A22F00103FB5A1F0AA2
:10A2E00007706370E3E770B503F007020025B74C11
:10A2F000012A02D0022A11D00EE0B84805220068D7
:10A30000B0F91210B0F91000227008444000E56066
:10A31000606102F097FEA062002070BD2278052ADD
:10A3200017D1D4F814C0E268624528BF104607D29E
:10A3300012F0010F1CBF637803700CD0501CE0605A
:10A34000604506D10120E56008700320207002F00E
:10A3500087FE012070BDA66A22F00103F35A1E0A8F
:10A3600006706370EAE70020704770B50D4604463A
:10A3700013F0070F04D003F00700022805D002E015
:10A380001046FDF70DF8002070BDFDF70CF82070A9
:10A390000120287070BD70B503F0070203258B4CB7
:10A3A000012A02D0022A17D014E004F0B4F90646BC
:10A3B000FCF7F9FF0146304604F029FC2062002832
:10A3C0001ABF052020702570304604F004FC60623E
:10A3D0000020E060002070BD2278052A0BD1236A9E
:10A3E000E2689B5C0370501CE060626A904202D39A
:10A3F000012008702570012070BD002070470020EA
:10A4000070477FB51C460E46054613F0070F08D16E
:10A4100004F050F828B1012202A9252001F06CFFB8
:10A4200003E004F00700022802D004B0002070BD51
:10A4300002F03FFC28700120307004B070BD2DE99F
:10A44000F04103F007020027604E88460546012AC6
:10A4500002D0022A0BD007E0052030700A20F760F6
:10A46000706102F05BFBB0620020BDE8F0813078E3
:10A47000052819D1F2687069824228BF104608D2B7
:10A4800012F0010F1CBF7078287010D0F068401CCB
:10A49000F0607169884207D10120F76088F80000F8
:10A4A0000320307002F047FB0120BDE8F08100245A
:10A4B00002F0FFFB012804D1F068B16A20F001002E
:10A4C0000C5A200A28707470E0E770B50D460446F7
:10A4D00013F0070F04D003F00700022805D002E0B4
:10A4E000104604F015F9002070BD04F014F9207036
:10A4F0000120287070BD7FB51C460E46054613F03E
:10A50000070F08D103F0D6FF28B1012202A91F20AE
:10A5100001F0F2FE03E004F00700022802D004B0CC
:10A52000002070BD08F0E2FA28700120307004B0FD
:10A5300070BD7FB51C460E46054613F0070F08D1C7
:10A5400003F0B8FF28B1012202A9202001F0D4FEB7
:10A5500003E004F00700022802D004B0002070BD20
:10A5600008F0CAFA28700120307004B070BD7FB5C1
:10A570001C460E46054613F0070F08D103F09AFF5C
:10A5800028B1012202A91B2001F0B6FE03E004F06D
:10A590000700022802D004B0002070BDFDF72CF89F
:10A5A00028700120307004B070BD7FB51C460E4687
:10A5B000054613F0070F13D103F07CFF80B1012291
:10A5C00002A90C2001F098FE0EE000007885001032
:10A5D00014A90010C1850010C82801100C870010B4
:10A5E00004F00700022802D004B0002070BD08F07B
:10A5F00039F928700120307004B070BD7FB51C4659
:10A600000E46054613F0070F08D103F053FF28B19B
:10A61000012202A90F2001F06FFE03E004F0070001
:10A62000022802D004B0002070BD0FF016F900F02F
:10A630000F0040F0100028700120307004B070BD91
:10A640002DE9F04103F0070CFB4D0E460746BCF127
:10A65000010F07D0F94C13F0070F07D0BCF1020F20
:10A660001BD017E00020E860286113E0E8680428A8
:10A670003CBF21680A54032809D12068216800687A
:10A68000C97800BA20F0FF000843FBF7DEFEE86857
:10A69000401CE8600020BDE8F081286970B9FBF734
:10A6A000D9FE216820F07E42100E08702168100C3F
:10A6B00048702168100A88702068C2702A69042ACC
:10A6C00006D22068032A805C387004BF01203070F5
:10A6D000501C28610120BDE8F0817FB51C460D4665
:10A6E000064613F0070F08D103F0E4FE28B101225B
:10A6F00002A9102001F000FE03E004F00700022888
:10A7000002D004B0002070BD0FF0ABF800F00F04D1
:10A710000FF0A3F864F31F1030700120287004B00C
:10A7200070BD70B5C44D144613F0070F04D003F08C
:10A730000702022A06D003E01046F5F73CFE6C63E0
:10A74000002070BD95F8342002700120087070BDA3
:10A7500070B50D46044613F0070F04D003F0070050
:10A76000022805D002E01046FBF75AFE002070BD1B
:10A77000FBF759FE20700120287070BD2DE9F041D3
:10A7800003F0070CAD4DAC4C4FF00008BCF1010FCD
:10A790000DD013F0070F1AD02246A94E03271278C6
:10A7A000BCF1040F1DD0BCF1020F3DD02FE0C4F866
:10A7B0000C80286880F80080286880F8018028686C
:10A7C00080F80280286880F80380052007E0E068B0
:10A7D00004281CD229680A54401CE060062020701E
:10A7E00015E0062A13D103F065FE80B128680078D1
:10A7F00010B101280ED009E0286840780028706860
:10A8000014BF40F0800020F08000706027700020AE
:10A81000BDE8F081286840780028706814BF40F4D3
:10A82000007020F40070F0E7052A0FD17268736899
:10A83000C2F3C01203F4007342EA53122B681A7079
:10A8400002700120C4F80C80087027700120BDE858
:10A85000F08110B503F00702774C012A02D0022ADA
:10A860000DD00AE004F02EFA0021206200281ABF61
:10A870004FF4056060626162E160002010BD636AB0
:10A88000E2689A4228BF104607D2D4F820C01CF8CC
:10A8900002C080F800C0501CE060984204BF012054
:10A8A0000870012010BD10B4DFF898C113F0070F35
:10A8B00004D003F00702022A13D00FE0012A04BFDC
:10A8C000DCF8000040F0010006D0002A04BFDCF8EC
:10A8D000000020F0010001D1CCF8000010BC0020E5
:10A8E0007047DCF80030002213F0010F18BF01227E
:10A8F000534BD3F804C0544B1B68B3F8F030C3F388
:10A900000334012303FA04F41CEA040F18BF42F0D5
:10A91000020202700B7010BC0120704770B5144623
:10A920000E46054613F0070F04D003F00700022877
:10A930000ED00BE0002C14BF0120002002F0BEFE60
:10A9400024B13F48016821F440510160002070BDEE
:10A9500002F0BBFE002814BF012200222A70012051
:10A96000307070BD2DE9F04103F0070C324C0F46FA
:10A970008046BCF1010F12D0314E13F0070F4FF09B
:10A98000030510D02046BCF1020F027826D0BCF19E
:10A99000040F02BFE0680128062A33D036E0052004
:10A9A0002070002018E0E06810B1012804D011E008
:10A9B0006270062020700DE07168607800EA020382
:10A9C00019437160716820EA020291437160F9F7DE
:10A9D0004FFB2570E068401CE06017E0E06801284C
:10A9E00008BF062A03D16078F9F758FB2570706814
:10A9F00088F8000001203870E068401CE060012009
:10AA0000BDE8F0816078F9F749FB25700020BDE8CA
:10AA1000F08170B5044603F007000D4602281CBF04
:10AA2000002070BDFCF7C7FD002814BF01220022E2
:10AA300022700120287070BD78850010E44C02005F
:10AA400000100040144C00400C87001070B50D46FB
:10AA5000044613F0070F04D003F00700022805D0C6
:10AA600002E0104607F028FE002070BD07F027FE28
:10AA700020700120287070BD70B50D46044613F09B
:10AA8000070F04D003F00700022805D002E01046AB
:10AA9000F6F70FFA002070BDF6F70EFA20700120CD
:10AAA000287070BD70B503F00702DFF830C40C46A3
:10AAB0000546012A08BF05200DD013F0070F08BF77
:10AAC000062008D0022A09D0042A04BF9CF80000FE
:10AAD000062809D00EE08CF800000BE0FCF792FD90
:10AAE00028700120207070BD03208CF80000012028
:10AAF000FCF78BFD002070BD70B503F00702F74D29
:10AB00000E460446012A04BF0020E86001D0022A54
:10AB100001D0002070BD10F090F9EA68002A04BF4F
:10AB2000000A207004D0012A02D120700120307068
:10AB3000501CE860012070BD03F0070210B4E74B21
:10AB4000012A04BF0020D86001D0022A02D010BC24
:10AB500000207047DA68022A0CD24FF0010C002A5C
:10AB600008BF80F800C005D0012A03D1402404703A
:10AB700081F800C0501CD86010BC0120704770B52F
:10AB8000044603F007000D46022807D013F0070F14
:10AB900004BF1046FCF7FEFB002070BDFCF7FDFB78
:10ABA00020700120287070BD70B503F0070C0026DE
:10ABB000CB4DCA4C82B0BCF1010F06D013F0070F89
:10ABC0001FD0BCF1020F2DD029E068460DF0F7FB35
:10ABD000BDF80000296800090870BDF80200C0F344
:10ABE0000321BDF8000041EA001029684870296877
:10ABF000BDF80200887028689DF80410C170E660F6
:10AC00000DE0E06804283CBF29680A54401CE0605D
:10AC1000042804D104221320296801F06DFB02B03E
:10AC2000002070BDE268042A02D22B689B5C03708E
:10AC3000501CE060042804D10120E6600870032065
:10AC4000207002B0012070BD70B503F0070C002623
:10AC5000A34DA24CBCF1010F06D013F0070F0CD08E
:10AC6000BCF1020F19D016E00DF09CFB2A68010A16
:10AC7000117029684870E6600DE0E06802283CBF6A
:10AC800029680A54401CE060022804D102221420E2
:10AC9000296801F031FB002070BDE268022A02D26F
:10ACA0002B689B5C0370501CE060022804D10120DB
:10ACB000E660087003202070012070BD70B503F0BD
:10ACC000070C0026864D854CBCF1010F06D013F011
:10ACD000070F12D0BCF1020F1FD01CE00DF04AFB91
:10ACE0002A68010E11702A68010C51702A68010A45
:10ACF00091702968C870E6600DE0E06804283CBFE8
:10AD000029680A54401CE060042804D1042215205C
:10AD1000296801F0F1FA002070BDE268042A02D22D
:10AD20002B689B5C0370501CE060042804D1012058
:10AD3000E660087003202070012070BD2DE9F0410D
:10AD400003F0070C0027664D644EBCF1010F06D0DE
:10AD500013F0070F22D0BCF1020F44D040E00DF0F9
:10AD600059FB04460DF050FB80460DF05EFB01469A
:10AD7000286880F800802A6808095070C4F303220C
:10AD800042EA01112A68200C91702968CC70296868
:10AD900008712968200E4871F76021E0F0680028EA
:10ADA00004BF29680A7029680978012901D039B1DE
:10ADB0000CE0002818BF06283CBF29680A5405E0AB
:10ADC00028680771286847710520F060F068401C0A
:10ADD000F060062804D106221620296801F08CFABA
:10ADE0000020BDE8F081F268062A02D22B689B5C45
:10ADF0000370501CF060062804D10120F760087031
:10AE0000032030700120BDE8F08110B503F0070287
:10AE1000324C012A02D0022A27D024E003F052FF4C
:10AE20000023002804BF236263621BD000F150019D
:10AE300021624168B1F5887F90F820100CD390F81A
:10AE4000212001EB020C01FB02C190F8222090F8B6
:10AE500023001044084404E090F822000A1801FB83
:10AE600000206062E360002010BD636AE2689A42DD
:10AE700028BF104607D2D4F820C01CF802C080F8C2
:10AE800000C0501CE060984204BF012008700120FF
:10AE900010BD03F00702012A02D0022A05D002E009
:10AEA0000E490020C86000207047012202700A701D
:10AEB0001046704710B513F0070F04D003F00702D7
:10AEC000022A05D002E0104601F042FE002010BD2B
:10AED000044A127802700120087010BD78850010B5
:10AEE000E44C0200C185001010B513F0070F04D028
:10AEF00003F00702022A05D002E0104602F0BDF876
:10AF0000002010BDFB4A127802700120087010BDAD
:10AF10000020704703F00702F74B012A04BF00200E
:10AF2000D86001D0022A01D000207047DA684FF0C3
:10AF3000010C002A08BF80F800C0501CD86001280E
:10AF400008BF81F800C0012070471FB513F0070F3C
:10AF500007D103F0AFFA20B1012202A90B2001F0C2
:10AF6000CBF904B0002010BD70B503F00700E24C2F
:10AF70001546012804BF0020E06024D013F0070F1D
:10AF800021D103F097FAF0B1E068DC4E03283CBF12
:10AF900031680D54401CE060032814D1F7F799FD87
:10AFA0003068B0F8010045BAF7F79AFC040018BF02
:10AFB000F7F731FF306829460078F6F734FB002CAC
:10AFC00018BFF7F72BFF002070BD70B503F0070026
:10AFD000C94D1446012804BF0020E86020D013F0BA
:10AFE000070F1DD103F066FAD0B1E868C34E0228FE
:10AFF0003CBF31680C54401CE860022810D1F7F7C0
:10B0000068FDF7F76DFC040018BFF7F704FF306820
:10B0100041780078F6F7B3FB002C18BFF7F7FEFE77
:10B02000002070BD70B50D46044613F0070F04D024
:10B0300003F00700022805D002E01046F7F70BFFE7
:10B04000002070BDF7F70AFF20700120287070BD46
:10B050007FB51C460E46054613F0070F08D103F0D6
:10B0600029FA28B1012202A9172001F045F903E0CD
:10B0700004F00700022802D004B0002070BD07F0E1
:10B08000CCFB002814BF012200222A70012030705E
:10B0900004B070BD7FB51C460E46054613F0070F81
:10B0A00008D103F007FA28B1012202A9182001F003
:10B0B00023F903E004F00700022802D004B00020C6
:10B0C00070BD07F097FB28700120307004B070BD90
:10B0D0002DE9F04103F0070C874C0E460746BCF102
:10B0E000010F07D0854D13F0070F07D0BCF1020FF9
:10B0F00019D015E00020E060206111E0E06803282D
:10B100003CBF29680A54401CE060032808D1286825
:10B11000B0F8010040BA01B228680078FDF719FFC5
:10B120000020BDE8F0812269022A12D242B92868C3
:10B130000078FDF717FF2A68010A517029688870A6
:10B14000286822691044012A4078387004BF012021
:10B1500030702069401C20610120BDE8F08110B5ED
:10B1600003F007006449012808BF00200CD013F049
:10B17000070F624B02D0042808D018E0C8680428E2
:10B180003CBF1B681A54401CC86010E0C868042803
:10B190000DD31868196840788978000440EA0120C6
:10B1A0001968C978014318680078F8F7BCFA0020DC
:10B1B00010BD7FB51C460E46054613F0070F08D19B
:10B1C00003F078F928B1012202A9282001F094F8AF
:10B1D00003E004F00700022802D004B0002070BD94
:10B1E00002F044FD28700120307004B070BD10B52D
:10B1F00003F00702404C012A02D0022A07D004E0E3
:10B200000020E060F9F717FBE061002010BDE26864
:10B21000042A07D2C2F10303D4F81CC0DB002CFAC5
:10B2200003F30370501CE060042804BF0120087081
:10B23000012010BD10B503F00700012807D103F06D
:10B2400039F920B1002211461C2001F055F80020E8
:10B2500010BD2DE9F04103F00705274E174688463B
:10B260000446012D04BF0020F0601BD013F0070F2F
:10B2700016D103F01FF998B1F068204B03283CBFAA
:10B2800019680F54401CF06003280BD1186890F91E
:10B29000022090F9011090F90000FAF705FF01E093
:10B2A000022D02D00020BDE8F081F06830B1012805
:10B2B00009D002280CD003280FD015E01420FAF78B
:10B2C0009AFD207010E01520FAF795FD20700BE034
:10B2D0001620FAF790FD207006E01720FAF78BFD94
:10B2E0002070012088F80000F068401CF060012008
:10B2F000BDE8F081C785001078850010E44C02009D
:10B3000070B50D46044603F007000021FE4E0128EB
:10B3100014BF13F0070FF16001D0022801D0002004
:10B3200070BDF06840B101280BD002280ED0032870
:10B3300011D0042814D019E00120FAF75CFD207028
:10B3400014E00220FAF757FD20700FE00320FAF70F
:10B3500052FD20700AE00420FAF74DFD207005E050
:10B360000520FAF748FD207001202870F068401C85
:10B37000F060012070BD70B503F0070C0026E34CAF
:10B38000E14DBCF1010F06D013F0070F0CD0BCF15A
:10B39000020F1FD01CE007F074FBEE6021680870FC
:10B3A0002168000A487013E0E868022803D2216887
:10B3B0000A54401CE86002280AD1EE602068007838
:10B3C00010F0010F04D002221920216800F094FF30
:10B3D000002070BDEA68022A28BF104604D2236804
:10B3E0009B5C0370501CE860022804D10120EE60D1
:10B3F000087003202870012070BD7FB51C460E46E2
:10B40000054613F0070F08D103F054F828B10122C4
:10B4100002A9232000F070FF03E004F007000228D7
:10B4200002D004B0002070BD0EF04EFE2870012046
:10B43000307004B070BD7FB51C460E46054613F053
:10B44000070F08D103F036F828B1012202A91E2007
:10B4500000F052FF03E004F00700022802D004B01D
:10B46000002070BD0EF03BFE28700120307004B04B
:10B4700070BD7FB51C460E46054613F0070F08D178
:10B4800003F018F828B1012202A9222000F034FFAD
:10B4900003E004F00700022802D004B0002070BDD1
:10B4A00011F049FE28700120307004B070BD7FB5E6
:10B4B0001C460E46054613F0070F11D102F0FAFFA5
:10B4C00070B10EF018FE01469DF8080081420BD0C5
:10B4D0000EF00EFE012202A91D2000F00DFF03E078
:10B4E00004F00700022802D004B0002070BD0EF066
:10B4F00002FE28700120307004B070BD2DE9FF41BC
:10B50000814E1C460F46054613F0070F1CD102F072
:10B51000D1FFC8B19DF80800002818BF012802D04B
:10B52000022807D014E0F070012202A9082000F0E0
:10B53000E3FE0DE0F07004208DF80800012202A95E
:10B54000082000F0D9FE03E004F00700022803D031
:10B5500004B00020BDE8F081F07828700120387038
:10B5600004B0BDE8F0817FB51C460D46064613F0D9
:10B57000070F08D102F09EFF28B1012202A908207E
:10B5800000F0BAFE03E004F00700022802D004B085
:10B59000002070BDFBF710FF801E052813D2DFE8E6
:10B5A00000F003070E05100000240DE001240BE05D
:10B5B000022406F0B2F8042808BF052404E003249E
:10B5C00002E0042400E0FF2434700120287004B05D
:10B5D00070BD2DE9F0411C4617460E46054613F096
:10B5E000070F0BD102F066FF40B1384607F05EF856
:10B5F00000221146012000F07FFE03E004F0070066
:10B60000022802D00020BDE8F08107F052F828702F
:10B6100001203070BDE8F08110B5104613F0070F1F
:10B6200008BF07F00DF9002010BD10B5104613F04B
:10B63000070F08BF07F00BF9002010BD70B50446D6
:10B6400003F007000D4602281CBF002070BD07F064
:10B6500006F920700120287070BD03F0070230B495
:10B66000294B4FF0000C012A05D0022A04BF1A789A
:10B67000022A0BD01EE0022018702548C3F80CC027
:10B680006FF07F410068081AD86113E0DA68042A75
:10B6900028BF104606D2DD69D40025FA04F40470F0
:10B6A000501CD860042805D10120C3F80CC00870D4
:10B6B0000320187030BC0120704713F0070F04BF3F
:10B6C000144802700020704710B503F007000E49BF
:10B6D000012804BF0020C86013D013F0070F10D159
:10B6E000C8680A4B04283CBFD3F800C00CF80020FF
:10B6F000401CC860042804D104221220196800F0FC
:10B70000FBFD002010BD000078850010E44C020015
:10B71000AC8400102E8400102DE9F047164603F08B
:10B7200007020024F74F012A04BFFC603C6164D08B
:10B73000DFF8D48313F0070F07D0022A33D0042A8E
:10B7400004BF387806284FD058E0FD68002D08BFA8
:10B750003E6225D0012D06D0D7F81490AC1E4C4582
:10B7600016D284B908E0701C7861396A0844B0F5D3
:10B77000007F88BF7C6113E04FF400724FF47A3190
:10B78000E24813F02BFFE249386A096820440E545E
:10B79000601C484504D1DD48C0F8FC8106203870A3
:10B7A000681CF8602AE0FF2202707B69CBB1D7F8F1
:10B7B00020C03A699444BCF5007F10D2D54D2D6865
:10B7C000454518BF047005D10CF5783C9CF800C8BD
:10B7D00080F800C0501C984204BF01200870501C23
:10B7E00038610120BDE8F0874FF47A30F8F7D4FAD9
:10B7F000C6494FF47A30F8F771FB3C700020BDE881
:10B80000F0872DE9F0478C4603F007010024BD4F77
:10B810001646012904BFFC603C6162D013F0070F9B
:10B82000BD4BDFF8F88207D0022932D0042904BFCB
:10B83000387806284DD055E0FD68002D08BF3E62DF
:10B8400024D0012D06D0D7F81490AC1E4C4515D24B
:10B850007CB908E0701C7861396A0844B0F5007F53
:10B8600088BF7C6112E04FF400721946A74813F0BC
:10B87000B5FEA749386A096820440E54601C484543
:10B8800004D1A248C0F8FC8106203870681CF8601A
:10B8900028E0FF2101707B69C3B13A6A39690A4423
:10B8A000B2F5007F10D29E4D2D68454518BF04703B
:10B8B00004D102F5783292F800260270481C9842B2
:10B8C00004BF01208CF80000481C38610120BDE84D
:10B8D000F0871D461846F8F75FFA8C492846F8F7B6
:10B8E000FDFA3C700020BDE8F08770B503F007005A
:10B8F000844C1546012804BF0020E06014D013F0EA
:10B90000070F11D102F0D6FD70B1E068804902281E
:10B910003CBF0A681554401CE060022804D1022292
:10B920000968052000F0E8FC002070BD2DE9F04119
:10B93000054603F00700764C724E0F4601280AD0E8
:10B9400013F0070F14D002281BD0042804BF30784E
:10B95000062834D03FE00020F0602168087021689C
:10B960004870216888702168C8700520307032E006
:10B97000F06804282FD221680A54401CF060062089
:10B9800028E0F06860B906F09EFC21680870226823
:10B99000010A51702268010C000E91702168C87074
:10B9A000F06804283ABF2168095CFF21297024BF90
:10B9B00001213970401CF0600120BDE8F08102F0E7
:10B9C00079FD40B12068C178006861F31F6006F01E
:10B9D00075FC032030700020BDE8F0810020704726
:10B9E0007FB51C460E46054613F0070F08D102F03E
:10B9F00061FD28B1012202A9262000F07DFC03E0B0
:10BA000004F00700022802D004B0002070BD06F048
:10BA10004CFF28700120307004B070BD03F00700A7
:10BA20003849012808BF002009D013F0070F07D1BB
:10BA3000C86818B93B4B1B681A448A61401CC8602F
:10BA4000002070472DE9F04103F007012D4C164608
:10BA50000546012907D0334F13F0070F386806D089
:10BA6000022919D015E00020E060206111E0A569ED
:10BA700005F062FE01280CD1A0693968884224BF14
:10BA8000E031814205D9E068042838BF2E54401CBB
:10BA9000E0600020BDE8F081A66905F04DFE50B1E0
:10BAA000A26939688A4224BF01F1E000904284BF54
:10BAB0002069305C00D8FF2028702069401C20617C
:10BAC0000120BDE8F0817FB51C460E46054613F007
:10BAD000070F08D102F0EEFC28B1012202A91120C3
:10BAE00000F00AFC03E004F00700022802D004B0D2
:10BAF000002070BD11F087F928700120307004B06B
:10BB000070BD000078850010554E564D24A90010D8
:10BB1000E44C0200FCE9030000E60300324E564DFF
:10BB2000FCE703002C8700100020704700207047BE
:10BB300070B50D46044613F0070F04D003F007005C
:10BB4000022805D002E0104609F0A7FE002070BDD3
:10BB500009F0AFFE20700120287070BD10B503F011
:10BB60000702F84CF84B4FF0000C012A02D0022AD1
:10BB700034D031E0C3F80CC002F09CFC00282BD07C
:10BB8000F24802F0AFFD38B3F1480068007E10F0D3
:10BB9000040FEE4810D0418C2268090A1170226807
:10BBA00090F822105170018C2268090A9170216866
:10BBB00090F82000C8700FE0018C2268090A11700B
:10BBC000226890F820105170418C2268090A917007
:10BBD000216890F82200C870002010BDDA68042A9D
:10BBE00028BF104604D22468A45C0470501CD8609E
:10BBF000042803D10120C3F80CC00870012010BD37
:10BC000070B503F00701CF4DCF4C012902D00229B6
:10BC100014D011E0012001F062FC0020E06001F08E
:10BC200073FC2081296808702A68010A0028517075
:10BC300004BF002001F053FC002070BDE168022920
:10BC400002D22A68525C0270481CE060012070BD7C
:10BC50002DE9F04103F007020026BB4D0F460446D4
:10BC6000012A02D0022A09D005E005202870EE60E2
:10BC70002889400068610020BDE8F0812878052807
:10BC800017D1EA686869824205D212F0010F1CBF21
:10BC90006878207010D0E868401CE86069698842C4
:10BCA00007D10120EE60387003202870002001F0D9
:10BCB00016FC0120BDE8F08101F03FFC010A217073
:10BCC0006870E8E71FB513F0070F04D1012202A93D
:10BCD0001A2000F011FB04B0002010BD00207047B6
:10BCE0000020704703F007009749012806D013F0A1
:10BCF000070F04BF0878012806D014E0012008705F
:10BD00000020C86088610DE0C868042805D28B69EE
:10BD1000401C42EA03228A61C860042803D1032040
:10BD20000870886908620020704703F00700DFF898
:10BD300018C2012807D013F0070F04BF9CF80000B9
:10BD4000022809D01EE002208CF800000020CCF868
:10BD50000C00CCF81C0015E0DCF80C00022808D21E
:10BD6000DCF81C10401C42EA0121CCF81C10CCF875
:10BD70000C00022806D1DCF81C00CCF824000320BB
:10BD80008CF800000020704770B403F00702002513
:10BD90006D4C012A02D0022A06D002E00220207057
:10BDA000E56070BC002070472278022A1CD1D4F8CC
:10BDB00024C0E268624528BF10460ED212F0030F7D
:10BDC00004D1236A53F8046BC4E90763237F03702B
:10BDD000E069000AE061501CE060604504D1012088
:10BDE000E56008700320207070BC0120704770B5BA
:10BDF00003F007000025544C0E46012806D013F02E
:10BE0000070F04BF2078022805D02BE00220207005
:10BE1000E560E56126E0616AE068884219D2E1697F
:10BE2000090A41EA0262401CE26110F0030FE0607F
:10BE30000FD1206AB0F5802F28BF026006D2B0F57E
:10BE4000005F03D304224349F8F79CF8206A001DE1
:10BE50002062616AE068884204D10120E5603070A8
:10BE600003202070002070BD70B503F0070C002582
:10BE7000354CBCF1010F08BFE5603AD013F0070F55
:10BE800003D0BCF1020F36D033E0052A08BF4FF4CF
:10BE90007A302DD005DC16D2DFE802F0171A1D200B
:10BEA00022002B48202A006808BFF83020D006DC8A
:10BEB000102A1DD0112A08BF244819D003E0302AC7
:10BEC00011D0312A12D0A56113E04FF400500FE0D9
:10BED0004FF47F300CE04FF4483009E01E4807E093
:10BEE0004FF47C3004E001F07FFC01E010F03FFBF8
:10BEF000A061002070BDE268042A07D2C2F10303EA
:10BF0000D4F818C0DB002CFA03F30370501CE06077
:10BF1000042824BF01200870012070BD70B403F014
:10BF2000070C094DBCF1010F07D0064C13F0070FA9
:10BF300014D0BCF1020F2ED02AE00020E860286166
:10BF400026E00000E44C020078850010A8300110C3
:10BF50000C8700109485001000EE0300E8680528A7
:10BF60003CBF21680A54042810D123682268D4F801
:10BF700000C0D3F80130A96912781BBA9CF804C03C
:10BF800023F0FF0343EA0C0341F82230401CE86031
:10BF900070BC002070472B6973B1042B07D2226854
:10BFA000032B1A445278027004BF01200870581CF9
:10BFB000286170BC012070472268D5F818C012783B
:10BFC0005CF8222026684FEA126C86F801C02668C9
:10BFD0004FEA124C86F802C026684FEA122C86F807
:10BFE00003C0D4F800C08CF80420D8E710B503F0E3
:10BFF0000700012804D1002211460E2000F07CF930
:10C00000002010BD2DE9F04103F00704A94E1746AA
:10C0100088460546012C04BF0020F06017D013F0BD
:10C02000070F12D102F046FA78B1F068A24902284F
:10C030003CBF0A681754401CF060022807D1022256
:10C040000968072000F058F901E0022C02D0002016
:10C05000BDE8F081F26812B1012A04D009E0FBF7D3
:10C06000ABF9287005E0FBF7ADF92870012088F8DE
:10C070000000F068401CF0600120BDE8F08170B560
:10C0800003F0070000258B4C012808D013F0070FA0
:10C090000BD0042804BF2078062825D02DE0A56108
:10C0A000E5616570E560257027E0E068022807D249
:10C0B000A16942EA0121A16161781144617010E037
:10C0C000042807D2E16942EA0121E1616178114463
:10C0D000617006E0052804D261788A4204BF062117
:10C0E0002170401CE06008E0D4E9060101F016FC74
:10C0F000002804BF0120A0702570002070BD10B57D
:10C100006C4C13F0070F07D003F00700042804BF9E
:10C110002078062822D02BE0E068022807D2A16907
:10C1200042EA0121A16161781144617013E0634921
:10C13000091808D260490968014401F8022C6178A5
:10C140001144617007E05E49091804D261788A429F
:10C1500004BF06212170401CE06009E05949A06934
:10C1600001F0FEFB002804BF0120A0700020207019
:10C17000002010BD03F0070CBCF1010F00D0BEE79A
:10C180004C49002088614870C8600870704730B41E
:10C1900003F007050024DFF81CC1012D07D013F0C0
:10C1A000070F0DD0022D3CD0042D54D06FE0CCF8F9
:10C1B0001840CCF81C40CCF80C408CF8004066E0ED
:10C1C000DCF80C0002280BD2DCF8181042EA01213E
:10C1D000CCF818109CF8011011448CF8011019E0EB
:10C1E000042817D2DCF81C10032842EA0121CCF8FD
:10C1F0001C109CF801301A448CF801200AD1062248
:10C200008CF80020DCF81820114304BF4FF40071B3
:10C21000CCF81C102C49401CCCF82C10CCF80C008D
:10C2200035E0DCF80C20042A28BF10460AD2C2F1FF
:10C230000303DCF82C50DB0025FA03F30370501CD9
:10C24000CCF80C00042803D10120CCF80C40087075
:10C2500030BC012070479CF80000062815D1DCF89E
:10C26000180000224102DCF81C0043021046B2EB29
:10C27000930F06D251F8045B401C2A44B0EB930F95
:10C28000F8D3CCF82C208CF80040CCF80C4030BC13
:10C29000002070474FF47F300168880A424211EB5A
:10C2A000822218BF401C404201EB8000C01C20F0DD
:10C2B0000300704778850010E44C0200FEFDFFFF8C
:10C2C000FDFDFFFF24A90010EFBEADDEF748002200
:10C2D00002704270827002714271C270DFF8D0C386
:10C2E000114600200CEBC1031A54401C0828FBD354
:10C2F000491C2029F5D3704713F0E3B92DE9F0412B
:10C3000015460E460746F8F7ABF900F0080408207A
:10C31000F8F7A1F92A463146384613F0D2F9054616
:10C320002046F8F793F92846BDE8F081DF48807889
:10C330007047DE4840787047DC49002048707047FD
:10C340002DE9F04100250C46292880F0F181DFE835
:10C3500000F0F0CD15232C3B1A48EF4BF08389BA3F
:10C36000EE8E97A1EDECEBEAE9CEF1FFE6E5E4E332
:10C37000E2E1E0F0DFDEF0DD9CF0F6000020F9F70E
:10C380003BFB00F0A5B92078AC280CBF01200220AF
:10C39000FBF7E9F800F09CB921780120FBF727F8BA
:10C3A000C2490120487000F093B9E178206861F338
:10C3B0001F6002F0A7F901210320FBF718F8BB4921
:10C3C0000120487000F084B9208840BA05F07EFF53
:10C3D00002210320FBF70BF8B4490120487000F05C
:10C3E00077B961782078C7E0B04E01277770307850
:10C3F00070BBF6F780FC58B324783770FAF7DCFF8F
:10C40000012808BF002414F0040F18BFFCF7FFFD3B
:10C4100014F0020F06D01F20FBF776FFF9F7D2FBCE
:10C4200044F0010414F0010F10D0FAF7C5FF022800
:10C4300002D106F04FF948B1FAF7BEFF052802D144
:10C4400001F0C9FA10B10020F9F7A9FB0020307003
:10C450000020707000F06CB92078401E01F01AFEC8
:10C4600000F036B9207806F000FA00F031B92078F3
:10C4700010F00F0018BF01200DF003FA00F058B9BA
:10C4800020780DF0F4F900F053B9207806F001FAA5
:10C4900000F04EB9207818B1012809D000F048B951
:10C4A000002010F0ADFC002010F063F8002006E042
:10C4B000012010F0A5FC032010F05BF8012010F023
:10C4C0007BF800F035B9207860B1FAF775FF0228E3
:10C4D00018BF012506F0AEF901460220FAF787FFE2
:10C4E00000F026B900210620FAF781FFF0E020785D
:10C4F000002818BF012006F086F92078002818BF10
:10C50000012001F053FA00F013B918E00DE106E143
:10C5100001E1D3E0CEE0DDE09EE068E0D2E01BE0A8
:10C5200016E007E07DE073E06DE063E055E026E0B3
:10C530003AE05BE0207806F052F900F0F9B801F03B
:10C5400095FB01462078814218BF01F08AFBEFE09D
:10C55000208806F01CFABBE0207820B1012845D0E5
:10C56000022805D0E4E04FF47F30F7F715FCDFE058
:10C5700001F0F8FF00210420FAF739FFA8E0F8F7EE
:10C580006FF800F008040820F8F765F84749CA7802
:10C59000002A04BF00228A702046F8F757F80121CC
:10C5A0000620FAF724FF93E02078062804D2DFE87B
:10C5B00000F00306090B0E1102210846DCE70221F8
:10C5C0000520D9E7002106E000210420D4E700215E
:10C5D0000620D1E704210320CEE7E078226800237B
:10C5E00060F31F626221072004F0A2FFA0E0F9F7C8
:10C5F000EFFD6DE02068E17800BA20F0FF0008430D
:10C600000BF0E4FE25E0208840BA0BF0CEFE8FE070
:10C610002068E17800BA20F0FF0008430BF0AEFE7E
:10C6200086E020780BF0F3FE6078A178000140EA04
:10C6300011100BF0FDFEA178607901F00F0140EAC6
:10C640000160E1782279090441EA022108430BF0F4
:10C65000E5FE0BF0F0FE6BE0FAF7AEFE02281CBF21
:10C660000628052864D12078012804D0022818BFA4
:10C67000002805D02CE00CF000F8002106207BE714
:10C68000FAF7B2FE0546FAF797FE0646207800282C
:10C6900004BF0020F9F7B0F9022D14BF052D062EB6
:10C6A00016D106F0C7F80146284665E7B0850010A8
:10C6B00024AB0010207806F014FA09E0207806F088
:10C6C00018FA05E02078002818BF0120FAF779FF52
:10C6D00001252DE00DF003FD247806F0D2F9012CA0
:10C6E00011D0022C12D0042C18BF082CF0D140F02D
:10C6F000005006F002F9042C18BF082CE8D120469F
:10C700000DF0E8FCE4E706F0F8F8F8E740F08050B8
:10C7100006F0F3F8F3E7207810F010FD08E0207839
:10C720000DF0CFFC06F00CF802E0207800F0B2FA31
:10C730002846BDE8F081C849CA681043C860704700
:10C7400010B5D0B1FAF738FE0446F8F7BFFB052C58
:10C750000ED07820F4F7C1FB0520F8F7A4FBBF4802
:10C76000F8F7D6FCF8F7B9FCBDE81040F8F73CBC88
:10C770003C20F4F7B2FB0320EFE7F8F73EFCF8F7B4
:10C78000B9FC0020F8F7C4FCBDE81040F8F780BB06
:10C79000B14910B508208871FAF70EFE022818BFBB
:10C7A000012811D0032818BF05280DD00020F6F766
:10C7B000AAFAF8F722FCF8F79DFC0020F8F7A8FC8D
:10C7C000BDE81040F8F764BBAFF28B00BDE8104045
:10C7D000F6F799BA2DE9F0474FF00008F6F79BFA03
:10C7E000DFF874A20446DAF80C00C14640B1DAF86A
:10C7F0000C0010F0400F18BF44F00404CAF80C906D
:10C8000014F00F0666D00127FAF7D6FD054630462C
:10C81000F6F79EFA012E1DD0FAF7D4FD44EA006423
:10C82000002322460321072004F082FE14F0050FA6
:10C8300014BF00200120F3F79EFD14F0060F49D02D
:10C840004FF0010805F046FF0646022D2ED0052DBB
:10C850000AD03FE09AF80600854208BF00278AF810
:10C860000650002FD8D1E8E714F0020F03D00020C3
:10C87000F9F7D2F820E07A4840698047044601F091
:10C88000F5F901281CBF207810F0040F02D010F039
:10C89000080F02D00120F9F7BFF8724C206858B198
:10C8A0000120F9F7A9F8C4F8009005E014F0020F90
:10C8B0001CBF0120F9F7A0F801F099F8002818BF73
:10C8C00001F09CF8022E05D0022D4FF0020004D09A
:10C8D00001F076F84046BDE8F08705F0A3FFF9E7E0
:10C8E0002DE9F04F83B00026F8F775FCFAF764FDE8
:10C8F000022804D101F09AFD002818BF0126FFF795
:10C9000069FF002818BF0126DFF84C8198F8020063
:10C9100000287DD0D8F808006D464FF0FF344FF066
:10C92000000940B1D8F8082000230121084604F08E
:10C93000FFFDC8F80890F7F793FE00F0080A0820FA
:10C94000F7F789FE98F80300DFF81CB1F8B198F802
:10C9500005000BEBC001401CC0B288F80500202880
:10C9600028BF88F8059098F80300401E88F8030057
:10C970004C780F780020002C05DD0A1892782A5494
:10C98000401C8442F9DC81F8009081F80190504607
:10C99000F7F75CFE002C47DB22466946F8B2FFF74A
:10C9A000CFFC08B101263FE0D8F808006D464FF0F3
:10C9B000FF3440B1D8F8082000230121084604F0D4
:10C9C000B7FDC8F80890F7F74BFE00F0080A0820FA
:10C9D000F7F741FE98F8030008B398F805000BEB51
:10C9E000C001401CC0B288F80500202828BF88F884
:10C9F000059098F80300401E88F803004C780F78E3
:10CA00000020002C07DD0A1892782A54401C00E010
:10CA10001AE08442F7DC81F8009081F801905046DA
:10CA2000F7F714FE002CB7DAF7F71AFE00F0080447
:10CA30000820F7F710FE98F80310002908BF88F8BF
:10CA400002902046F7F702FE002E14BF01200020BE
:10CA500003B0BDE8F08F0000B0850010E7E60000ED
:10CA6000A45102001C86001024AB001002460020D6
:10CA7000022928BF704752B1012A18BF704701EB45
:10CA80004100C0EB4110FE4901EB8000704740F2CD
:10CA9000DB104843FB49F7E770B5F7F7E1FD00F01D
:10CAA00008060820F7F7D7FDF74C00256078FF2827
:10CAB00006D240F6D861F34812F095FDE570257175
:10CAC000E079FF2805D2E821ED4812F08CFD2572AF
:10CAD00065723046BDE87040F7F7B8BDDFF8ACC30B
:10CAE00000FB01F31CEB030C88BF7047E64B1A6296
:10CAF000C3E906017047DFF890C30028DCF818305E
:10CB000018BF0360E0480029C06918BF0860002A08
:10CB10001CBFDCF82010116058437047DA4801212F
:10CB20004171007840F2DB1180F001004843D549A3
:10CB300001EB80007047D448C278002132B10279FD
:10CB400022B9027882F001020270C170417170470F
:10CB5000CD4900231E284A78487006D01F2804BFFC
:10CB60000120087002D0512800D10B701046704788
:10CB7000C548007840F2DB1180F001004843C1490C
:10CB800001EB800070472DE9F007BF4F97F800C018
:10CB900040F2DB140CFB04FCBA4CBE6904EB8C0CB9
:10CBA00003FB06F40CEB440C8E4234BF35460D46B5
:10CBB000FC69E31A934238BF1A46BB78012B16BFB3
:10CBC000052B6C0800244FF00008002A9CBFBDE82C
:10CBD000F00770472346AC420FD297F80290B9F1A4
:10CBE000050F30F8139006BFA3EB040A2CF81A9037
:10CBF0002CF813905B1CAB42EFD308F101080CEB4F
:10CC0000460C00EB41009045E4D3BDE8F0077047C7
:10CC10002DE9F0419C4F14468C4601467A780698DF
:10CC20001D468A4218BFBDE8F081012139710128F3
:10CC300002D0022824D029E0387840F2DB114843A2
:10CC40009049BE6901EB8001A64234BF32462246BC
:10CC5000F869A84238BF05460023002D16D90020E8
:10CC6000002A06D91CF8007021F81070401C82427E
:10CC7000F8D85B1C01EB4601A444AB42EFD305E0BE
:10CC800000232A4621466046FFF77DFFBDE8F041BC
:10CC900000F0A0BC7C4A01281146D072497808BF38
:10CCA000242004D0002806BF2429FF20704750709C
:10CCB00070477548C07A704770B4DFF8D4C1DCF8AB
:10CCC00000C0DCF818C01CF0040F1ABF012424EACD
:10CCD0000C060CF0010605680C68002E1CBF1B1B1F
:10CCE0005C1E1CF0020F1CBF521B551E1CF0040FD3
:10CCF00019BF04600D6005600C6070BC70470028AF
:10CD000008BF70476049634B4A7863491B78002A23
:10CD1000097818BF022A05D0042A18BF092A01D0B1
:10CD2000012230E75D4A1278012A84BF5C4A1378F9
:10CD3000012200F069BC2DE9F041534C0F4601215E
:10CD40002171584A1578534A167828B1A1700023EA
:10CD500032462946FFF717FF3FB10520A070002398
:10CD6000324629463846FFF70EFF00F033FCFF201D
:10CD7000A070BDE8F0812DE9F04FDFF80C918BB089
:10CD8000012189F804104749444C454E0D7841492A
:10CD9000DFF8F0B00F7899F80110122934D00DDCCB
:10CDA000092921D005DC00291CBF0229042911D141
:10CDB0001AE0102918BF11290CD125E0222977D0BB
:10CDC00004DC132920D0212972D003E0242970D05B
:10CDD000512919D0002800F0308100233A46294615
:10CDE000FFF7D1FE00F029B92178012902D92E4997
:10CDF00037780D78002800F0208100233A46294634
:10CE000000F002FC00F019B9F5F763FEF5F768FDD4
:10CE10000090002818BFF5F7FEFF2078012888BF92
:10CE20003778F5F775FF10F0020F18BF7F1CDFF899
:10CE30007C8099F8016099F8000040F2DB114143D1
:10CE4000D9F818000BEB8104A84238BF0546D9F881
:10CE50001C00B84238BF0746F6F78AF80190002058
:10CE6000F6F7E7FC4FF0000A002F4EDD4FF0000907
:10CE7000002DC4BF0AEB4A0000EB0A1B3DDD19E0A0
:10CE8000FCBA001024AC0010C08500104AFCFFFF63
:10CE90000C87001042850010488500104385001063
:10CEA00045850010418500104485001000000130C8
:10CEB0003EE045E0019810F90900262824BF002033
:10CEC00024F8190015D200F0010108EB813100EBC4
:10CED000D07001EB8B014010102E51F820001AD0B9
:10CEE000112E1FD0122E0CBFC0B2F6F7A8FC24F8EA
:10CEF000190009F10109A945C1DBFE480AF1010A3F
:10CF0000BA45806904EB4004B0DB0098002818BFE4
:10CF1000F5F784FF91E010F4003FC0F34230E6D013
:10CF20004042E4E710F4803FC0F30420F8D1DEE78C
:10CF300000287DD00023BA1C2946FFF724FE7CE0A0
:10CF400000287AD00646EC480068007E10F0040FF6
:10CF500007BF2C46BA463C46AA46A1084FEA9A02A9
:10CF60000592A4EB9400069200916208401ECDE960
:10CF700001020391AAEB9A0104904FEA5A02491E5A
:10CF8000CDE9072109915346224605A96846FFF7D6
:10CF900093FE5346224605AF06A9E84601A8FFF7CF
:10CFA0008BFE5346224607F1080108F10800FFF7FF
:10CFB00083FE5346224607F10C0108F10C00FFF7EF
:10CFC0007BFE5346224607F1100108F11000FFF7DF
:10CFD00073FE99F8000040F2DB11414300220BEB95
:10CFE0008100914620F8129058F82210A1F1010C0E
:10CFF000491C61451ED357F822104B1E491C99420B
:10D000000FD303FB05C136F9114030F912108C42E1
:10D01000C8BF20F8124057F822105B1C491C9942E7
:10D02000EFD258F822100CF1010C491C614500E0C8
:10D0300003E0E0D2521C052AD4D30BB0BDE8F04F78
:10D0400000F0C8BAAB4801218172807980F00100FC
:10D0500000EB4001C1EB4010A84901EB8000704794
:10D06000A448027A002132B1427A22B9827982F050
:10D07000010282710172817270479E491E28CA792D
:10D08000C87108BF002003D01F2808BF012000D1AD
:10D090008871104670479748807980F0010000EB56
:10D0A0004001C1EB4010954901EB800070472DE92C
:10D0B000F04F9349DFF83C8285B00F7891490E78A4
:10D0C000012188F8091098F807108C4C4FF00009DE
:10D0D000102918BF11293AD0122918BF132936D0A8
:10D0E000F0B198F8061001EB4102C2EB411104EBDC
:10D0F0008102002116EB070C18BF7F4C10D023686B
:10D10000002E5B8A03BF30F811500B4422F81350F5
:10D1100030F8113018BF22F81130491C8C45EED878
:10D12000F7F79EFA00F008040820F7F794FA98F849
:10D130000A0000281CBF012188F808107CD0204676
:10D14000F7F784FA88F8099005B0BDE8F08FF5F795
:10D15000C0FCF5F7C5FB0290002818BFF5F75BFE91
:10D1600098F80750D8F82400009098F8060000EBD3
:10D170004001C1EB401004EB800BF4F73DFC0028AC
:10D180006AD01120F3F739FC00280CBF12201120BF
:10D1900060F3070A0120F3F730FC002814BF0120D8
:10D1A000022060F30F2A0AF0FF000190F6F741FB1E
:10D1B000F5F7DCFE00240390002E1FD903980257D8
:10D1C000142AA8BF143A02DA0A2AA8BF1232262A61
:10D1D00028BF2BF814900ED2DDE90010F5F702FA03
:10D1E000102D4AD0112D4FD0122D0CBFC0B2F6F722
:10D1F00026FB2BF81400641CB442DFD30BEB46066D
:10D20000CAF3072B5846F6F714FBF5F7B1FE0024D6
:10D210008246002F1AD91AF90420262A28BF26F898
:10D22000149010D258460099F5F7DCF9102D31D042
:10D23000112D36D0122D00E039E00CBFC0B2F6F748
:10D24000FEFA26F81400641CBC42E4D302980028BD
:10D2500018BFF5F7E3FD63E70120F3F7CEFB0028E5
:10D2600014BF0120022060F3070A1120F3F7C5FB69
:10D27000002814BF1120122093E710F4003FC0F3E0
:10D280004230B6D04042B4E710F4803FC0F30420EF
:10D29000F8D1AEE710F4003FC0F34230D1D04042A5
:10D2A000CFE710F4803FC0F30420F8D1C9E798F825
:10D2B000060080F0010088F8060088F808903EE734
:10D2C00070B50D460B4901220A710F4A497816784C
:10D2D0000E4A212914781EBF2229232970BD002857
:10D2E00018BF002D20D0002322463146FFF74BFC0B
:10D2F000631C0DE0C08500100C870010FCBA001004
:10D3000046850010478500104185001042850010B9
:10D31000012221462846FFF736FC05EB4400A31CFA
:10D3200001223146FFF72FFCBDE8704000F052B9F2
:10D3300070B50446C068D74D68B1697859B9D64907
:10D34000097801298CBFD549D5490B78D5490122E7
:10D35000097800F059F9A06820B16978002908BF60
:10D36000FFF709FD6878102804BF0020FFF703FDD0
:10D370006878112804BF0020FFF7FDFC68781228A8
:10D3800004BF0020FFF7F7FC6878132804BF0020D3
:10D39000FFF7F1FC206920B1E979002908BFFFF708
:10D3A00086FEE879102804BF0020FFF780FEE879A8
:10D3B000112804BF0020FFF77AFEE879122804BF85
:10D3C0000020FFF774FEE879132818BF70BD002015
:10D3D000BDE870406BE62DE9F74F8046B2480D4638
:10D3E000002690F800A0AE48AA49344690F8009074
:10D3F000BAFBF5F000FB09F701200871487B0978BA
:10D40000DFF8A8B288420ED0A24A40F2DB114843AE
:10D410000BEB8001107840F2DB1250430BEB8000E5
:10D42000920012F0EAF80298002888BFDFF864B290
:10D430002DD99BF80EC00022BCFBF9F009FB10C1EE
:10D4400001FB0AF100FB0510002D12D938F8143049
:10D450009BF8001040F2DB1E01FB0EFE9349641C9A
:10D4600001EB8E0100EB020E521C21F81E3095429A
:10D47000ECD80CF10100C0B28BF80E00B84224BF0A
:10D4800000208BF80E00761C02988642D1D3814989
:10D49000887B401EC0B2887387429CBF781E887309
:10D4A0000878487303B0BDE8F04F00F093B87948AE
:10D4B000017800F1280281F0010132F811100029F1
:10D4C00018BF7047017881F00101017000210182CD
:10D4D000037822F81310764A0078115470476D498A
:10D4E000087370476B48007B704770B5694C002526
:10D4F000257025732582658240F6D8616B4812F04D
:10D5000072F8A562A58270BD6249087800224A823D
:10D5100080F001001431095C69B140F2DB11634A0B
:10D52000414332F82110A1F55062B63A02BF614979
:10D5300031F81000704700207047564B187803F1FF
:10D54000140C80F001014FF6FF701CF80120012A35
:10D5500018BF704740F2DB104843544A02EB80008A
:10D560005A8A30F81200521C5A82524B33F811205A
:10D57000521E1204120C23F8112004BF00220CF8D2
:10D58000012070474B49A1F12802137801EB4301B8
:10D590000B8803440B8092F800C0012102F11403B0
:10D5A00003F80C10118A084410827047394A138A14
:10D5B00003EB5000404B01445B1824BF0020704730
:10D5C000117840F2DB125143384A02EB810101EB42
:10D5D0004000704770B5F7F743F800F008060820E0
:10D5E000F7F739F82B4C60790025002801BF207827
:10D5F00080F001002070E5701CBF0120E070304613
:10D60000F7F724F8257170BD2DE9F04799461646C5
:10D610000D460446F5F7B1FC5FEA000C1CD01D492D
:10D62000087840F2DB125043204AD1F8188002EB10
:10D63000800009FB08F200EB4200454594BF2F46ED
:10D640004746C969A1EB0901B14238BF0E46002126
:10D65000002E09D8BDE8F0874B46324629462046C1
:10D66000BDE8F047FFF78FBA0023002F08D91CF957
:10D67000032034F8122020F813205B1C9F42F6D8B8
:10D68000491C00EB480004EB4504B142ECD3BDE873
:10D69000F0870000C085001043850010458500100C
:10D6A00042850010488500104185001024AC001010
:10D6B000D4850010E88500104AFCFFFF414900288E
:10D6C00014BF00200120087070473E4800780028F1
:10D6D0000CBF01200020704701203A494870704774
:10D6E000384800214170017800291ABF406800289D
:10D6F00070473548016821F00101016070473148E9
:10D70000017821B130490A6842F001020A60002123
:10D7100041608160C160016170472A48017821B190
:10D7200029490A6842F001020A60002141608160D3
:10D73000C1600161704700B50178427885B0890108
:10D7400041EA82018DF80010418809098DF8011025
:10D75000818809098DF80210817801F00F020179A2
:10D7600062F31F118DF80310017A8DF80410417ACD
:10D770008DF805108179C27901F03F0102F00C02A9
:10D7800041EA02118DF80610C179827A890102F00E
:10D79000010241EA42118DF80710C17B8DF8081093
:10D7A000017C8DF80910407C00F00F008DF80A0014
:10D7B00000208DF80B000390684611F087FF05B03C
:10D7C00000BD0000EC850010144C0040002818BF7C
:10D7D00047484849886370474648806B44498842B7
:10D7E0000CBF01200020704742487047424B4FF069
:10D7F000000C1C681B1F1D683E4B19605A603F4996
:10D80000D963DC6214F0804F22D0290C5985290A93
:10D8100083F8291083F82850598D19B1598D0122A8
:10D8200042EA014C93F8291039B193F829100222E9
:10D8300042EA014C32490C681C6393F8281039B154
:10D8400093F82810032242EA014C2E490C685C63CD
:10D850002D490C60091DC1F800C02C4A8169116076
:10D86000B0E816109960DA601C61C3F814C090E843
:10D8700007109861D9611A62C3F824C0986B1C49DB
:10D88000884202D1234922480860FEE72249012844
:10D8900004BF09607047022818BF70470847154841
:10D8A000D0F8EC201C498A4204BFD0F8F0208A420C
:10D8B00008D1D0F8F4208A4201BFD0F8F8208A427B
:10D8C00001207047C0F8EC10C0F8F010C0F8F41058
:10D8D000C0F8F8100020704706480F49C0F8EC1057
:10D8E000C0F8F010C0F8F410C0F8F810704700004D
:10D8F000504D5544005F01102CED00E0544C414662
:10D9000038ED00E034ED00E0344C00403C4C004089
:10D91000AD2007B0304C0040ADDEADDE70B50E4638
:10D920000446F9F749FD042811D1A4F5C0708028F8
:10D930000DD2A019A0F28110802808D2650200241F
:10D94000002E04D92846F6F727FA012801D0002036
:10D9500070BD641C05F50075B442F3D3012070BDA1
:10D9600070B50D460446F9F727FD04280AD1A4F541
:10D97000C070802806D260022946F6F7AFFA012867
:10D9800008BF70BD002070BD10B5074CFEF7A8FFA2
:10D99000012808BF10BD206800F095FE002818BFC0
:10D9A000F9F77BFDF2E700000C870010FA4A002827
:10D9B000916814BF41F0010021F0010090607047B0
:10D9C000F54B99680A0E120721F07F4142EA006088
:10D9D000084398607047F0488068C0F30360704760
:10D9E000ED488068000F7047EB4800697047EA48CF
:10D9F000006A7047E849012008627047E649002044
:10DA000008627047E44800787047002818BF01207A
:10DA1000E14908707047E048406A7047DE480021DD
:10DA20004162017070472DE9F04186B000270FF088
:10DA30009CFB0646A021D94811F04DFE0024254646
:10DA40004FF00308305D10F0800F18D0601C8DF887
:10DA500001008DF807508DF80080ADF804508DF866
:10DA60000850ADF802508DF806508DF809508DF829
:10DA70000E50355501276946C848F2F79AFD601CDB
:10DA8000C4B20A2CDED3C64CE07A68B1012F0BD1A8
:10DA90000021C248F2F74BFCE07C28B100231A4673
:10DAA00003210420F2F73AFC06B0BDE8F0410FF084
:10DAB000CCB92DE9F04387B040F20F31F9F716FEEB
:10DAC000002804BF07B0BDE8F08311F009FE11F093
:10DAD0000CFEF7F739FF5FEA00097CD1F3F79CFCF5
:10DAE000B048F4F748FF0120F4F738FFF3F7DEF908
:10DAF000AD4DA94EAD4F10F0010FC84613D0002018
:10DB0000F3F7DDF9C5F800802020F6F7A4F8A8485F
:10DB1000F6F7A7F82020F6F790F833202860386849
:10DB200090F81F012BE0F6F7BDFDA248F6F76FFE57
:10DB3000F6F756FEF6F77FFE41003868B0F80E2182
:10DB4000B1FBF2F1491CC1F34F01718090F8100153
:10DB500010F0FF0070700AD0F6F76DFE39684000D3
:10DB6000B1F80C11B0FBF1F0401CC0F34F010846B6
:10DB7000F6F7D1FD17202860386890F81E01F06094
:10DB8000F4F7A7FFF4F7ACFE002808BFF5F727F974
:10DB9000707838B1401E10F0FF00707004BF7088BC
:10DBA000F6F7B9FDB068C0F3036421460520F2F72B
:10DBB00097FBFEF795FE012807D0B068C0F303601D
:10DBC000A04208BFB9F1000F27D0F5F723FCC5F834
:10DBD0000080202000E017E0F6F73DF80020F6F77F
:10DBE00040F8F6F7E8FD40B1F6F7CDFDF6F703FE95
:10DBF0000020F6F70CFEF6F762FDF4F76AFFF4F783
:10DC000071FE0020F4F7B7FE11F06FFD11F072FD08
:10DC1000F9F7E1FE07B0BDE8F0836846F5F7A9FB28
:10DC200098B16846FFF784FBF9F7C6FB2146009AD6
:10DC300007F052FD684611F062FD814607F0C2FD13
:10DC4000F5F7E8FBF9F73FFCB3E73868D0F8B00028
:10DC500010F0704F02D0F9F720FCAAE7F9F73AFC70
:10DC6000A7E704283CBF4C49486070474A484068D1
:10DC7000704770B5054600240CF03DFA022801D02B
:10DC8000204670BD4C4800EB0510C1684248426B0D
:10DC900091421CBF012181630124F1E770B5054663
:10DCA000002404F01BFE70B10CF019FA08280AD009
:10DCB000414800EB0510C1683748426B91421CBFD8
:10DCC000012181630124204670BD3B4A014602EBDD
:10DCD00001110020CA6830494B6B9A4208BF704757
:10DCE00001208863704770B505460024F7F79AFE57
:10DCF00001280FD12848D0E90A1291420AD100F137
:10DD00003C0101EB0511426BC96891421CBF012126
:10DD100081630124204670BD2DE9F047234F03465F
:10DD200000243A6880002646D2F80011082B31BF43
:10DD300021FA00F0D2F80421203822FA00F000F095
:10DD40000F00DFF85480C1F303229042C8E90A02B1
:10DD50000FD001F00F01814270D1F7F763FE012867
:10DD60006CD1386890F8040100F00F00C8F8280062
:10DD700064E00020DFF84090C8F8380009EB041197
:10DD8000486808281AD23A688000D2F8002122FA9E
:10DD900000F000F00F051AE00086001078890010EE
:10DDA0006489001067500010104800400C87001074
:10DDB00091480010CB4800103C8600103A68800063
:10DDC0002038D2F8042122FA00F000F00F050F2DC0
:10DDD00004D0896820468847012807D0641C042C99
:10DDE000CCD3D8F8380001280CD103E02646C8F877
:10DDF0002850F6E709EB0610C068C8F83400002088
:10DE0000F7F7FAFDD8F83010D8F82800814215D07D
:10DE1000C8F83000F3F747F80446F3F747F8D8F8A6
:10DE20002820D8F80410002341EA022141EA0441E5
:10DE300041EA00628921072003F07AFBD8F8280024
:10DE4000BDE8F0872DE9F04139480068B0F91611B6
:10DE5000B0F9140111F026FCF2F799FC0120F7F754
:10DE6000CBFD00200CF044F90FF053F90420FFF72C
:10DE700053FFF7F7A6FD002004F091FE2D4D00267C
:10DE800001202E616E61C5E906606E6011F03CFCF8
:10DE9000F9F792FA05282AD1A868010FC0F30364A4
:10DEA000A14202D02E616E61AE612046FFF734FFC1
:10DEB00007462146052003F0FFFB7CB3022C29D046
:10DEC000042C30D0A8680E2C4FEA106120F07F405F
:10DED0004FEA017118BF41F000710843A860FEF7D6
:10DEE000FFFC012803D0F9F767FA0528D4D00EF01B
:10DEF000ACFFF7F780FD0FF015F90F48416821F4EA
:10DF00000071416000202E63F7F786FD03206860F2
:10DF1000BDE8F0813846FFF7CCFDE0E7FFE7384683
:10DF200011F0F7FBDBE7384604F0ADFFD7E7000060
:10DF30000C87001000860010001000407047002879
:10DF400008BF704780220146014811F047BB704767
:10DF5000E4C30010704705283CBFFE4908707047B5
:10DF60000020FC4988604860FB48006890F8CD00BC
:10DF7000052838BF087070470020F6494860704790
:10DF8000F4480078704770B5F34D0024286890F885
:10DF9000B80010F0020F0BD0F9F70EFA022807D1E3
:10DFA000EC482968007801EB8000B0F8D00084B21A
:10DFB000204670BD70B5E84D4FF48054286890F845
:10DFC000B80010F0020F0DD0F9F7F6F9022809D1C8
:10DFD000E0482968007801EB8000D0F8D000000C00
:10DFE000C0F31304204670BDDA488078002818BFBB
:10DFF000012070472DE9F041F9F7DEF9022803D13D
:10E0000004F068FB022803D04FF48050BDE8F08193
:10E010004FF480552E4604F025FCDFF83C8304467F
:10E02000CC4FD8F8000090F8B81011F0010F0CD0C8
:10E03000B0F8C200B9684042814206DC2CB1002031
:10E04000641EB860204604F010FCD8F8001091F867
:10E05000B80010F0040F18BF002C0AD0B1F8C800A7
:10E06000621E9040B1F8CA20824238BF1046C0F309
:10E070001306D1F8F00010F0020F1CBFB978002988
:10E0800002D0000CC0F31305B54298BF35462846B0
:10E09000BDE8F0812DE9F04FDFF8BCA287B0DAF8D7
:10E0A000001091F8B82012F0020F0DD0A94A91F893
:10E0B000CC90DFF8A8B21778002809DB484503D2D6
:10E0C000B84218BF064643D107B00020BDE8F08F24
:10E0D0003E464FF0FF38F4F705FCF5F729FC002524
:10E0E000B9F1000F34D9DAF80000002400EB850004
:10E0F000B0F8D00081B22046F3F795FAF4F76FFE3E
:10E100006846F5F736F9002866D0029878B10146DE
:10E1100093489BF8002000785043421E07D331F902
:10E12000020B0028B8BF40420444521EF7D2F5F754
:10E1300071F9F4F7D7FB002322469221072003F060
:10E14000F7F9A04584BF2E46A0466D1C4D45CAD3A5
:10E15000B74244D0052E3CBF7E490E70DAF800006D
:10E16000B0F8CE1039B300EB870200EB8600B2F8AE
:10E17000D020B0F8D00092B280B2801A484340F369
:10E180000F34F7F7A9F8774B9BF80020002193F89C
:10E1900000C002FB0CF2002A0DD930F811202244F5
:10E1A00020F811209BF8002093F800C0491C02FBC6
:10E1B0000CF28A42F1D84FF4800004F0A3FCDAF8A4
:10E1C0000000002300EB86008021B0F8D00082B26E
:10E1D000072003F0ADF909E0F9F75FF990E704F0E3
:10E1E00041FB03283CBF401C04F03FFB012007B06B
:10E1F000BDE8F08F584857490068B0F8C200424265
:10E2000088688242BCBF401E886070472DE9F04F8D
:10E2100093B093460E4604464FF0000A04F022FBEA
:10E22000DFF834814B4F0500D14610D111F076FA5A
:10E23000D8F80010B1F8C410884208D30120C7F8FC
:10E24000089004F012FB13B00120BDE8F08F002EFF
:10E250001FDDB8680028B8BFC7F8089007DBD8F8FA
:10E260000010B1F8C0108842BCBF401CB860D8F89C
:10E270000000B968B0F8C000884215DC032D13D245
:10E28000681CC7F8089004F0F0FA13B00120BDE84C
:10E29000F08F09D1D8F80000B0F8C2004142B86848
:10E2A0008842C4BF401EB860B87850B1D8F80000AA
:10E2B00090F8F00010F0040F1EBF002013B0BDE86E
:10E2C000F08FD8F80000B0F9BE108C420EDD7968EE
:10E2D00021447960B0F8BA00884210DC4FF0FF307A
:10E2E000C7F80490FFF7D6FE824608E07868002859
:10E2F00005DD002CD4BF01212146401A7860DFF8EB
:10E30000689099F8000007283BD1184859460078D2
:10E310004200684611F071F9ADF80040ADF80260B6
:10E32000ADF804503889ADF80600B888ADF808009B
:10E33000D8F80000B0F8BE10ADF80A10B0F8C01060
:10E34000ADF80C10B0F8BA10ADF80E10B0F8C2006D
:10E350000EE00000F48600100C87001041850010CC
:10E360004585001042850010C185001048850010C9
:10E37000ADF8100099F80000072804BF6846FEF7C2
:10E38000BEFC504613B0BDE8F08F474810B500689A
:10E39000D0F8F00010F4807F06D0C0F303300121E4
:10E3A00001FA00F0F5F77AFE4049002048708870C5
:10E3B00010BD70B53D4D0024A878002814BF01267B
:10E3C0000026687828B904F05CFA002808BF00210C
:10E3D00000D001218E4227D00A1C18BF0122AA704A
:10E3E00031480068D0F8F03013F0040F0ED021B19E
:10E3F000C3F30310052808D206E00021A960696074
:10E4000090F8CD00052800D22870012413F0020FE7
:10E4100018BF0124002A18BF0122002382210720EF
:10E4200003F086F8F1F78CFF204670BD2DE9F0412E
:10E430001D4800270068D0F8F01011F4807F30D01C
:10E440001A4E7078051C18BF0125C1F30330184A15
:10E450005268012303FA00F0024011F4007F0AD051
:10E4600092B10BF03CFE042818BF08280AD0022005
:10E470000BF030FE06E03AB10BF031FE042818BF75
:10E480000828F4D1012403E0002401200BF022FE2F
:10E49000A54206D0201C18BF01207070FFF789FF2D
:10E4A00007463846BDE8F0810C870010F48600105E
:10E4B000001000407148007870477048406800F5CF
:10E4C000407070476D48406800F58070704770B5C7
:10E4D0006A4C4FF448306A4A60600168914204BF58
:10E4E0004168B1F50C7F3BD18168B1F5464F37D813
:10E4F000644AC568954223D04FF0000C034662463B
:10E50000BCEB910F0AD253F8046B521C86EA0C0C38
:10E51000B2EB910FF7D3BCF1000F21D1026A7AB1AF
:10E520004FF0000C03466246BCEB910F06D253F845
:10E53000046B521CB444B2EB910FF8D365450FD174
:10E54000012500F5807000F0BEF848B1606800F564
:10E55000407000F0C7F800281EBF2570012070BD74
:10E56000002070BD4549002008704FF44830F5F791
:10E5700013BC4248017841B14068414A0168914268
:10E5800002BF4168B1F50C7F7047002070473B4BDC
:10E590005B6803F580731844F5F7F4BC374B5B6890
:10E5A00003F540731844F5F7EDBC3448406800F5B6
:10E5B000A0607047314B5B6803F5A0631844F5F722
:10E5C000E1BC2E484068006970472C4949680A69D7
:10E5D00082429CBF0020704700EB400001EB00101E
:10E5E00000F5C0607047254A526802EB8000436A1C
:10E5F000406E1A4400FB0120704720498860704734
:10E600001E48806870472DE9F0011C4B002201274D
:10E61000D3E901469046831893F92030002B12DB92
:10E6200007FA02FC1CEA060F0DD002F0FF0C04EB07
:10E630008C0CDCF82450DCF864C0254403FB0C533C
:10E6400041F8223001E041F82280521C102AE2D326
:10E65000BDE8F00170470029B8BF704730B4944658
:10E66000064A526802EB8000446A406E224401FB75
:10E67000002030BC1A466146F5F784BC00870010C4
:10E6800054465053EFBEADDE10B5FFF720FFB0B1DA
:10E69000FFF713FF01464FF4B672174810F09EFFC4
:10E6A000FFF710FF154C01464FF4E872206810F098
:10E6B00095FF2068C06BBDE8104004F057B80220F9
:10E6C000F8F751FFE1E758B10D4A0168914207D1CF
:10E6D000406820F00F00B0F5407F04BF0120704774
:10E6E0000020704730B1006820F00F00802804BF80
:10E6F0000120704700207047A83001100C870010DF
:10E7000041505352FE4948607047FD488068704749
:10E71000FB4948707047FA48407870470200F94852
:10E720004FF008010068438A008A03FB00101CBFF9
:10E73000C01C20F0030070472DE9F04104460D464F
:10E740000846F8F733FE78B1012606FA04F010F017
:10E75000CC0F18BF002C07D0032C05D8E9494FF483
:10E76000403201200B6802E00020BDE8F081A042A9
:10E7700013D006FA00F111F0CC0F0BD0598A1F8A82
:10E780004FF0080C01FB07C1C91C21F0030C0CEB76
:10E790004C010A44401C0328E9D90120A8420CD0AE
:10E7A000B3F812C01C8A08210CFB0411C91C21F00B
:10E7B0000301401C0A440328F0D91046BDE8F0814B
:10E7C0002DE9F04F0E4690F821A090F8209000F12E
:10E7D0005005ADF20C4D1746012411463046FFF7A7
:10E7E000ABFFA11E012E08BFC74906D0022E08BFED
:10E7F000C64902D0032E08BFC5494FF0000830B10A
:10E8000002688A4204BF4068CDE9002001D0CDE90A
:10E810000018C048022E01680CBFB1F98A00B1F996
:10E820003A0086460CBFB1F98820B1F938209346EA
:10E8300000230AFB09FCBCF1000F0ED935F91310B7
:10E840007145D8BF8B4505DC9142C8BF0A4681425D
:10E85000B8BF08465B1C9C45F0D8104400EBD07054
:10E8600042100023BCF1000F88BFE94616D935F9E4
:10E870001300801A00EBD07041107F29C8BF7F21A0
:10E8800005DC11F1800FB8BF6FF07F0100DA0024C2
:10E8900009EB03005B1C01729C45E8D88DF804402D
:10E8A0009DF80500FF283CBF401C8DF80500ADF821
:10E8B00006206C4639463046FFF73EFF78B1914955
:10E8C000082209684B8A098A03FB01222146F5F7D1
:10E8D00059FB01280CBF4FF001084FF000084046DB
:10E8E0000DF20C4DBDE8F08F2DE9F0479846154626
:10E8F0000E468146F8F757FDF8F758FD002808BF87
:10E90000BDE8F0877E4F844C3878814588BFBDE8EC
:10E91000F0870CD287F800904FF00000B8704FF0ED
:10E92000FF024FF014017C4810F07BFE19E097F8CD
:10E9300002C0BCF1050F28BFBDE8F087BCF1000F95
:10E9400018BF00200DDD14F82010B14206D104EBF1
:10E9500080014978A94208BFBDE8F087401C6045A6
:10E96000F1DBB87804EB800104F820604D70A1F869
:10E970000280401CB870BDE8F08770B505461646A9
:10E980000C460846F8F712FD00281CBF681E032835
:10E9900032BF022E002070BD04EBC400400105EB25
:10E9A000450100EB411006EB460100EB011000F5BC
:10E9B000403000F5686070BD2DE9F04F97B04FF022
:10E9C000000816460D460746CDF83080FF2230215C
:10E9D0006846CDF8348010F024FEDFF840A14FF4F3
:10E9E0007F30CDF800A00168880A424211EB8222F4
:10E9F00018BF401C404201EB8000C01C20F0030007
:10EA000000F500504649428A437C52BA007C63F3C9
:10EA10001F4242EA006001900888A1F1040940BA4F
:10EA2000ADF80A003869039099F800008DF81800D5
:10EA3000002231462846FFF7A0FF04460122314656
:10EA40002846FFF79AFF4FF0010C012D04D0022D4C
:10EA500018BF032D40D082E00022114624B3236862
:10EA6000534521D1237A647A28B1D0F800B0D34538
:10EA700004BF027A417A181902EB010A504583BF9C
:10EA8000ADF830C0ADF83430ADF83640ADF8308078
:10EA90009CBFADF83420ADF83610BDF83400BDF899
:10EAA00036100844ADF83200BDF83400BDF8361019
:10EAB0009DF81820C0B28DF80800C9B20CFA02F215
:10EAC0008DF8091012F00E0F19BF401C8DF80800C8
:10EAD000481C8DF8090042E0002134B322685245F9
:10EAE00023D1227A18B10368534508BF017A8A42BC
:10EAF00086BFADF830C0ADF83220ADF8308011E0FF
:10EB0000108700100C8700104654525946544D325D
:10EB100046544D332C870010D8F000104646485319
:10EB20001487001098BFADF83210022D18BF032DC6
:10EB300015D1387C10F0300004BF17B0BDE8F08F5D
:10EB4000BDF832003146401C8DF808002846FFF71A
:10EB5000F3FD00280CBF404640798DF80900FE48BF
:10EB60000DF1380A6B46B0E816108AE8161090E8E6
:10EB7000071012AC84E807109DF81800082813D27B
:10EB80000EA951F82000B0F1FF3F0DD007EBC000F7
:10EB9000D0E90A10CDE9041099F80200EF4982008B
:10EBA00003F11C0010F029FDBDF830106C46CAB20C
:10EBB00031462846FFF7E1FE48B130222146F5F7FD
:10EBC000E1F901280CBF4FF001084FF00008404662
:10EBD00017B0BDE8F08F0146012200208A4012F0F4
:10EBE000CC0F08BF7047082928BF7047DFE801F045
:10EBF0000B0404040B0B040C0821D9480068428A5A
:10EC0000008A02FB001070474FF490707047012398
:10EC100010B50022834013F0CC0F14D0082812D274
:10EC2000DFE800F01104040411110D07FFF784FD63
:10EC300003E000220120FFF7A0FE024603E04FF4AC
:10EC4000443000EB8122104610BD2DE9F04106460C
:10EC50000127F8F7A8FB8046F8F7A8FB002808BFB3
:10EC6000BDE8F081BF4D686810F4807F18BF0224B2
:10EC70000DD00120A04010F0CC0F05D04246214617
:10EC80003046FFF79DFD0746306978B90BE010F478
:10EC9000007F18BF0324ECD110F0070018BF012437
:10ECA000E7D1BDE8F0812878112805D242462146F7
:10ECB0003046FFF781FE07463846BDE8F081A94996
:10ECC000C8607047A74810B4C068002808BF4FF458
:10ECD0007C30A54A016891421CD14168B1F5007FA2
:10ECE00018D3836800228446B3F5056F88BF4FF4BC
:10ECF00005630021B1EB930F24BF10BC70475CF893
:10ED00002140491C2244B1EB930FF8D3002A04BFE1
:10ED100010BC7047002010BC704770B50022C26064
:10ED2000D0F808C0012113460446BCF5056F88BF22
:10ED30004FF4056C0022B2EB9C0F06D254F822501F
:10ED4000521C2B44B2EB9C0FF8D35A42C260854A46
:10ED5000127912F0800F07D14FF47C304FF4056226
:10ED60002146F5F70FF9014601290CBF01200020CB
:10ED700070BDFF2270B50025044605614FF40061A7
:10ED8000503010F04EFCA584E584E562A562656311
:10ED90002563E563A56365642564E5640120A564D6
:10EDA00070BD2DE9F0414FF47C3104466E4E086889
:10EDB000B04218D14868B0F5007F14D38A680023A8
:10EDC0000D46B2F5056F94BF94464FF4056C0020D4
:10EDD000B0EB9C0F26D255F82070401C3B44B0EBA2
:10EDE0009C0FF8D3F3B1FF224FF40561204610F0D9
:10EDF00018FC4FF40870C4E900604FF40560A0608F
:10EE00000020E06084F8200084F8210084F82200CB
:10EE100084F8230020616061A061E0612046FFF773
:10EE2000A8FF07E0B2F5056F88BF4FF405622046E2
:10EE300010F0D4FB0120BDE8F08170B402684FF4FB
:10EE400008715160016801F1500291F821C091F8F8
:10EE500020300CFB03F102EB41010022BCF1000F5A
:10EE600008D900EB4204521CB4F8DE4021F8024BF2
:10EE70009445F6D80022002B08D900EB4204521C1E
:10EE8000B4F8064121F8024B9342F6D80022BCF1B7
:10EE9000000F08D900EB4204521CB4F8644021F87A
:10EEA000024B9445F6D80022002B08D900EB42040F
:10EEB000521CB4F88C4021F8024B9342F6D8B0F8BB
:10EEC000DA2021F8022BB0F8DC2021F8022BB0F870
:10EED000D82021F8022B00240022BCF1000F0ED90B
:10EEE00004EB440505EB041500EB850505EB420634
:10EEF000521CB6F8526121F8026B6245F6D300222B
:10EF0000002B0ED904EB440505EB041500EB850539
:10EF100005EB4206521CB6F8826221F8026B9A4257
:10EF2000F6D3641C042CD7D370BC70472DE9F74F7F
:10EF300088B000250A992C462E460968049101F1F3
:10EF400050030999002984BF0849D1F800802AD9C3
:10EF5000002200280CE00000F04C0200D8F0001065
:10EF60000C8700101087001053454C462C8700106A
:10EF700088BFB8F93A700DD933F9021B0029B4BF24
:10EF8000C1F1000C8C46BC45BCBF0D44641C521C36
:10EF90008242F1D30999761C8E42D9D3002CC8BF86
:10EFA00095FBF4FA08DC4908414301EB500204994F
:10EFB00001EB4201B1F950A00021029101910499A5
:10EFC00050310091002103910999002969D9009ECF
:10EFD0004FF00109FE4906964FF0000B09685F46A5
:10EFE000D846B1F81CE091F82410CDF814B0079180
:10EFF000002829D9B6F900204FF0000C0699934457
:10F00000634600280DD9B1F90040A51A48BF151B69
:10F010007545B8BF0CF1010C01EB49015B1C834243
:10F02000F1D307998C4503D305997F1C11440591B1
:10F0300008F1010806EB49068045DBD3002FC4BF69
:10F04000059991FBF7F101DC9BFBF0F1039B0A9A18
:10F0500009B202EB4302A2F86410DD4A1268538B36
:10F06000AAEB0303994209DD128B52448A4205DD63
:10F07000019A114401910299491C02910099099A3F
:10F0800001EB400100910399491C039191429ED3E9
:10F090000299002905DDDDE9011291FBF2F10191F0
:10F0A00002E05146CDF804A00A9AA2F8DA10002135
:10F0B000029103910499503100910021049100289C
:10F0C00065D9C349009F069709684FF0000B099E58
:10F0D000B1F820E091F82510D846D946CDF814B003
:10F0E0000791002E2BD9B7F900204FF0000C06999C
:10F0F00093446346002E0DD9B1F90040A51A48BFCC
:10F10000151B7545B8BF0CF1010C01EB40015B1CF0
:10F11000B342F1D307998C4504D3059908F101084E
:10F120001144059109F1010907EB4007B145DAD314
:10F13000B8F1000FC4BF059991FBF8F101DC9BFB0E
:10F14000F6F1049B0A9A09B202EB4302A2F88C1072
:10F150009F4A1268538BAAEB0303994209DD128B75
:10F1600052448A4205DD039A114403910299491CD5
:10F1700002910099891C00910499491C04918142D3
:10F180009FD302980028C4BF039991FBF0FA0A9814
:10F19000A0F8DCA001980A99504400B200EBD070AE
:10F1A0004010A1F8D8000BB0BDE8F08F2DE9F04F6A
:10F1B000146887B015460E468046A1F12009202923
:10F1C00028BF4FF0FF3B05D24FF0010000FA06F0D8
:10F1D000A0F1010B31BF0020012000FA09F0401E10
:10F1E0000290B8F1200F3DBF012000FA08F0401E48
:10F1F0004FF0FF3038BF002207D3A8F120024FF0B4
:10F20000010101FA02F1A1F10102C6F1200A202E4A
:10F2100034BF20FA0AF100FA09F1B2401143B040BC
:10F22000CDE90001206920F4FE6020616948406852
:10F2300010F0010F79D010F4807F05D02A463146B6
:10F24000404601F04DFA8AE010F4007F2A4631462C
:10F25000404602D001F05CFC81E001F021F9002081
:10F26000A86107466861B8F1000F22D905EB470095
:10F27000B0F98C000028B8BF404200B25449096878
:10F28000B1F93810814211DD7A0905EB820C07F0E3
:10F290001F0301219940DCF8142083B21143CCF8FC
:10F2A0001410FAB2FF210420FFF71EFB7F1C474514
:10F2B000DCD30027B8F1010F1CBFA8F101000390B7
:10F2C0004DD005EB4700B0F98E30B0F98C20991A7B
:10F2D00048BFD11A09B2DFF8F8C0DCF800C0BCF9A9
:10F2E00032C08C4537DAB5F9DC10B2EB010C48BFFF
:10F2F000A1EB020C0FFA8CFC5A1A48BFCA1A11B2C1
:10F300008C4513DB7A0905EB820107F01F0C012203
:10F310004B6902FA0CF21A434A61B0F88C30FAB227
:10F32000FF210420FFF7E0FA15E02BE0791C4B09E0
:10F3300005EB830E01F01F0C0122DEF8143002FAF7
:10F340000CF21A43CEF81420B0F88E30CAB2FF2166
:10F350000420FFF7C9FA03987F1C8742B1D369697B
:10F36000E869B14008432063A969286AB1400843AD
:10F3700060636969202E34BF21FA0AF101FA09F1AC
:10F38000084360631348007910F0040F00F0F58122
:10F39000002028630746E862002E27D90C4905EBB8
:10F3A00047000968B0F95201B1F95C20824203DCE0
:10F3B000B1F95E10814216DA7A0905EB820C07F08A
:10F3C0001F0301219940DCF82C2083B2114303E094
:10F3D0002C87001010870010CCF82C10F9B2FF22F7
:10F3E0000220FFF781FA7F1CB742D7D30020A86222
:10F3F00007466862B8F1000F22D905EB4700B0F963
:10F400008202FE490968B1F95C20824203DCB1F94D
:10F410005E10814211DA7A0905EB820C07F01F03B6
:10F4200001219940DCF8242083B21143CCF8241048
:10F43000FAB2FF210220FFF757FA7F1C4745DCD3C1
:10F44000002028640746E863002E2FD9EB4905EB1E
:10F4500047000968B0F99E01B1F960208242DCBF23
:10F46000B1F96220904210DD7A0905EB820C07F0B9
:10F470001F0301219940DCF83C2083B21143CCF8F2
:10F480003C10FF22F9B201200BE0B1F96C2082425E
:10F49000DCBFB1F96E10884205DD83B2F9B2FF22FC
:10F4A0001020FFF721FA7F1CB742CFD30020A863BA
:10F4B00007466863B8F1000F2FD9D04905EB470024
:10F4C0000968B0F9CE02B1F960208242DCBFB1F91F
:10F4D0006220904210DD7A0905EB820C07F01F03D1
:10F4E00001219940DCF8342083B21143CCF8341068
:10F4F000FF21FAB201200BE0B1F96C208242DCBF9F
:10F50000B1F96E10884205DD83B2FAB2FF211020F6
:10F51000FFF7EAF97F1C4745CFD300202865E86450
:10F52000A86407466864002E22D9B44905EB470059
:10F530000968B0F9EA01B1F96420824203DCB1F94B
:10F540006610814211DA7A0905EB820C07F01F037D
:10F5500001219940DCF84C2083B21143CCF84C10C7
:10F56000F9B2FF220320FFF7BFF97F1CB742DCD3BB
:10F570000027B8F1000F22D9A04905EB4700096820
:10F58000B0F91A03B1F96420824203DCB1F96610C4
:10F59000814211DA7A0905EB820C07F01F03012181
:10F5A0009940DCF8442083B21143CCF84410FAB2FD
:10F5B000FF210320FFF798F97F1C4745DCD3696AD8
:10F5C000E86AB14040EA0107A763A96A286BB14025
:10F5D0000843E063696A202E34BF21FA0AF101FA78
:10F5E00009F141EA0000E0630590696BE86B01FAFC
:10F5F00006F140EA01022264A96B286C01FA06F1C7
:10F6000040EA01006064696B34BF21FA0AF101FA33
:10F6100009F141EA000161646B6CE86C03FA06F3DE
:10F6200040EA0300A0640390AB6C286D03FA06F374
:10F6300040EA0300E0646B6C34BF23FA0AF303FA78
:10F6400009F343EA0000E0640690059832EA0705F2
:10F6500021EA000C47EA05022564049240EA0C09FD
:10F6600006EB0801C4F844C008BFBCF1000F46D047
:10F6700000231A461846002988BF4FF001083ED9DA
:10F680004FEA501A04EB8A0A00F01F0EDAF840A085
:10F6900008FA0EFE1AEA0E0F03D0864294BF521CDF
:10F6A0005B1C401C8142EBD8012B10D105EA0B00FA
:10F6B0003843A06302980CEA000305981843E063FE
:10F6C00025EA0B00206402982CEA00006064012AFD
:10F6D00015D1206C009A00EA0203A26B1A43A263C0
:10F6E000626C019BD4F83CC0134043EA0C03E36313
:10F6F000009B98432064019822EA00006064DDE9E1
:10F7000003208243A264049840EA0205069820EA96
:10F71000090049EA0007E06408BF002822D000235E
:10F720001A461846002988BF4FF0010C17D94FEA36
:10F73000501804EB880800F01F09D8F848800CFA2C
:10F7400009F918EA090F03D0864294BF521C5B1CCA
:10F75000401C8142EBD8002B18BF002A02D10020A8
:10F76000A064E0642648007910F0010F05D0206BFA
:10F77000A8432063606BB8436063206B0099084224
:10F7800003D1626B01990A4203D0216941F0100153
:10F79000216110EA0B0F03D1616B0298014203D083
:10F7A000206940F020002061A06B0099084203D13D
:10F7B000E26B01990A4203D0216941F040012161C5
:10F7C00010EA0B0F03D1E16B0298014203D02069CC
:10F7D00040F080002061206C0099084203D1626CE7
:10F7E00001990A4203D0216941F48071216110EA34
:10F7F0000B0F08D1616C0298014203E02C870010C6
:10F800001087001003D0206940F400702061A06CC4
:10F81000002804BFE06C002803D0206940F4806019
:10F82000206107B00120BDE8F08F2DE9F04FCBB08B
:10F8300017460D460446F3F755F80120F1F7DDF8B9
:10F8400006461120F1F7D9F8304314BF01200220F9
:10F850008DF8180014BF112012208DF81900F2F74E
:10F86000CBF838B19DF818009DF819108DF81810D4
:10F870008DF819009DF81800F1F7BFF8002818BF9F
:10F88000284604909DF81900F1F7B7F8002818BF32
:10F8900020460590F3F76AFB0022002D88BF24A9BB
:10F8A0000BD98356142BA8BF143B02DA0A2BA8BF2E
:10F8B00012338B54521CAA42F3D3F3F759FB0021A5
:10F8C000002C88BF24AA07D9435C02EB010C491C19
:10F8D0008CF826308C42F7D8F3F71AFA0390FE48DA
:10F8E0000DF1180A007910F0200F55D007F1DE0055
:10F8F000009028300025E9460DF1100B01905BF8CF
:10F9000025601AF80500F3F794FF0024002E1AD999
:10F9100005EB450000EB051024A901EB400818F9A0
:10F920000420262A28BF002006D21AF8050000214C
:10F93000F2F758FEF3F783FF59F8251021F8140069
:10F94000641CB442EBD36D1C022DD8D3E34C267853
:10F950001D2E21D100210A460DF11C085BF8225012
:10F960000020002D88BF59F822C007D93CF810307C
:10F9700028F81130401C491C8542F7D8521C022A35
:10F98000ECD31D2E08D14046FDF791FB20781D28B1
:10F9900004BF07A8FDF78BFBCF4D287910F00C0FA3
:10F9A00000F0AF83039800F0F000F3F768F89DF8DB
:10F9B0001800F1F724FE07909DF81800F1F78EFE6D
:10F9C000002437901AF80400F2F754FD44A941F8D6
:10F9D00024001AF80400F1F7BEFE0EA941F8240035
:10F9E0001AF80400F2F70BF820A941F824001AF8DD
:10F9F0000400F2F73CF822A941F824001AF80400A8
:10FA0000F1F73AF846A918AA41F824001CA81AA947
:10FA100002EB840200EB840001EB84010092CDE94B
:10FA2000011016A800EB840314A800EB840212A8AE
:10FA300000EB84011AF80400F2F7FBFA1AF804004C
:10FA4000F2F729FC1EA941F824001AF80400F2F785
:10FA500061FD10A941F82400641C022CB2D3A04E11
:10FA60003068B0F848109DF81800F1F7DCFD00246C
:10FA700000211AF80400F2F7E3FC994E306890F880
:10FA80004A101AF80400F1F77AFE1AF8040000216F
:10FA9000F1F7CFFF1AF804000021F2F702F81AF884
:10FAA00004000121F0F7CEFF3068B0F84C101AF8CE
:10FAB0000400F2F77AFB1AF804000021F2F7F2FCD6
:10FAC000641C022CD4D384484FF00009007910F054
:10FAD000040F00F0DD813446206890F84B3090F838
:10FAE0005920B0F850100091CDE9012390F84F3023
:10FAF00090F84E2090F858109DF81800F2F7DDF8B5
:10FB0000206890F84B3090F85920B0F850100091D0
:10FB1000CDE9012390F84F3090F84E2090F858101E
:10FB20009DF81900F2F7C9F89DF818000021F2F7C6
:10FB3000B9FC9DF819000021F2F7B4FC3AADF3F7D7
:10FB40004EF9FCF7CDFE012806D02846F3F711FC4C
:10FB500000287DD0F3F75EFCF2F7C4FE3E99002248
:10FB600004AD002055F82230002B0ED902EB420CD8
:10FB70000CEB021C07EB0C1C31F8026B0CEB400881
:10FB8000401CA8F852618342F6D8521C022AE8D3DE
:10FB90005448D0E90010CDE90C109DF81800F0F79A
:10FBA0002CFF48909DF81900F0F727FF49909DF829
:10FBB000180040A9F1F780FE9DF8190042A9F1F75D
:10FBC0007BFE9DF8180008A9F1F7E8FE9DF81900E2
:10FBD0000AA9F1F7E3FE424C206890F84B3090F808
:10FBE0005920B0F852100091CDE9012390F84F3020
:10FBF00090F84E2090F858109DF81800F2F75DF834
:10FC0000206890F84B3090F85920B0F852100091CD
:10FC1000CDE9012390F84F3090F84E2090F858101D
:10FC20009DF81900F2F749F89DF818000CA9F1F7B2
:10FC300093FE9DF819000CA9F1F78EFE00249DF8A3
:10FC400018000021F2F72EFC9DF81900002100E0B9
:10FC500017E0F2F727FC9DF818000021F0F7B3FE3B
:10FC60009DF819000021F0F7AEFE1AF804000121FA
:10FC7000F0F7A9FE1AF80400C0F3011001280AD118
:10FC800002E0F7F70AFC5CE784F0010001211AF8B2
:10FC90000000F0F798FECDF8E090CDF8E4909DF8E4
:10FCA000180038A9F1F7E8FD9DF8190038A9F1F717
:10FCB000E3FD04A8002150F824801AF80400F2F7AC
:10FCC00037FD00250190B8F1000F55D904EB440031
:10FCD00024A900EB041007E010870010C78500106E
:10FCE0002C870010E84C020001EB400107EB001BE1
:10FCF0000091009838AA00214657CDF8E090CDF841
:10FD0000E4901AF80400F2F730FC202E06DBA6F18E
:10FD1000200101208840CDE9389003E00120B04067
:10FD2000CDE938091AF8040038A9F1F7A5FD38988B
:10FD300038AAC043389039980921C04339901AF83D
:10FD40000400F2F712FC3AAEF3F749F8FCF7C8FDED
:10FD5000012806D03046F3F70CFB00287ED0F3F7DD
:10FD600059FBF2F7BFFD019800880BEB45016D1CB4
:10FD7000A1F89E014545BCD3CDF8E090CDF8E490C4
:10FD80001AF8040038AA0021F2F7EFFB641C022CD9
:10FD9000FFF455AF9DF8180008A9F1F7DDFD9DF8B7
:10FDA00019000AA9F1F7D8FD9DF818004899F0F755
:10FDB0000AFE9DF819004999F0F705FE9DF8180014
:10FDC00040A9F1F759FD9DF8190042A9F1F754FD3A
:10FDD000FE4C206890F84B3090F85920B0F8541041
:10FDE0000091CDE9012390F84F3090F84E2090F823
:10FDF00058109DF81800F1F760FF206890F84B301C
:10FE000090F85920B0F854100091CDE9012390F8F2
:10FE10004F3090F84E2090F858109DF81900F1F7E7
:10FE20004CFF9DF818000121F2F73CFB9DF81900EA
:10FE30000121F2F737FB3AACF2F7D1FFFCF750FDA6
:10FE4000012806D02046F3F794FA00287DD0F3F776
:10FE5000E1FAF2F747FD002204AC00E081E03E99B0
:10FE600054F822C00020BCF1000F0ED902EB42036F
:10FE700003EB021307EB031331F8025B03EB4006BD
:10FE8000401CA6F8EA518445F6D8521C022AE7D352
:10FE9000CF48007910F0080F7ED0CC4C206890F845
:10FEA0004B3090F85920B0F856100091CDE901235D
:10FEB00090F84F3090F84E2090F858109DF81800A8
:10FEC000F1F7FBFE206890F84B3090F85920B0F81D
:10FED00056100091CDE9012390F84F3090F84E2054
:10FEE00090F858109DF81900F1F7E7FE00210DF188
:10FEF000100C00205CF82120002A0CD901EB4103F2
:10FF000003EB011307EB031303EB4005401CA5F8BB
:10FF100036928242F8D8491C0229EAD3206800258B
:10FF200090F86800B5EB400F36DA206890F868006A
:10FF3000A842D4BF012100219DF81800F2F7B2FABF
:10FF4000206890F86800A84200E00DE0D4BF0121CD
:10FF500000219DF81900F2F7A5FA3AAEF2F73FFF3B
:10FF600005E0F7F79AFAF1E6F7F797FA66E7FCF794
:10FF7000B7FC012805D03046F3F7FBF9D8B3F3F707
:10FF800049FAF2F7AFFC3E994FF0000904AB0022AA
:10FF9000104653F8296000E058E0002E05D931F9E9
:10FFA0001030401C1A448642F9D8B2FBF6F2701E9B
:10FFB0003DD009EB490303EB091307EB031B31F9B0
:10FFC000103001EB400C3CF9028CB3EB080348BF46
:10FFD0005B4231F91080B8EB020831F910804CBF58
:10FFE000A2EB0808A8EB02083CF902EC3CF902CCB1
:10FFF000BEEB020E00E00FE04CBFA2EB0C0CACEB32
:020000021000EC
:10000000020CE0450BEB400C09DDBCF936824345A0
:10001000C8BFACF8363208E0F7F73FFAA7E7BCF9FB
:1000200034829845B8BFACF83432401EC7D109F1CC
:10003000010901EB4601B9F1020FA7D320686D1C3D
:1000400090F86800B5EB400FFFF66FAF9DF8180011
:100050000799F1F7E8FA9DF818003799F1F74DFB89
:1000600000241CAD1EAE20AF0DF188080DF5887977
:100070000DF58C7B59F824101AF80400F2F7E0F91A
:100080000EA850F824101AF80400F1F778FB57F87E
:1000900024101AF80400F1F7CCFC58F824101AF8D0
:1000A0000400F1F7FEFC5BF824101AF80400F0F7E6
:1000B000C9FC1AA918A851F8241055F8242050F8A2
:1000C0002400CDE9000116A8029250F8243014A8AB
:1000D00050F8242012A850F824101AF80400F1F760
:1000E000ECFD56F824101AF80400F2F75EF810A898
:1000F00050F824101AF80400F2F7D4F9641C022C0A
:10010000B8D30398F2F7BBFC4BB0BDE8F08F304892
:10011000012181601121017000218170FDF7EFBA8A
:100120002B490020886070472DE9F04FDFF8A0A030
:10013000ADF56F7D01271120CAF808704FF0000857
:100140008AF800008AF80280FDF7D9FADAF804008C
:100150004FF4407131EA000008BF002600F07C81B6
:100160001D20FCF7F5FCED901D20FCF786FFEE90BE
:100170004FF46D716846DAF80C400FF034FA0094D1
:10018000BAF8040010F4804F1CBF2046FEF7F1FDC2
:100190006A46009890F8203090F821C050300CFB4F
:1001A00003F100EB41000021BCF1000F08D902EB84
:1001B000410630F8025B491CA6F8DE508C45F6D8A3
:1001C0000021002B0DD930F8025B03E02C870010D2
:1001D0001087001002EB4106491CA6F806518B421D
:1001E000F1D80021BCF1000F08D902EB410630F82C
:1001F000025B491CA6F864508C45F6D80021002B00
:1002000008D902EB410630F8025B491CA6F88C5075
:100210008B42F6D830F8021BA2F8DA1030F8021B35
:10022000A2F8DC1030F8021BA2F8D810002500213B
:10023000BCF1000F0ED905EB450606EB051602EBE7
:10024000860606EB410B30F8029B491CABF8529135
:100250006145F6D30021002B0ED905EB450606EBD0
:10026000051602EB860606EB410B30F8029B491C93
:10027000ABF882929942F6D36D1C042DD7D3614618
:100280001846FEF753FEDAF804003E4610F4004F1D
:1002900003D1694600F08CFF0646ED98FCF758FC48
:1002A000EE98FCF7EAFE94F8209094F82150002E86
:1002B0001CBFB9F1000F002D00F0CE809AF80400A9
:1002C00010F0020F04D06A462946484600F015FE99
:1002D0009AF8040010F0050F04D06A4629464846F3
:1002E000FEF764FF9AF8040010F0080F79D0009A26
:1002F000DFF8E4E66846116921F4C051116100217C
:10030000CDF86080CDF85C80002D19D9DEF800C0F2
:1003100000EB4103B3F93632BCF96AC09C450CDAF4
:100320004B0900EB830301F01F0BD3F85CC007FA05
:100330000BFB4CEA0B0CC3F85CC0491CA942E5D38B
:10034000C0F858800021C0F85480B9F1000F19D9C5
:10035000DEF800C000EB4103B3F96633BCF96AC0B4
:100360009C450CDA4B0900EB830301F01F0BD3F81B
:1003700054C007FA0BFB4CEA0B0CC3F854C0491CE1
:100380004945E5D3916BC36D1943436DAB401943A8
:100390009163D16B036E1943836DAB400B43D36301
:1003A000416D202D39BFC5F1200C21FA0CF1A5F1CA
:1003B000200C01FA0CF11943D163416D002904BFEF
:1003C000816D002903D0116941F400611161C16D93
:1003D000002904BF006E002803D0106940F480504B
:1003E00010619AF8040010F0400F0FD16069401CB2
:1003F00060612069002814BFE069A06900F1010074
:1004000014BFE061A0616846FEF717FDC4F80C80D8
:10041000A36800222146A446B3F5056F88BF4FF4B8
:1004200005630020B0EB930F06D25CF82070401CEF
:100430003A44B0EB930FF8D35042C8609AF80400E6
:1004400010F0800F05D14FF47C304FF40562F3F7C4
:1004500099FD2046FEF7F9FB41208DF8B403BEB1AB
:10046000207C8DF8B503607C8DF8B603A07C8DF8F8
:10047000B703E07C8DF8B80300230522EDA907201F
:1004800001F0E3F8CAF808800DF56F7DBDE8F08F44
:10049000FF208DF8B5038DF8B6038DF8B703E9E7B3
:1004A0002DE9F74F84B04FF0000AC2F820A00646AD
:1004B000C2F81CA00598DFF82085174654464FF077
:1004C0000109002821D907EB4400B0F96400002895
:1004D000B8BF404200B2D8F80010B1F938108142DC
:1004E0000FDD610907EB810104F01F03CA6909FAF6
:1004F00003F31A43CA6183B2E1B2FF220420FEF77C
:10050000F3F90598641C8442DDD3002401281CBF44
:100510000598451E46D007EB4403B3F96620B3F9AE
:100520006410501A48BF881A00B2D8F800C0BCF94D
:1005300030C0844533DAB7F9DA00B1EB000C48BFBC
:10054000A0EB010C0FFA8CFC111A48BF811A08B2FB
:10055000844511DB600907EB800004F01F02C169CC
:1005600009FA02F21143C161B3F86430E1B2FF222B
:100570000420FEF7B9F912E0601C410907EB810184
:1005800000F01F0CCA6909FA0CFC42EA0C02CA61AD
:10059000C1B2B3F86630FF220420FEF7A5F9641C4F
:1005A000AC42B8D3D8F8000090F8361000297DD0BE
:1005B00090F837003D68814288BF084600240599BD
:1005C000002984BF401C009070D94FF0010E0098A4
:1005D0004FF000090121CA46012852D9FE4800689F
:1005E0000390B0F93A3004FB066002900EFB0660FF
:1005F000019004FB061005EB4000B0F950C0BCF1BF
:10060000000FB4BFCCF100006046834239DB0EFB23
:10061000061005EB4000B0F950000028B4BF42427C
:10062000024693422DDB029A521A05EB4202B2F9BE
:100630004E80B8F1000FB4BFC8F1000242469342A9
:100640001FDB019A521A05EB4202B2F94E20002A32
:10065000B4BFC2F1000B93469B4512DCA0EB0C0C1F
:100660000398B0F934006045B8BF09F10109A2EB65
:1006700008028242C8BF0AF1010A491C009881425F
:10068000B7D3BAEB090048BFA9EB0A00D249096801
:1006900091F83610884214DB600907EB800004F003
:1006A0001F030121C2699940114300E014E0C161B8
:1006B00007EB4400E1B2B0F86430FF220420FEF7FB
:1006C00013F90598641C844206D2002C18BFA4F1CB
:1006D000010E7FF47CAF78E707B00120BDE8F08F12
:1006E0002DE9F74F064688B0002017681062D061E8
:1006F00090615061B94804900020009001900290F0
:10070000824603900998154647F6FF7BA0F1010940
:10071000A6F10108002871D90024002E69D94FEAFA
:10072000EA700AEBD06020F01F01AAEB0101012260
:1007300002FA01F1401105EB8000CDE906011C3001
:1007400005900AFB064007EB4000BAF1000FB0F934
:10075000500018BFCA450BD1002C18BF444507D123
:100760009D490968B1F99220B1F99010B2B911E030
:100770009949049B09689842B1F98A20B1F9881017
:10078000C4BF0294CDE903A05845BCBF8346CDE960
:10079000004AEBE7904A1268B2F98A2019B98E49EB
:1007A0000968B1F98810904201DC88421EDA069986
:1007B0004FF0010CCA6907990A4305990A60E117CD
:1007C00004EBD1614A1105EB820303F1140221F01D
:1007D0001F015B69611A0CFA01F11943116083B2C0
:1007E000E2B20AF0FF010620FEF77EF8641CB44274
:1007F000A7D309980AF1010A82458DD3764C206867
:10080000B0F88E00002846D00499A1EB0B0181427C
:1008100041DD03980399400905EB800001F01F03B7
:10082000C269012101FA03F31A43C2610198019AD6
:10083000400905EB800002F01F02C36901FA02F2D1
:100840001A43C2610298029A400905EB800002F047
:100850001F02436901FA02F21A4342610098009AAA
:10086000400905EB800002F01F02436991401943E3
:100870004161049883B20298C2B20398C1B20620C3
:10088000FEF732F800981FFA8BF3C2B20198C1B29A
:100890000620FEF729F85048006890F88C000028E0
:1008A00000F032814FF0000A002E7DD90998801E99
:1008B000009007EB4A000999B0F950000024012983
:1008C00073D04FEAEA710AEBD16121F01F02AAEB63
:1008D0000202012303FA02F2491105EB8101CDE97D
:1008E000031214310291611C019101FB06A107EB77
:1008F0004101B1F950B0BBF1000FC8BF00285EDD67
:10090000BBEB000148BFA0EB0B018345CCBF5A46AF
:1009100002464FF44843594391FBF2F101F2FF11B3
:100920004A0A002C1CBF00998C420AD1BAF1000F70
:1009300018BFC24504D12849096891F88D100CE010
:1009400014B100998C4204D12349096891F8991097
:1009500003E02149096891F88C1019B91E4909680A
:1009600091F88C108A422ADDE11704EBD1614A111B
:1009700005EB820221F01F0102F11C03A4EB010C24
:10098000D269012101FA0CF111431960039983B274
:1009900006204A6904990A4302990A600AF0FF0294
:1009A000E1B2FDF7A1FF01E012E00CE001981FFAAF
:1009B0008BF3C1B20AF0FF020620FDF795FF641C1D
:1009C00058464C458FD30AF1010AB245FFF471AF86
:1009D0004FF0000A099803E02C8700100080FFFF09
:1009E000002884BFB01E00907DD90AFB06F007EBFB
:1009F00040000024B0F95000012E7FD04FEAEA7188
:100A00000AEBD16121F01F02AAEB0202012303FAD3
:100A100002F2491105EB8101CDE902121C3101916D
:100A20000AFB064107EB4101B1F952B0BBF1000FDF
:100A3000C8BF00285EDDBBEB000148BFA0EB0B0187
:100A40008345CCBF5A4602464FF44843594391FB75
:100A5000F2F101F2FF114A0ABAF1000F18BFCA45BC
:100A600009D1002C1CBF00998C4205D1FA490968B4
:100A700091F88D100CE014B100998C4204D1F64924
:100A8000096891F8981003E0F349096891F88C100F
:100A900019B9F149096891F88C108A422ADD029946
:100AA0004FF0010CCA6903990A4301990A60E117E2
:100AB00004EBD1614A1105EB820303F1140221F02A
:100AC0001F015B69611A0CFA01F11943116083B2CD
:100AD000E2B20AF0FF010620FDF706FF601C1FFAD4
:100AE0008BF3C2B201E00FE008E00AF0FF0106203C
:100AF000FDF7FAFE641C5846444591D309980AF163
:100B0000010A8245FFF471AF0BB00120BDE8F08F00
:100B10002DE9F74F8AB006460C980C99A6F1010909
:100B20000768002008620C990546C8610C99886125
:100B30000C9948610B98A0F10108002856D90024AF
:100B4000002E4FD9E81705EBD06020F01F01691A7D
:100B5000012202FA01FB41110C9800EB810000F127
:100B60001C0A009005FB064007EB4000002DB0F981
:100B7000501018BF454508D1002C18BF4C4504D172
:100B8000B5480068B0F9B20003E0B3480068B0F9B6
:100B9000B00018B9B0480068B0F9B00081421EDD5D
:100BA00000984FF0010CC06940EA0B00CAF8000041
:100BB000E01704EBD06043110C9A20F01F0002EB09
:100BC000830303F114025B69201A0CFA00F0184346
:100BD00010608BB2E2B2E9B20720FDF785FE641C1B
:100BE000B442BFD30B986D1C8542A8D39A490868BC
:100BF00090F8D120002A1CBF90F8D000002800F007
:100C000078810B980025002840F27381801E08909F
:100C1000B01E02900024002E40F26681A5F1010A68
:100C200000210AFB061007EB40000790681C0190AA
:100C300000FB061007EB40000690E81705EBD060BC
:100C400020F01F01691A012202FA01F105914111F8
:100C50000C9800EB810004901C30039005FB0640CB
:100C600007EB40000090B0F950200B98731EA0F1E4
:100C7000010C0021084645B1012D1CD00AFB06409D
:100C800007EB40000121B0F9500065452DD0DDF89B
:100C900020B05D451FD1002C14BF4FF0000B4FF06A
:100CA000010B4C450CBF4FF0010E4FF0000E5BEAFC
:100CB0000E0B1AD10FE0002C14BF4FF0000B4FF0B9
:100CC000010B4C450CBF4FF0010E4FF0000E5BEADC
:100CD0000E0BDAD1D2E7DDF804B0491C0BFB064B52
:100CE00007EB4B0BBBF950B058443CB1012C1BD067
:100CF000DDF800B0491CBBF94EB058449C4229D0E5
:100D0000DDF808B05C451FD1002D14BF4FF0000B7B
:100D10004FF0010B45450CBF4FF0010E4FF0000E98
:100D20005BEA0E0B16D10FE0002D14BF4FF0000B45
:100D30004FF0010B45450CBF4FF0010E4FF0000E78
:100D40005BEA0E0BDAD1D3E7DDF800B0491CBBF942
:100D500052B05844B5B94CB14FF0010B0BFB064BE8
:100D600007EB4B0B491CBBF94EB058449C4209D0D1
:100D70004FF0010B0BFB064B07EB4B0B491CBBF970
:100D800052B05844654512D13CB10AFB064B07EB03
:100D90004B0B491CBBF94EB058449C4207D00AFB90
:100DA000064B07EB4B0B491CBBF952B0584474B9C6
:100DB000002D18BF65450AD0DDF81CB0891CBBF9B1
:100DC00052B05844DDF818B0BBF952B058449C42B8
:100DD00013D1002D18BF65450FD00AFB064307EB62
:100DE0004303891CB3F94E301844019B03FB0643AF
:100DF00007EB4303B3F94E301844002914BF002A0F
:100E0000FF2310D06423584390FBF1F002EBC201A2
:100E100001EB0211D0EB810059BF1044401E801A33
:100E2000401C90FBF2F3002D18BF45450AD1002C61
:100E300018BF4C4507D10848006890F9D31090F9C5
:100E4000D20021E00CB14C4508D10348006890F96C
:100E5000DD1090F9DC0017E02C870010002D18BF82
:100E6000454504D0012C1CBF0298844206D1FE489F
:100E7000006890F9DF1090F9DE0005E0FA4800689C
:100E800090F9D11090F9D00051EA000C05D1F64844
:100E9000006890F9D11090F9D0008B4201DC8342B8
:100EA0001EDA04984FF0010CC169059801430398BC
:100EB0000160E01704EBD06043110C9920F01F0093
:100EC00001EB830101F114034969201A0CFA00F0C7
:100ED0000843186093B2E2B2E9B20720FDF704FDBF
:100EE000641CB442FFF4BAAE0B986D1C8542FFF44B
:100EF00091AE0DB00120BDE8F08F2DE9F04FD2F892
:100F00000090804689B0D9F81000164620F00F00F6
:100F1000C9F8100047F6FF7003906FEA00000290D6
:100F20004FF0FF00049005904FF000001061F0605A
:100F3000B0605FEA010A09F1500B0546706067D0A6
:100F400005FB08F04FF0000E3BF91010CDE9005EF4
:100F50000A46012017467346B8F1010F19D905FB5F
:100F6000080C3BF91C408C42C4BF21468646BC425B
:100F7000BCBF27460190B4EB020C48BFA2EB040CA7
:100F80000FFA8CF29A42C8BF13462246401C4045D5
:100F9000E5D30298814202DDCDE9045E0291039817
:100FA000874203DA0198039707950690C81B48BF4C
:100FB000781A02B2AC480068B0F91CC0944503DB53
:100FC000B0F91E00834220DDEA1705EBD26253110F
:100FD00006EB830C22F01F020CF10C03AA1A01206D
:100FE000DCF80CC090404CEA000018608BB20EF0A8
:100FF000FF02E9B20520FDF777FC0198BBB2C2B24F
:101000000098C1B20520FDF76FFC6D1C554597D3C4
:101010000025B8F1000F57D93BF91510002086467E
:10102000034600900A46012017460195BAF1010FC8
:1010300019D900FB085C3BF91C408C42C4BF214617
:101040008646BC42BCBF27460090B4EB020C48BFAA
:10105000A2EB040C0FFA8CF29A42C8BF1346224648
:10106000401C5045E5D3C81B48BF781A02B27E48E1
:101070000068B0F920C0944503DBB0F92200834238
:101080001FDDEA1705EBD262531106EB830322F052
:101090001F0203F1040CAA1A01205B689040184358
:1010A0008BB2CCF80000EAB20EF0FF010520FDF78C
:1010B0001BFC0198BBB2C2B20098C1B20520FDF77B
:1010C00013FC6D1C4545A7D3F068002804BF3069A8
:1010D000002805D0D9F8100040F00800C9F8100029
:1010E0007068002804BFB068002805D0D9F8100047
:1010F00040F00400C9F810007168F06801FA0AF1C4
:101100000843C9F82800B168306901FA0AF10843B8
:10111000C9F82C007168BAF1200F39BFCAF120025A
:10112000D140AAF1200291400843C9F82C0003984D
:10113000A9F824000298A9F82600B6F9D810029858
:10114000401A44BF0298081A474C2168B1F9181098
:1011500088420EDDD9F8100040F00200C9F81000F6
:10116000029883B20598C2B20498C1B20520FDF777
:10117000BBFBB6F9D8100398081A44BF0398401A6D
:101180002168B1F91A1088420EDDD9F8100040F03C
:101190000100C9F81000039883B20698C2B20798FC
:1011A000C1B20520FDF7A0FB09B00120BDE8F08F1A
:1011B0002DE9F04F04462D4887B00F4600684FF0E8
:1011C000000890F8F80000F00F0500F0C7FA0128B9
:1011D0000BD040F20F312846F6F788FA012813D0D9
:1011E000002000F0B8FA00F091B900210846F1F7AC
:1011F0007CFCEFF75BFE50B11D48D0F8401341F482
:101200008031C0F8401302E0012000F0A4FA194830
:10121000067819480578002D18BF002E00F074815B
:101220003868002180F8206080F8215080F8221072
:1012300080F82310F2F750FBF1F76AFD00900020D0
:1012400014F0030F18BF0D4814F0200F1CBF40F01E
:10125000F00040F00050DFF81080002876D00099B0
:1012600040F47F0008400BE02C8700100C87001032
:10127000005000404185001042850010070000101A
:1012800014F4407F18BF20F47F00F1F7F8FB04202E
:10129000F7F768FE60F30F09824600210420F7F794
:1012A00058FE0220F7F75EFE60F31F49002102207E
:1012B000F7F74FFE14F4407F17D00020F0F79FF9A6
:1012C00006900020F0F70AFA05900020F0F743FAA4
:1012D00004900020F0F793FB03900020F0F7C7FB89
:1012E00002900020F0F759FF019014F4807F4FF036
:1012F000FF3B2CD0D8F80000B0F8841000291CBFA8
:101300000020F0F790F9D8F8000090F88610002936
:101310001CBF0020F0F733FAD8F8000090F88700DF
:1013200010F00F0F05D000F00F00411E0020F0F765
:1013300080FBD8F8000090F8870010F0F00F38D04C
:101340000BEB10110020F0F7ACFB32E05DE014F481
:10135000007F2ED0D8F80000B0F8AC1000291CBFD8
:101360000020F0F760F9D8F8000090F8AE100029DE
:101370001CBF0020F0F703FAD8F8000090F8AF0087
:1013800010F00F0F05D000F00F00411E0020F0F705
:1013900050FBD8F8000090F8AF0010F0F00F04D028
:1013A0000BEB10110020F0F77CFB00210846F0F752
:1013B000E7FE1F20F6F7A8FFF1F794FA14F4407F38
:1013C00017D000200699F0F72EF900200599F0F7C4
:1013D00094F900200499F0F7D2F900200399F0F76E
:1013E00028FB00200299F0F75CFB00200199F0F740
:1013F000C7FE51460420F7F7ACFD4FEA2941022011
:10140000F7F7A7FD0098F1F73AFB14F02C0F04D082
:101410003A4629463046FEF708FA14F0030F71D019
:1014200000973F68AA46B14607F15005F1F7A0FDC5
:101430008346F1F757FA374CA08810F4407F03D069
:101440000020F0F788F901903248406810F4807F5E
:1014500005D0D8F8000090F8861059B107E010F4D4
:10146000007F07D0D8F8000090F8AE1011B100202E
:10147000F0F785F90020F2F7DCF90026BAF1000F49
:1014800023D906EB4600002400EB061816E01BF9F2
:101490000400262811D2C107490C00EBD07001EBE3
:1014A0008801401001EB800000F1405000F58030D1
:1014B0000068F2F7C4F925F8020B641C4C4501D210
:1014C000262CE4DB761C5645DBD31248808810F4CA
:1014D000407F03D000200199F0F751F90E4C20789D
:1014E0001D280AD107F15000FBF745FC20781D2884
:1014F00004BF07F15000FBF73EFC51464846009AF6
:10150000FDF714FD4FF00108F1F7C5FB07B04046A9
:10151000BDE8F08F10870010C185001070474FF0B4
:10152000FF3070477A484068704779494860704793
:1015300010B584B007280BD14FEA111C012404FA1E
:101540000CFC734C64681CEA040F04BF04B010BDAB
:101550009B0100F00F0043EA800040F001008DF88D
:1015600000008DF801108DF80220100A8DF803009C
:10157000100C8DF80400100E8DF8050000208DF879
:1015800006008DF807000290039068460EF021F8DF
:1015900004B010BD2DE9F04F0E464FF0000185B0AC
:1015A0005FEA02080091019102914FF001024FF0B1
:1015B00006070D460C46039104BF05B0BDE8F08F49
:1015C000EB467B0100F0070943EA890040F0030A7B
:1015D00016F814000BF80200501C36F81420C0B2A4
:1015E000120A0BF80020401CC2B2481CC1B2B9421A
:1015F0000ED1681C85B28DF800A0FF2D94BF28463F
:10160000FF208DF80D0068460DF0E3FF0021012258
:10161000601C84B24445DBD3002904BF05B0BDE89B
:10162000F08F480140EA890040F003008DF8000087
:10163000681C80B2FF2888BFFF208DF80D00684627
:101640000DF0C7FF05B0BDE8F08F10B584B00728D6
:101650000DD191F800C001244FEA1C1C04FA0CFCC7
:101660002B4C64681CEA040F04BF04B010BD9B013E
:1016700000F00F0043EA800040F001008DF8000008
:101680000F2A88BF0F2200206B46002A09D911F8C3
:1016900000C01C18401C84F801C09042F7D30F28EA
:1016A00005D200211A18401C51700F28FAD3184691
:1016B0000DF08FFF04B010BD70B5154E40EA012546
:1016C00002283488224618BF052803D1002918BFF4
:1016D000022900D12C46A24209D051B170880023C2
:1016E00044EA004290210720FFF722FF34807580F2
:1016F00070BDF3F7A0F84FF47A71B0FBF1F044EA53
:101700000042002390210720FFF712FFEEE70000C0
:1017100020870010FE4908707047FD480078704728
:1017200010B50446FCF741FF0146E02220460DF0CB
:1017300055FFF748446010BD58B1F64A0168914220
:1017400007D1406820F00F00B0F5807F04BF012072
:10175000704700207047EE4948707047EC48407869
:10176000704710B5EC48EA4C86B000686178B0F874
:1017700040000429C0F3032008D00421F5F7B6FF88
:1017800001281CBF002060700FD043E000210846F4
:10179000F1F7ABF9EFF78AFB88B1E048D0F84013D6
:1017A00041F48031C0F8401309E004206070052145
:1017B0000020EFF738FF00210846F0F706FA1F2057
:1017C000F6F7A2FD0DF08CFF0DF08FFF0020F4F76F
:1017D0009FF9EFF76BFB10F0010F04BF0120EFF74B
:1017E0001BFEF1F7C3FAFBF77BF801280CD0684623
:1017F000F1F7BFFD28B16846FBF79AFDF1F70AFE45
:10180000F1E7F5F74AFEEEE7F1F76CF80DF06DFF42
:101810000DF070FFF1F73FFA06B010BD2DE9F05F53
:10182000ADF5865DBA4E00200D907088002804BF8B
:101830000DF5865DBDE8F09FB74871780068022914
:10184000006CC0F303253CD0B26840F20F3412F4B0
:10185000007F1EBFC0F303310F290D4612F0800F29
:101860001EBFC0F303110F290D4612F4004F0CD018
:10187000C0F303600F2818BF0546F5F7BDFE0D90B5
:1018800000281CBF0020F5F79CFEB06810F0040F84
:1018900008BF40F20B3410F0020F08BF24F002041E
:1018A00010F0010F08BF24F0010421462846F5F787
:1018B0001DFF012814BF00200220707040F09284A8
:1018C0000DE000210846F1F710F9EFF7EFFA30B11B
:1018D0009248D0F8401341F48031C0F84013F1F73A
:1018E00017FA0E90307A10F0100F18BFF1F7D3FFEF
:1018F000307A10F0080F04BF1F20F6F705FD884866
:101900000778884800780190874890F800808748D9
:10191000007808900198002818BF002F1AD00DF009
:10192000DFFE0DF0E2FEB06810F4803F04BF00203F
:10193000F4F7EEF8B06810F4003F04BF0020F4F7AD
:1019400020F9307A10F0100F0CD00120F4F727F9AD
:1019500001200BE00898002818BFB8F1000FDED175
:1019600000F040BC0020F4F71AF90020F4F717F952
:10197000B06810F4803F18BFF4F757F8B06810F45F
:10198000003F18BFF4F7ECF8EFF790FA10F0010FF2
:1019900004BF0120EFF740FDF1F7E8F91E20FBF747
:1019A000D7F800210846FBF761F8834601210020A3
:1019B000FBF75CF8B468814614F4002F04D04FF4B0
:1019C000BE6114A80DF00FFE14F4800F08D00DF5C1
:1019D000C8604FF4BE610C900DF07DFE00200B90AE
:1019E00014F4000F05D041F23800742168440DF062
:1019F000FAFD0199002079430A911CBF47F6FF7256
:101A0000D14307D02BF8101029F810200A9B401C56
:101A10008342F7D81E20FBF730FB00210120FBF7A3
:101A200025F8044601210846FBF720F8054638480A
:101A3000806810F4801F04D0E8210DF575600DF06A
:101A4000D2FD0899002018EB01061CBF47F6FF7174
:101A5000CA4306D024F8102025F81010401C8642F6
:101A6000F8D82B484FF0000A4088002840F2C68181
:101A70000899781E4144491E109108991390491EF7
:101A8000701C0F91711E4008CDE91101FAF728FF73
:101A9000012800F0B38102A8F1F76BFC002800F0E8
:101AA000A681049800287CD00DF03DFE80461848A1
:101AB000007A10F0100F09D0404604990DF038FE5E
:101AC0000990404508BFDDF810800DE0002000239C
:101AD00000901A46194604980DF02FFE09900C4804
:101AE000007A10F0200F09D1F3F7F6FB019A00926B
:101AF00001463B464046099A0DF024FE0448008901
:101B000010F4804F1EBF09980028F3F713FC0FE074
:101B100028870010545354520C8700100050004086
:101B20004185001042850010468500104785001051
:101B3000FE48D0F808E01EF4004F28D0019800219C
:101B4000002824D900204FF47A73002F09D901FB13
:101B5000070238F912209A42B8BF1346401CB84217
:101B6000F5D301FB07F038F910C00020002F0AD987
:101B700001FB0702401C38F812308742A3EB0C032C
:101B800028F81230F4D80198491C8142DAD3B8F110
:101B9000000F4FD00A99002000294BD938F91010B6
:101BA00000E047E03BF910208A42B8BF2BF8101044
:101BB00039F910208A42C8BF29F810101EF4002FEE
:101BC00015D014AA47F6FF7C32F9102053189C4513
:101BD000DCBF14A921F810C009DD0DF1500C13F57C
:101BE000004FD4BF4FF4004111442CF810101EF4E4
:101BF000800F1BD0B0FBF7F107FB110213998A424B
:101C000014D008EB400138F91030B1F90220991ACC
